:020000040000FA
:10000000021F3F022003FFFFFFFFFF02200BFFFF45
:10001000FFFFFF022013FFFFFFFFFF02201BFFFF78
:10002000FFFFFF022023FFFFFFFFFF02202BFFFF48
:10003000FFFFFF022033FFFFFFFFFF02203BFFFF18
:10004000FFFFFF022043FFFFFFFFFF02204BFFFFE8
:10005000FFFFFF022053FFFFFFFFFF02205BFFFFB8
:10006000FFFFFF022063FFFFFFFFFF02206BFFFF88
:10007000FFFFFF022073FFFFFFFFFF02207BFFFF58
:10008000FFFFFF022083FFFFFFFFFF02208BFFFF28
:10009000FFFF70DFFFFF040000000002000000C847
:1000A000030002030369A5020269A532730000017F
:1000B00000000000000400FFFFFFFFFFFFFFFF0440
:1000C00003090424035400650078006100730020D4
:1000D0000049006E0073007400720075006D0065C9
:1000E000006E007400730024035400490020004394
:1000F000004300320035003300310020005500532A
:10010000004200200043004400430000035F005F02
:100110000030005800000000000000000000000057
:1001200000000000000000000000000000000000CF
:100130000000000000303132333435363738394171
:100140004243444546331C881C881C881C881C90EC
:100150001C74F8121BCD900391E06015900302749B
:10016000FEF0900304744DF0A37405F07A011207B9
:100170001C7F01021D6C74F8121BCD74FF121EB699
:100180007E00801F851882851983E064FE700690CA
:1001900003877401F0851882851983E0F890038441
:1001A000E068F07901AA18AB191210E9E9700302AE
:1001B0000287851882851983E064EF70027E07E06C
:1001C000C0E0900387E0FA900385E0F8EA28F8E4BD
:1001D0003400F9740228F582740339F583D0E0F015
:1001E000900387E0609E14600E14602B14603B1433
:1001F0006051146067809E900384E4F085188285C6
:100200001983E0900386F0C394809003874003E451
:1002100080827402020194851882851983E090031C
:1002200082F09003877403020194851882851983F4
:10023000E0900383F0900386E060199003877404D4
:10024000020194900385E004F0F8900386E0686072
:10025000030201959003877405020194900385E4DD
:10026000F0900387F0900384E0F885188285198365
:10027000E0686003020195900382E0644D60030230
:1002800001951203BF8002EEF97401121E370201BC
:100290007174F7121BCD74FB121EB6EAFEEBFF75EC
:1002A00008047509007808121ED07402121F377AEC
:1002B000907B0079041218EB7402121E3712070E9D
:1002C000121F88E0687003A3E069701285188285A8
:1002D0001983E0F47003A3E0F4600302039A74044A
:1002E000121F2F1207708A088B09A808A909740227
:1002F000121F88E8F0A3E9F07404121F88E0600878
:1003000079011201510203B3851882851983E068CF
:100310007003A3E0697076851882851983E0F47014
:1003200003A3E0F470197402121F887410F0A37410
:1003300020F08518828519837410F0A37420F0755D
:1003400008017509007808121ED07402121F377A4E
:10035000247B0812196F7402121E3775080478087E
:10036000121ED07402121F377A907B007904121883
:10037000EB7402121E3712070E121F88E06870031A
:10038000A3E069700479028006790480027903127F
:1003900001518E828F83741E80058E828F83E4F0DC
:1003A00012070E121F88E0687003A3E069700479D9
:1003B00001800279007405121E377F02021D6C74E1
:1003C000ED121BCD74F8121EB6900307E0FD9003EA
:1003D00006E0FCFAEDF8E4C8F9EA28FEE93408FF83
:1003E000751001750B00750A068E088F0974027866
:1003F00008121F1CC39508F8E49509F9740228F542
:100400000E740339F50F8E088F0974097808121FCE
:100410004EE508F511EE2410F508E43FF509EEF578
:100420000CEF5401F50D900383E014605914700330
:100430000204FB14700302057614601024FE70039E
:100440000206311470030206E10206F1750A03790F
:100450004E1213BD9003071207047402F0A37440F8
:100460001207027408120702F0A3F07418C394076D
:1004700004F510AA10A90B12071CA90A7408121E71
:10048000377F0C021D6C750A04794E1213BDEE45C0
:100490000D7005A9111219D5C3EE9425EF940850DB
:1004A0003CC3E5089424E50994084031E50E249600
:1004B000F8E50F3420F988828983E0701BA3AA82B3
:1004C000AB83E070139003887401F0888289837491
:1004D000A5F08A828B838004900388E4F07508106D
:1004E0007509007808121ED07C087D03EEFAEFFB38
:1004F00012196F7402121E37020473750A05E51192
:10050000C394794006750B0102047375124075138C
:10051000007812121ED07C097D037402780C121F21
:100520001CAA0CAB0DA9111218EB7402121E379005
:100530000307E0A3F0900306E0A3F0751043C3EEB9
:100540009425EF94084003020473C3E5089424E55E
:100550000994085003020473900388E070030204B6
:1005600073E50E2497F8E50F3420F988828983E437
:10057000F0A3F00204737508047509007808121ED0
:10058000D07402121F377A907B0079041218EB7432
:1005900002121E377402121F88E0F8A3E0F98518D2
:1005A00082851983E0687003A3E069851882851944
:1005B00083700BE0F47003A3E0F470578009E0F45B
:1005C0007003A3E0F4700D8518828519837410F010
:1005D000A37420F012070E121F88E8F0A3E9F0754B
:1005E00008017808121ED07402121F377A247B0883
:1005F00012196F7402121E377508047808121ED083
:100600007402121F377A907B0079041218EB74027F
:10061000121E3712070E121F88E0687003A3E069EC
:100620007006750A01020473750A02750B0702044D
:10063000739003D6E0600764026003020473EDFF69
:100640007A01790012071CE060030206D5800312CC
:10065000118512116CE970F77404121F881206F6E6
:100660007404121F887808121F6C85080C85090D08
:10067000850A0E850B0F9003C2780C121EF67404C7
:10068000121F88780C121F5DE5084509450A450BC5
:1006900070CE8EC2E5C554E04FF5C57404121F88B4
:1006A0001206F67404121F887808121F6C85080C55
:1006B00085090D850A0E850B0F9003C2780C121E5A
:1006C000F67404121F88780C121F5DE50845094571
:1006D0000A450B70CE7A01790012071C79080204D2
:1006E0007CEC900391F07003020473750A09020414
:1006F00073790602047CE4F0A37426F0A3E4F0A36B
:10070000F022F0A3E4F0A3F0A3F0A3F0A322851855
:1007100082851983E0F8A3E0F974022274F8121BB1
:10072000CDEAFE900305E0D2E7F0E9A3F0EE9003F6
:1007300003F08E0874042AFE7C028004E062080C38
:10074000ECFA3395E0FB74022AF58274033BF583DF
:10075000EEF8C3EA98EB9400A2D265D03340DDE511
:1007600008F074012AF97A027B0312112702017141
:1007700074E9121BCD7582007583FE121E198A164C
:100780008B177514007515008A828B83E4F0900333
:10079000D6E07006D2AAD2AF800464027005790058
:1007A000120151750C00750D20750E00750F00902B
:1007B00003D6E0600464027015121185120176E917
:1007C000F874096860030208AC7900120151E06412
:1007D000027007A29240030208877508007509029B
:1007E0007808121ED07402121F37850C08850D0977
:1007F000AA08E5095407FB850E0A850F0B740B78D0
:1008000008121E87A9081218EB7402121E377E0008
:100810007F009003CAC0828E10EFF5113395E0F58A
:1008200012F513850C08850D09850E0A850F0B78C6
:10083000087910121F099003C67808121EF67583F6
:1008400003D0827808121DFA501D851882851983FD
:10085000E5822EF582E5833FF583E0F9AA14AB1516
:100860001208DB8A148B150EEE70010FC3EF940291
:1008700040A09003CE780C121EF69003D2780C1292
:100880001DFA40030207AF7900AA14AB151208DB6A
:1008900079001208DB8B159003D6E07004C2AFC25A
:1008A000AAEA451570277AA57BA58021E870030286
:1008B00007CE74066870030207CE740768700302DF
:1008C00007CE8516828517837401F080BA75820081
:1008D000758302121E197F10021D6CC008C0097CAE
:1008E000088A088B09740F7808121F4EE508F8EA89
:1008F00025E0FAEB33FBE9A2E7500474014AFAE879
:10090000A2E0500874216AFA74106BFBE9C333F952
:100910001CEC70CDD009D00822C082C083120F33E6
:1009200060030209F0A3E0F8A3E060030209F0A36A
:10093000E064027002A3E060030209F09003B8E0F3
:100940002480600914604F14605C0209F0E86003C1
:100950000209F09003B2E060047801800278009010
:1009600003C0E8F0A3E4F09003B1E0600A9003C094
:10097000E04402F0A3E4F09003A6E0640460149065
:1009800003B374C0F0A37403F0A3E4F0A3740212E1
:100990000F95F0020E6E90039FE064047052900376
:1009A000C0E4F0A380D0E8547FFA90039FE0640491
:1009B000703EEAC394065038749F2AF582E43403EB
:1009C000F583E854806018A3A3A3A3A3A3A3E064C2
:1009D0000370047801800278009003C0E88094E5F9
:1009E00082240CF58250020583E0640370E980E301
:1009F0009003A67404809B74F8121BCDE9FE90034B
:100A0000BE120F366003020AD990039FE0640460AF
:100A10000B9003BC120F366003020AD99003B8E0B2
:100A2000541F6009146030146020020AD99003BA80
:100A3000E064017022EE9003B1F060047905800259
:100A400079067A00121BCB020ADF9003BCE0547FC8
:100A5000FA9003BAE060057900020AE1EAC394065D
:100A60005077EA90620EF0749F2AF8E43403F9900C
:100A700003BCE05480602EEE600474108002744069
:100A8000906211F0EE60047B0380027B00EB8882B1
:100A90008983A3A3A3A3A3A3A3F0EE600479088092
:100AA0002F7907802BEE60047B2080027B80EB9007
:100AB0006214F0EE60047B0380027B00E8240CF5F6
:100AC00082E439F583EBF0EE6004790A800279095B
:100AD000121BCB90620EE480059003A67404F0799B
:100AE000017F01021D6C79001209F7E97003121BE6
:100AF000BA2279011209F7E97003121BC922C082D8
:100B0000C0839003BC120F367015A3120F36700FFE
:100B10009003BA120CD95480FAE9FBEA4B600790B3
:100B200003A67404801AE8906200F090039F6009A5
:100B3000E06402700C74038007E0640370037402C5
:100B4000F0020E6E74F5121BCD9003BAE0FAA3E02A
:100B50001460081460101460398057121754120C76
:100B6000B6A37B8080417900121776120CB67B8089
:100B7000E92402F9E43AFA121E6DFC1919E0FAA30D
:100B8000E92403F9E43AFA121E6DF9ECA3F0A3E9A3
:100B9000801CEAF91217E49003B3EAF0A3EBF0A388
:100BA000E4120CC5A37B00121E6DA3F0A3E4F002B7
:100BB0000C709003B3E4F0A3F0A3F0750B00900465
:100BC0007DE0FAA3E0FB020C4E850B08750900746A
:100BD000037808121F1CEA2508F8EB3509F9900381
:100BE000BA120CCFE493C0E0EFFCD0E06C705DA3D0
:100BF000E4936E70579003BC120CCFA3A3E493C090
:100C0000E0EFFCD0E06C704488828983A3A3A3E466
:100C1000936E703888828983A3A3A3A3E493F50815
:100C2000740193F5099003B3E508F0A3E509F0A377
:100C30007480F088828983A3A3A3A3A3A3E493F879
:100C4000740193F99003B6E8F0A3E9F0050B900462
:100C50007F120CD9C39AF508E99BF509740378084B
:100C6000121F4EC3E50B9508E495095003020BC90A
:100C70009003B3E0FCA3E0FDA3E0FEEC4D4E900337
:100C8000A6700474048029E0640460259003BEE02B
:100C9000FAA3E0FB9003B6E0F8A3E0F9C3EA98EB0F
:100CA0009950089003B6EAF0A3EBF09003A6740104
:100CB000F07F04021D6C9003B3EAF0A3EBF0A37481
:100CC00080120CC522F09003B3E0F9A3E0FA22E011
:100CD000FEA3E0FF8882898322E0F8A3E0F9E822FE
:100CE00074EE121BCDEA2404F8E43BF98808890964
:100CF0008882F583E4936025900481120CD9FEE983
:100D0000FF8007EE2404FE50010F8E828F83E49350
:100D1000F8740193F9EA687002EB6970E6750B00EC
:100D2000803F9062147490F07410120E3570037549
:100D30000A408E828F83A3A3A3E493550E6006E539
:100D40000AD2E0F50AE50A906215F0EA906213F023
:100D5000EC240CF582E43DF583E4F090620EF0059E
:100D60000B850882850983E493F8E50BC39840035B
:100D7000020E307A0079051216E78A0C8B0DEA45CF
:100D80000D60DCEA2402F8E4350DF9881089118839
:100D900082F583E493540FF51290620EF0750A0009
:100DA0008A828B83A3A3A3A3E4932407F50EA3E471
:100DB000933400F50F7403780E121F4EAA0EA8127A
:100DC000749F28F8E43403F9E8FCE9FD750E017519
:100DD0000F00E512780E121F1CE50EF50EE50C242F
:100DE00003F8E4350DF9851082851183E493A2E7B9
:100DF0004003020D229062117448F07408120E35FF
:100E00007003750A408E828F83A3A3E493550E600E
:100E100006E50AD2E0F50AE50A906212F0EA90626D
:100E200010F08C828D83A3A3A3A3A3A3A3020D59C7
:100E30007F0B021D6CF088828983E4935403640164
:100E400022C082C083120F337010A3120F36700AB3
:100E5000A3E064017002A3E060079003A67404801D
:100E60000C9003B374A0F0A37403120F8BF0D08323
:100E7000D0822274F3121BCD90039FE064026014B1
:100E80009003BC120F36700CA3120F36700690033D
:100E9000BBE060099003A67404F0020F2E7A00797B
:100EA00001121BCB9003BAE0606F7A00F91217763B
:100EB0008A0A8B0BEA450B605890039F7404F090EC
:100EC00003BAE09003A0F0750800850A82850B83C1
:100ED000A3A3A3A3E493F8E508C398504AA8087411
:100EE000A128F8E43403F9E8FEE9FF8E828F83E459
:100EF000F07A0079041216E78A828B83A3A3A3E415
:100F000093F88E828F83E06870E7120CE00508800A
:100F1000B99003A67404F0800E9003A0F090039F94
:100F20007403F0F91216677A007902121BCB7F0660
:100F3000021D6C9003BAE0F8A3E0F9E8492274F6C8
:100F4000121BCD90039FE0640470199003B8E06415
:100F5000817011120F33700C9003BEE064017002B7
:100F6000A3E060079003A67404801A9003BCE024F9
:100F7000A1F508A3E03403F5099003B3E508F0A355
:100F8000E509120F8BF07F03021D6CF0A3E4F0A3C0
:100F900004120F9522F0A3E4F09003A6042274F744
:100FA000121BCD90039FE0640470649003B8E0646A
:100FB00001705C9003BE120F3670549003BAE0FBD0
:100FC0009003BCE0FA9003A0E0F91217AE8A088BF8
:100FD00009AE08AF09EE4F60369003BCE0FA790322
:100FE000121BCB9003BAE0C0E09003BCE024A1F850
:100FF000A3E03403F988828983D0E0F0EEFAEFFBB6
:10100000120CE09003BCE0FA7904121BCB8006902E
:1010100003A67404F07F02021D6CC082C0838003AB
:10102000121A31A2E840F9A823E854046009782391
:10103000E654FBF612140EA823E854106009782336
:10104000E654EFF612142FA823E8A2E05005782307
:1010500054FCF690620EE0FA7404F0906214E0A280
:10106000E05039A9A8C2AF906216E0F8A3E0E8FB0F
:10107000E9A2E792AF8017906228E0C0E090039366
:10108000E0F812111CD0E0F0900393E004F0EBFDC7
:1010900074FF2DFB0470E0906214E4F0EA90620E9D
:1010A000F0E0FC7404F0906211E0A2E040319003A3
:1010B00095E0F8900394E06860257A4090039412DC
:1010C000115FE0906228F0900394E004F008900330
:1010D00095E06860041AEA70E39062117401F0EC24
:1010E00090620EF0D083D0822274F8121BCDE9FEFC
:1010F0007900801212111CE08A828B83F090039297
:10110000E00412115409900392E0F8900393E06810
:101110006005E9C39E40DD7F01021D6C748528F5E2
:1011200082E43404F58322C082C083E9FC80188AFB
:10113000828B83E0C0E090039512115FD0E0121122
:1011400054900395E004F0ECF874FF28FC0470DF81
:1011500079018090F08A828B83A3AA82AB8322E0FC
:10116000F8748528F582E43405F58322C082C083B3
:10117000900395E0F8900394E068600479018002A0
:1011800079000210E402101A74FB121EB67E009061
:1011900006857808121F6C794A1213BD9006857473
:1011A00001F0A3F0A37469F0A374A5F09003D778BD
:1011B00008121EE170047E0180159003DB7808128E
:1011C0001EE16008E59D541864107003022000EED3
:1011D000F9121334C280D291EEA2E050030212E75A
:1011E000AA18AB19120291E970030212E7C29185A5
:1011F0001882851983E0C3943C500EE0F8743CC318
:1012000098F50895E0F5098006750800750900E471
:10121000F50AF50B9003DF780C121F6C7808790C37
:10122000121AD1790612015112101A120176E9F838
:101230007409687007790612015180277407686085
:1012400016A2935012E8600874066860030212E761
:10125000A292400F0212E7750800750900750A0096
:10126000750B0085080C85090D850A0E850B0F90FE
:1012700003C27808121EF6E50C450D450E450F70A9
:10128000A7D2807907120151800312101A12116C33
:10129000E970F77E007F007401121F88E4F0A374E8
:1012A00026F0A3E4F0A3F07401121F887808121F3F
:1012B0006C85080C85090D850A0E850B0F9003C2FD
:1012C000780C121EF67401121F88780C121F5DE54F
:1012D000084509450A450B70CEA29250FCA29350D6
:1012E000F81213B8022000D280D291794E1213BDA9
:1012F000750800750900750A00750B007905120163
:101300005112101A120176E9F874096860EE74013E
:101310006870EE12101A9003E37808121EF690031C
:10132000E77808121DFA50EB1213B802200074057A
:10133000121E372274F8121BCDE9FE53BEFBE59D49
:10134000A2E650FA0078F8790100E824FF18E934A1
:10135000FFF9E84970F375C6807480659E70FA43A2
:10136000BE049062707408F01213ADEE700853F46E
:10137000FEC29043FE017403F5D575D4899003969F
:10138000E4F0A374C2F0A37401F0A3E4F0A3F0A30B
:10139000F0A37408F01213D37AFF7BFF1219EC53F9
:1013A000F4FED29043FE011213AD021117D2804316
:1013B000FD01C29143FE0222D280C29122781075B3
:1013C000B60FE5B4A2E750FAE5BBC39940F118E8BF
:1013D00070ED2274F7121BCD7A0079011217768A0C
:1013E000828B83A3A3A3A3A3A3A3E493A2E6900366
:1013F000B2500474018001E4F09003B1E4F0906213
:101400000F7403F0E0A2E750FB7F02021D6CC08264
:10141000C08390039F7402F0A3E4F09003A6F079D8
:1014200003121667752100752200D083D0822274C2
:10143000F6121BCD90620EE0FEE4F0906211E0FF28
:10144000A2E4501D7480F09003A67407F0E52145D6
:10145000226009852182852283121F979003A6E4CA
:10146000F0EFA2E2500B906211E4F09003A6F0803E
:10147000679003A6E0F87402687046906216E0FF79
:101480009003B3121DACEFF97A207B6212168174BF
:1014900003121E37EFF89003B612164512164F2F9F
:1014A000121657A3E0F8A3E0F9E8496004744080FD
:1014B000027448906211F0E849600302163B02167C
:1014C000177406687009852182852283121F979000
:1014D00003A6E060030215C2EFA2E0400302163B40
:1014E0007508B8750903750A007808121ECC7908CA
:1014F0007A207B621216817403121E3775210075E3
:1015000022009003B8E054E0601D24E0700302154F
:101510009D24E0607224C0604824E070030215A896
:1015200024E0606E0215B3A3E014602624FE601D63
:1015300024FE600A24FC601F24FE60208075120ACD
:10154000FE9003A6E06404707278608070120AF264
:1015500080EF120AE680EA120E7380E5120F9E8079
:10156000E0A3E0600E24FA600F24FE601024FE6009
:1015700011804012091980C9120B4480C4120E4117
:1015800080BF120F3E80BA7521B675221B121BB6A2
:1015900080AF7521B875221B121BB880A47521512C
:1015A00075221B121B51809975218175221B121BFC
:1015B00081808E9003A67404F0808E7840E890625B
:1015C00011F09003A6E0F874016870617F02900347
:1015D000B6E0F8A3E0F9C3E89420E994005007E8E6
:1015E000F5087F0A80037508209003B3121DACA98B
:1015F000087A207B621216AC7403121E37AC0812F4
:10160000164F2C121657A808A3121645EF90621118
:10161000F0E8C394205024E5214522600985218209
:10162000852283121F979003A6E4F0800E7405684C
:101630007009852182852283121F97EE90620EF039
:101640007F03021D6CC3E098F0A3E09400F02290A9
:1016500003B31216D9E922F9E43AFA9003B3E9F098
:10166000A3EAF0A3EBF022C082C083E99003A7783D
:1016700005F0A3D8FC9003AC7805F0A3D8FC0214C5
:101680002A74F8121BCDEAFCEBFDE9F87408121F6E
:10169000881216D460118C828D83E0121EA0E9247A
:1016A0000109E43AFAD8EF7F01021D6C74F8121BAD
:1016B000CDEAFCEBFDE9F87408121F881216D4601D
:1016C00011121E6D8C828D83F0E9240109E43AFA2F
:1016D000D8EF80D31216D9E822E0F9A3E0FAA3E00C
:1016E000FB22D083D08222C082C083E9FCEAFD7A4B
:1016F000007B00800312173290039DE0F8A3E0F90D
:1017000090047BE0687003A3E069602490039EE08E
:10171000F5838882A3E493F8EC68700D90039DE054
:10172000FAA3E0FB1217328007ED6870C8ED60C5C0
:1017300080B090039DE0F8A3E0F5838882E493F8FD
:1017400090039DE028F8A3E03400F990039DE8F0B1
:10175000A3E9F022C082C0831217657A00790112D2
:1017600016E70216E2900479E0F8A3E0F990039DF1
:10177000E8F0A3E9F02274F7121BCDE9FFEAFE12AC
:1017800017657A0079021216E7EA4B601CEF6010C9
:101790008A828B83A3A3A3A3A3E4936F70E480093D
:1017A000EEF874FF28FE0470D97F02021D6C74F5F8
:1017B000121BCDEAFF8B087A001217767A027904A1
:1017C0001216E7EA4B60188A828B83A3A3E4936F17
:1017D00070EA8A828B83A3A3A3E493650870DD7FFC
:1017E00004021D6C74F7121BCD74F0121EB6E97A58
:1017F000007B00600C146010146014146018021850
:10180000D47AF37B030218D47AF77B030218D47AD4
:101810001B7B040218D490043FE060030218D090B0
:1018200003EB7408121F377408121DD9750808F5E8
:10183000097808121ED07402121F377AE87B0779E4
:101840007F1218EB7402121E377808121ED0740A29
:10185000121F377402121F2F121C907402121E37AF
:101860008B09EA450970197509007808121ED07CA9
:101870000C7D787402121F2F121D267402121E375F
:101880007C287D00EDF8851882851983E58228F58E
:1018900082E43583F583E0FFECF8743F28F8E43404
:1018A00004F9EF1218DC88828983F0EFC41218DC87
:1018B000C0E0E824FEF582E934FFF583D0E0F00DC6
:1018C00074FC2CFCEDC3940840BA90043F742AF0D9
:1018D0007A3F7B047410121E370217A9540FFA7452
:1018E000692AF582E43404F583E02274F6121BCDF4
:1018F000890A740F550AF508750900740B780812E7
:101900001F1CEA2400F8EB3480F9E82400E93509CB
:10191000F985C709A2AFE433F508C2AFE50AC4549C
:101920000FFAE5C754F84AF5C7740A121F88E0FA9F
:10193000A3E0FB801C88828983E08C828D83F08801
:10194000828983A3A882A9838C828D83A3AC82AD74
:1019500083EAFEEBFFEE24FF1AEF34FFFBEE4F703D
:10196000D48509C7E508A2E092AF7F03021D6C741D
:10197000F7121BCDED900389F0ECA3F0A37462F095
:10198000A37473F0A3E0541FF07409121F88E0F5EC
:1019900008A3E0F509E508333354FC90038EF07496
:1019A000067808121F4EE50890038DF090038F749F
:1019B00012F0A37442F075D1FE75D601EA906271FF
:1019C000F0EBA3F0906270E0D2E1F0E0A2E740FB20
:1019D0007F02021D6CC082C083E9C333906272F043
:1019E000906270E0D2E0F0D083D0822274F7121BB4
:1019F000CD7523007524007525008A268B27EA9073
:101A0000620BF08A088B0974047808121F4EE508EF
:101A1000906207F08A088B0974097808121F4EE556
:101A200008543E906209F0758B00C2E87F02021DE7
:101A30006C74F7121BCDE59DA2E650FA906206E0A9
:101A4000F9A2E25034AA26EA90620BF0F508852745
:101A50000974047808121F4EE508906207F08A089E
:101A600085270974097808121F4EE508543E9062D4
:101A700009F0906201E0D2E0F0E9782346F6906246
:101A800002E0F50875090074047808121F1C782319
:101A9000E50846F608E50946F6906204E0F50875A3
:101AA000090074097808121F1C7824E50946F6E934
:101AB000A2E050037525017406596003752500E501
:101AC0008BA2E55006758BDF752500121BCC021A20
:101AD00027080808EAC0E0EBC0E086F0E7A4FA189F
:101AE0000986F0E7A42AFA180986F0E7A42AFA186A
:101AF0000986F0E7A42AFA1986F0E7A4FBE5F02AA4
:101B0000FA190886F0E7A42BFBE5F03AFA190886E3
:101B1000F0E7A42BFBE5F03AFA18180986F0E7A4E1
:101B2000C5F02BFBE43AFA1908E7C5F0C6A426F67F
:101B3000E5F03BFBE43AFA1886F0E7A4F6E5F00896
:101B400026F6E43B08F6E43A08F6D0E0FBD0E0FAEB
:101B500022C082C0839003B9E0F8742268700890B4
:101B600003A6E0701A80117420689003A6700DE03F
:101B7000700D121BA89003A6740280027404F080FA
:101B800043C082C0839003B9E064219003A6701320
:101B9000E07013121BA8A37407F0A3E4F09003A64F
:101BA0000480027404F0801C9003B37496F0A37454
:101BB00003F0A3E4F02280028000C082C08390037F
:101BC000A67404F0D083D0822280EF22222518C58B
:101BD00082C0E0E51934FFC583C0E0E518C39582F3
:101BE00024F910AF08858319858218800885831928
:101BF000858218D2AFCEF0A3E520F0A37808E608DE
:101C0000F0A3DEFAEFF0A3E58124FBF8E608F0A3E9
:101C1000E608F0A30808E608F0A3E608F0A315819B
:101C20001581D0E0FED0E0F815811581E8C0E0EE26
:101C3000C0E02212010002020000205104A816098F
:101C40000001020301090243000201008019090496
:101C50000000010202010005240010010424020218
:101C60000524060001052401000107058203400048
:101C70004009040100020A00000007058402400038
:101C800000070504024000004E1C0000711C00000B
:101C900074F8121BCD7408121F88E0FEA3E08015B3
:101CA000A3AA82AB838C828D83A3AC82AD83EE2406
:101CB000FF1EEF34FFFFEE4F60198C828D83E0F83A
:101CC0008A828B83E0F9E86960D6E9C398FA95E0E7
:101CD000FB80047A007B007F01021D6CE47921788F
:101CE00007B800028004F709D8FCE490030278C129
:101CF00079018002F0A3D8FCD9FA7AC27B03900064
:101D00008E78C479018015E493A3AD82AE838A8274
:101D10008B83F0A3AA82AB838D828E83D8E9D9E727
:101D2000121188121F9274F7121BCDEAF8EBF974A6
:101D300009121F88E0FEA3E0FF80188C828D83E0EB
:101D400088828983F0A3A882A9838C828D83A3AC27
:101D500082AD838E088F09E50824FF1EE50934FF54
:101D6000FFE508450970D47F02021D6C8519838543
:101D70001882E0A3FEE0A3F5207808E0A3F608DFD0
:101D8000FAE0A3FFE0A3C0E0E0A3C0E0E0A3C0E06E
:101D9000E0A3C0E010AF088582188583198008850C
:101DA0008218858319D2AFD083D082227403800039
:101DB000CCC0E0EDC0E0E518C39CCCAD1950011DCE
:101DC00010AF068C188D1980068C188D19D2AF12A1
:101DD0001DD9D0E0FDD0E0FC22CAC0E0E0A3C5825E
:101DE000CCC582C583CDC583F0A3C582CCC582C5D1
:101DF00083CDC583DAE6D0E0CA22C008C3E096F5F9
:101E00000808A3E096420808A3E096420808A3E069
:101E10009645087001D3D00822C5822518C582C511
:101E200083351910AF07F5198582188007F51985D4
:101E30008218D2AFC5832200C0D0251810AF08F594
:101E400018500C05198008F51850020519D2AFD0AA
:101E5000D0222518F58210AF08F518400C1519800E
:101E600008F51840021519D2AF85198322BB01026B
:101E7000E722C082C08389828A83BB0003E080029C
:101E8000E493D083D082226016080808C6C313C624
:101E900018C613C618C613C618C613C6D5E0EA225C
:101EA000BB000EC082C0838A838982F0D083D08237
:101EB00022BB0101F722251810AF08F518400C15B8
:101EC000198008F51840021519D2AF227403800456
:101ED00074028000C0E0F404121E52D0E0121F7B96
:101EE00022E066701008A3E066700A08A3E066703E
:101EF0000408A3E06622E026F608A3E036F608A36D
:101F0000E036F608A3E036F622E627F60809E637BB
:101F1000F60809E637F60809E637F622700422606B
:101F20000D18C6C333C608C633C6D5E0F41822253B
:101F300018FAE43519FB222518FCE43519FD227541
:101F4000D00075813F751802751903021CDC600C06
:101F500008C6C313C618C613C6D5E0F422E6F008B7
:101F6000A3E6F008A3E6F008A3E6F022E0F608A353
:101F7000E0F608A3E0F608A3E0F622CAC0E0E6F027
:101F8000A308DAFAD0E0FA222518F582E43519F52B
:101F9000832200000080FBE473FFFFFFFFFFFFFFD1
:101FA000FFFFFFFFFFFFFFFFFFFFFFFFFFFFFFFF41
:101FB000FFFFFFFFFFFFFFFFFFFFFFFFFFFFFFFF31
:101FC000FFFFFFFFFFFFFFFFFFFFFFFFFFFFFFFF21
:101FD000FFFFFFFFFFFFFFFFFFFFFFFFFFFFFFFF11
:101FE000FFFFFFFFFFFFFFFFFFFFFFFFFFFFFFFF01
:0A1FF600850609433886000000004C
:020000040003F7
:01FFF000F020
:020000040000FA
:10200000022DC4022233FFFFFFFFFFFFFFFFFFFF90
:10201000FFFFFFFFFFFFFFFFFFFFFFFFFFFFFFFFD0
:10202000FFFFFFFFFFFFFFFFFFFFFF022B3AFFFF56
:10203000FFFFFF022255FFFFFFFFFFFFFFFFFFFF34
:10204000FFFFFFFFFFFFFFFFFFFFFFFFFFFFFFFFA0
:10205000FFFFFF02216DFFFFFFFFFFFFFFFFFFFFFD
:10206000FFFFFFFFFFFFFFFFFFFFFF022A54FFFFFD
:10207000FFFFFFFFFFFFFFFFFFFFFF0228A5FFFF9E
:10208000FFFFFF0221C401FFFFFFFFFFFFFFFFFF74
:1020900010201020010020FD000200000D32000081
:1020A0000000A7319132DD314F320000D131000004
:1020B0000000000000000000000000000000000020
:1020C00000000000000006FFFFFF00035F005F004C
:1020D0003000580000000000000000000000000078
:1020E00000000000000000000000000000000000F0
:1020F00000000000C42619271927192719272127AE
:10210000010104007918000000E8030000FFFF4807
:102110001903E803000064006400B801A0BB0D00CF
:10212000A0BB0D0002020008000005020704010523
:102130001E02051E020A0A01080803B80B02803EAF
:102140000102FEFFE8030A050001FFFF0A1401E097
:10215000010105030101FF0F10FEFF004F00000009
:1021600000724D00000000FF000000FF00C0E0749E
:10217000F2122665A2AFE433F508D2AFAFA7AEA145
:10218000EE5F54106006122F2B75A1EFEE5F54081E
:102190006008122F3175A1F78023EEA2E092F0EFD4
:1021A000A2E082F05017906198E0F890054EE0C3ED
:1021B00098A2D265D0335002E8F075A1FE751A00DE
:1021C000E5088066C0E074F2122665A2AFE433FE33
:1021D000D2AF9061A4E0F8759B00E5915854086077
:1021E000087591F7122F798023E5915854106008F3
:1021F0007591EF122F7F8014E591A2E092F0E8A292
:10220000E082F05007E0C2E0F01230D59061A3E028
:10221000F8E5E9585404600E1230AB75E9FB9061A3
:1022200093E0A2E640F2751A00EEA2E092AF7F01C1
:10223000022721C0E074F2122665A2AFE433FED279
:10224000AF9061A5E0F8E5BF585404600675BFFB88
:102250001230ED80D1C0E074F1122665E59DA2E652
:1022600050FA906206E0F9A2E25034AA2CEA906299
:102270000BF0F508852D0974047808122DE3E508A4
:10228000906207F08A08852D0974097808122DE3F9
:10229000E508543E906209F0906201E0D2E0F0E976
:1022A000782946F6906202E0F50875090074047812
:1022B00008122D147829E50846F608E50946F69037
:1022C0006204E0F50875090074097808122D147885
:1022D0002AE50946F6E9A2E05003752B0174065978
:1022E0006003752B00E58BA2E55006758BDF752B1F
:1022F0000012361B758B00C2E87F02022721C3E45F
:1023000098F8E499F912233F8026C3E49AFAE49BF3
:10231000FBE920E7E912233FE498F8E499F922C3A6
:10232000E498F8E499F912233FE498F8E499F9C3A2
:10233000E49AFAE49BFB22EB20E7CFE920E7E0B93F
:102340000010BB0008E88AF084F8AAF022E4FBC879
:10235000FA22EB70227B10C833C8C933C933500747
:10236000C39AC3DBF280069A50012ADBEAC833F431
:10237000C8C933F4C9FA2275F008E4C833C8C933B0
:10238000C933C99AC99B5004C92AC93BD5F0ECFB93
:10239000C833F4C8E4C9FA2274F51225FF74FA129E
:1023A0002C0B7508047509007808122B7A74041236
:1023B0002BEB7AF87B0779031249DD7402122B8D1F
:1023C0009081227808122DD47402122E617808129E
:1023D0002C6270487508027509007808122B7A740F
:1023E00002122BEB7AF67B0779031249DD74021295
:1023F0002B8D851882851983E0F47003A3E0F460C7
:102400001B851882851983E0F8A3E08882F5837420
:1024100002F0A3F0A37469F0A374A5F0C2AF75D65F
:102420009F0200007406122B8D7F040228E8080822
:1024300008EAC0E0EBC0E086F0E7A4FA180986F0ED
:10244000E7A42AFA180986F0E7A42AFA180986F000
:10245000E7A42AFA1986F0E7A4FBE5F02AFA19089E
:1024600086F0E7A42BFBE5F03AFA190886F0E7A41A
:102470002BFBE5F03AFA18180986F0E7A4C5F02B13
:10248000FBE43AFA1908E7C5F0C6A426F6E5F03BE6
:10249000FBE43AFA1886F0E7A4F6E5F00826F6E43D
:1024A0003B08F6E43A08F6D0E0FBD0E0FA22122E20
:1024B00056B9000302250EE47921780DB800028098
:1024C00004F709D8FCE49004D1785779188002F019
:1024D000A3D8FCD9FA781A9020867A01BA00028033
:1024E00007E493A3F608DAF97A277B1C9020947806
:1024F000DA79018015E493A3AD82AE838A828B835F
:10250000F0A3AA82AB838D828E83D8E9D9E7758246
:102510007D7583B77406122B1C75826F75834B749F
:1025200000122B1CE4CFC0E0E4CEC0E0E4CDC0E05C
:10253000E4CCC0E075F020E626F608E633F608E6BF
:1025400033F608E633F6181818EC33FCED33FDEEDD
:1025500033FEEF33FFC3EC9709ED9709EE9709EFD0
:1025600097191919400FFFEC97FC09ED97FD09EE3B
:1025700097FE191906D5F0BFECF709EDF709EEF74C
:1025800009EFF7191919D0E0FCD0E0FDD0E0FED03A
:10259000E0FF222518C582C0E0E51934FFC583C0DD
:1025A000E0E518C3958224F810AF08858319858269
:1025B000188008858319858218D2AFCEF0A3E52054
:1025C000F0A37808E608F0A3DEFAEFF0A3E5812493
:1025D000FAF8E608F0A3E608F0A3E608F0A3080876
:1025E000E608F0A3E608F0A315811581D0E0FED03F
:1025F000E0F8158115811581E8C0E0EEC0E02225E4
:1026000018C582C0E0E51934FFC583C0E0E518C3F2
:10261000958224F910AF0885831985821880088572
:102620008319858218D2AFCEF0A3E520F0A37808F5
:10263000E608F0A3DEFAEFF0A3E58124FBF8E60854
:10264000F0A3E608F0A30808E608F0A3E608F0A364
:1026500015811581D0E0FED0E0F815811581E8C024
:10266000E0EEC0E022C0D02518C582C0E0E51934F4
:10267000FFC583C0E0E518C3958224F310AF088539
:1026800083198582188008858319858218D2AFC87E
:10269000F0A3E9F0A3EAF0A3EBF0A37908E709F0CF
:1026A000A3D8FAECF0A3EDF0A3EEF0A3EFF0A3D0E3
:1026B000E0F0A3D0E0F0A3D0E0F0A3E520F0A3E5A4
:1026C000F0F0A32212010002020000205104A8161B
:1026D00009000102030109024300020100801909F7
:1026E000040000010202010005240010010424027C
:1026F00002052406000105240100010705820340AC
:10270000004009040100020A00000007058402409D
:10271000000007050402400000DF26000002270039
:1027200000851983851882E0C0E0A3E0F9A3E0FAF0
:10273000A3E0FBA37808E0F608A3DFFAE0FCA3E03F
:10274000FDA3E0FEA3E0FFA3E0C0E0A3E0C0E0A3A0
:10275000E0F5D0A3E0F520A3E0A3F5F010AF0885E5
:1027600083198582188008858319858218D2AFD095
:1027700082D083D0E0F8D0E032E4731E75F0108E82
:10278000218F22858226858325851882851983E0FD
:10279000CEA3E0CF852682852583EBC9EAC8EDCBA1
:1027A000ECCAC3E833C8E933C9EA33CAEB33CBC355
:1027B000EA9EF524EB9FF523B35004AB23AA24EC47
:1027C00033CCED33CDD5F0DAAE21AF2222D083D099
:1027D00082ECC0E0EDC0E0E493A3FCE493A3FDED44
:1027E0004C600D122928EC24FFFCED34FFFD80EF36
:1027F000E493A3FCE493A3FDED4C600D1229FFECE0
:1028000024FFFCED34FFFD80EFD0E0FDD0E0FCE4E0
:1028100093A3C0E0E493C0E022851983851882E089
:10282000A3FEE0A3F5207808E0A3F608DFFAE0A312
:10283000FFE0A3C0E0E0A3C0E0E0A3C0E0E0A3C0ED
:10284000E0E0A3C0E010AF088582188583198008F6
:10285000858218858319D2AFD083D082022B22D0F3
:1028600083D082E9C0E0E493A3C386F0C5F095F07D
:10287000F908E493A386F0C5F095F0700BE493A3F8
:10288000C3994005E9048002A3E475F002A42582FF
:10289000F582E5F03583F583D0E0F9E493A3C0E059
:1028A000E493C0E022C0E074F2122665A2AFE433E4
:1028B000FED2AFE58AA2E2500790050FE0D2E0F029
:1028C000E58AA2E3500790050FE0D2E1F0758A0097
:1028D000C2EB7A107B0090050BE0F91233BDEEA23B
:1028E000E092AF7F01022721851983851882E0A33A
:1028F000FEE0A3F5207808E0A3F608DFFAE0A3FFE6
:10290000E0A3C0E0E0A3C0E0E0A3C0E0E0A3C0E03B
:1029100010AF088582188583198008858218858301
:1029200019D2AFD083D08222C0E0C3E4939608745A
:1029300001939618400FE49366700808740193663B
:102940001870007019A3A3C3E493960874019396BA
:1029500018A3A3400DD0E0D0E0D0E0022809A3A343
:10296000A3A3A3A3D0E022D083D082C5F0E493A395
:10297000C5F0C395F0F5F0E493A3C395F04005E5E9
:10298000F0048001E475F002A42582F582E5F035BB
:1029900083F583E493A3C0E0E493C0E02274048051
:1029A000087403800474028000CCC0E0EDC0E0E550
:1029B00018C39CCCAD1950011D10AF068C188D1991
:1029C00080068C188D19D2AF122A9ED0E0FDD0E07F
:1029D000FC2274028000CCC0E0EDC0E0E518C39C8E
:1029E000CCAD1950011D10AF068C188D1980068CC6
:1029F000188D19D2AF122A7CD0E0FDD0E0FC22C0A5
:102A0000E0C0F088F0E493667008087401936618DB
:102A10007000A8F0A3A3700BD0F0D0E0D0E0D0E01D
:102A2000022809A3A3D0F0D0E022D083D082CCC06A
:102A3000E0E493A36006122ABF1470FAE493A36043
:102A400006122C371470FAD0E0FCE493A3C0E0E443
:102A500093C0E022C0E074F2122665758900C2C5F9
:102A60009019F5E0700E7A007B109005E4E0F91201
:102A700033BD8003123CC97F01022721CAC0E0E4B4
:102A800093A3C582CCC582C583CDC583F0A3C5827F
:102A9000CCC582C583CDC583DAE5D0E0CA22CAC0E1
:102AA000E0E0A3C582CCC582C583CDC583F0A3C5B4
:102AB00082CCC582C583CDC583DAE6D0E0CA22C008
:102AC000E0E493A3D39C5010E493A3C39C400AD0AA
:102AD000E0D0E0D0E0022A47A3A3A3D0E02270090F
:102AE000080808226016181818C6C333C608C6336B
:102AF000C608C633C608C633C6D5E0EA22C008C336
:102B0000E096F50808A3E096420808A3E09642087C
:102B100008A3E09645087001D3D00822C09FF59F16
:102B2000E473D09F22D083D082C09FE493C0E0742E
:102B30000193C0E0740293F59F22C0E0C0D0E8C0CA
:102B4000E0A8A8D2AFC2C7751A00E8A2E792AFD03A
:102B5000E0F8D0D0D0E0322518F58210AF08F51893
:102B6000400C15198008F51840021519D2AF8519C7
:102B700083227404800A7403800674028002740144
:102B8000C0E0F404122B57D0E0122E012200C0D076
:102B9000251810AF08F518500C05198008F51850C5
:102BA000020519D2AFD0D022BB0102E722C082C0F9
:102BB0008389828A83BB0003E08002E493D083D0C0
:102BC00082226016080808C6C313C618C613C618A2
:102BD000C613C618C613C6D5E0EA222518F8E43590
:102BE00019F9222518FAE43519FB222518FCE435D9
:102BF00019FD22C3E0C696F608A3E0C696F608A320
:102C0000E0C696F608A3E0C696F622251810AF088F
:102C1000F518400C15198008F51840021519D2AFA7
:102C200022BB000EC082C0838A838982F0D083D009
:102C30008222BB0101F722C0E0E493A36C7009D0AB
:102C4000E0D0E0D0E0022A47A3A3D0E022E76670FC
:102C5000100809E766700A0809E76670040809E7C2
:102C60006622E066701008A3E066700A08A3E066BA
:102C7000700408A3E06622C3E09608A3E09608A3C8
:102C8000E09608A3E096A2D265D03322C3E697F679
:102C90000809E697F60809E697F60809E697F62286
:102CA000C3E493960874019396087402939608748B
:102CB00003939622C3E096F008A3E096F008A3E001
:102CC00096F008A3E096F022E026F008A3E036F0A4
:102CD00008A3E036F008A3E036F022E647F608093C
:102CE000E647F60809E647F60809E647F622E6272A
:102CF000F60809E637F60809E637F60809E637F672
:102D000022E056F608A3E056F608A3E056F608A31C
:102D1000E056F622700422600D18C6C333C608C6FA
:102D200033C6D5E0F41822E056F008A3E056F008C8
:102D3000A3E056F008A3E056F022E493F6087401ED
:102D400093F608740293F608740393F622E026F6CD
:102D500008A3E036F608A3E036F608A3E036F6222C
:102D6000E657F60809E657F60809E657F60809E6B1
:102D700057F622E4C396F608E496F608E496F608B9
:102D8000E496F622C3E09608A3E09608A3E096082E
:102D9000A3E09622C6F4C608C6F4C608C6F4C60860
:102DA000C6F4C622600D08C6A2E713C618C613C62D
:102DB000D5E0F322C3E7960809E7960809E79608E5
:102DC00009E7962275D00075813F7518D1751904F1
:102DD000000224AEE0F608A3E0F608A3E0F608A39C
:102DE000E0F622600C08C6C313C618C613C6D5E0A9
:102DF000F422E6F008A3E6F008A3E6F008A3E6F064
:102E000022CAC0E0E6F0A308DAFAD0E0FA22E0F83D
:102E1000A3E0F9A3E0FAA3E0FB22E0FCA3E0FDA31A
:102E2000E0FEA3E0FF22EAF0A3EBF0A3ECF0A3EDB9
:102E3000F022E0FAA3E0FBA3E0FCA3E0FD22ECF02B
:102E4000A3EDF0A3EEF0A3EFF022E8F0A3E9F0A3E6
:102E5000EAF0A3EBF022E5C754F84401F5C7790185
:102E6000222518F582E43519F58322122B2573B536
:102E700006122B25ABB506122B25F6B606122B250E
:102E80007AB706122B254CA906122B25F6A9061295
:102E90002B252FAA06122B2576AA06122B2539AB35
:102EA00006122B2561AB06122B2587AB06122B25AC
:102EB0009BAB06122B25B0AB06122B25B9AB061225
:102EC0002B259FF903122B25CBF903122B254DFC43
:102ED00003122B25A4FC03122B25E4FC03122B2543
:102EE000F8FC03122B2511FD03122B2502FE031201
:102EF0002B25B3FE03122B25C7FE03122B2577BC0F
:102F000006122B259BBC06122B25B4BC06122B25C2
:102F1000E6BC06122B2516BD06122B2543BD061254
:102F20002B254DBD06122B25AFBD06122B25BEBD90
:102F300006122B25C8BD06122B25D5BD06122B2542
:102F4000FAAB06122B251AAC06122B2559AC061229
:102F50002B2574AC06122B2593AC06122B25F9AC4D
:102F600006122B2502AD06122B255FAD06122B256E
:102F700083AD06122B2544AE06122B2551AE061248
:102F80002B2562AE06122B2579C906122B2591C975
:102F900006122B25BDC906122B25398506122B25B5
:102FA000938606122B25A18606122B25B4860612BF
:102FB0002B25C98606122B25DE8606122B25F186C7
:102FC00006122B25658706122B25CA8706122B258C
:102FD000528806122B25CE8806122B2592890612BE
:102FE0002B25A28906122B25B18906122B2542C852
:102FF00006122B2566C806122B258EC806122B2515
:10300000B6C806122B2590AE06122B25B7AE0612B7
:103010002B25D6AE06122B253EAF06122B2582A6F7
:1030200006122B259BA606122B25A7A606122B25DA
:10303000BBA606122B25D9A606122B25E3A606123F
:103040002B25EDA606122B2500A706122B258DA7F2
:1030500006122B25FCA706122B252BA806122B25C2
:1030600079A806122B25C8A806122B25E3A806125C
:103070002B25EDA806122B25FEA806122B2541A90B
:1030800006122B2586CA06122B25D1CA06122B251D
:1030900022D105122B254CD105122B2569D1051201
:1030A0002B257CD105122B2592D105122B25F0D191
:1030B00005122B2523D205122B2514D605122B25FC
:1030C00074D705122B25A7D705122B25F1D705128A
:1030D0002B254ED905122B2576D905122B258BD9F8
:1030E00005122B259BD905122B25DFD905122B257F
:1030F0003ADA05122B254ADA05122B253ABF0612B9
:103100002B2554BF06122B257CBF06122B2595BFFD
:1031100006122B25B9BF06122B25D7BF06122B2569
:10312000EEBF06122B251CC006122B2537C0061237
:103130002B2537C606122B257DC606122B2532FC01
:1031400002122B2542FC02122B2549FD02122B25CF
:103150007DFD02122B259FFD02122B25C2FD0212BE
:103160002B25E0FD02122B251AFE02122B2583FED1
:1031700002122B25C5FE02122B2504FF02122B255D
:1031800035FF02122B256CFF02122B25BF9706126A
:103190002B25249806122B25CA9806122B25019957
:1031A00006122B2571F204122B2508F304122B258D
:1031B00035F504122B2520F804122B25AEF9041244
:1031C0002B251AFA04122B2569FD04122B25B4FEB7
:1031D00004122B25DBFE03122B2526FF03122B25C1
:1031E000B7F705122B255DFA05122B2502FB0512F8
:1031F0002B252EFB05122B255CFB05122B2591FBA5
:1032000005122B25B9FB05122B2519FC05122B25C0
:10321000CFBB05122B25C5BF05122B25ADC105124D
:103220002B25D6C205122B25B6C305122B2560C54A
:1032300005122B2530C605122B2584C605122B2519
:1032400043B306122B254DB306122B256EB306127F
:103250002B25A49305122B25A49805122B25129A31
:1032600005122B25CE9B05122B25499C05122B25DB
:10327000E89C05122B25E19D05122B25139F0512B5
:103280002B252BA005122B250BA105122B25E9BA06
:1032900004122B2521BB04122B2525C504122B2536
:1032A00006C604122B2552C704122B259BC80412F4
:1032B0002B2551C904122B2525CA04122B250CCB12
:1032C00004122B25F4CB04122B2596CC04122B25AB
:1032D000C0CC04122B2570CE04122B25E0CE041294
:1032E0002B25F9CE04122B2550D004122B2501D109
:1032F00004122B2583D104122B252FD204122B2547
:103300009FD204122B253BD304122B25B7D30412D2
:103310002B25D5D304122B25D7D404122B258DD5DC
:1033200004122B2533D604122B2509BB06122B259C
:1033300033BB06122B2547BC06122B254ABC0612AE
:103340002B25DBC806122B251DC906122B255FC9AC
:1033500006122B256FC906122B2538F105122B25D5
:1033600076F105122B25DFF105122B25FCF1051254
:103370002B2515F205122B25C7F205122B25D0F2AD
:1033800005122B2515F305122B254BF305122B25C2
:1033900062F305122B25D4F305122B2561F40512D7
:1033A0002B2597F405122B25EEF405122B2552F54B
:1033B00005122B2575F505122B25D9F505122B25A0
:1033C00035F605122B2570F605122B25A5F60512EC
:1033D0002B25B7F605122B25C9F605122B2501F76B
:1033E00005122B254DF705122B258BF705122B25E2
:1033F000EA8906122B252A8B06122B254D8B0612E5
:103400002B255E8B06122B25538D06122B25738DD3
:1034100006122B2502B106122B2538B106122B25D8
:1034200080B106122B25DCB206122B250080051276
:103430002B25318105122B256B8105122B252A8323
:1034400005122B25548305122B25E18505122B250A
:10345000218605122B25B88705122B254B880512CE
:103460002B25A38805122B25468905122B257E893D
:1034700005122B25C08905122B252F8B05122B2514
:10348000818C05122B25A48E05122B25D28E0512B8
:103490002B25F98E05122B25028F05122B25528F15
:1034A00005122B25E48F05122B25D49205122B250E
:1034B000579305122B2596C706122B25ACC706126B
:1034C0002B25B6C706122B2510C806122B255D9397
:1034D00006122B25739306122B25189406122B2502
:1034E000579406122B25749406122B25A5940612C8
:1034F0002B25F29406122B25259506122B25609577
:1035000006122B254C9706122B25AD9706122B255C
:103510006AC006122B25BFC006122B2519C1061240
:103520002B2587C106122B25F9C106122B2537C280
:1035300006122B2578C206122B25EAF701122B253D
:10354000F0F701122B2530F801122B2522FA011277
:103550002B2552FA01122B25C1FA01122B258FFBC4
:1035600001122B25D0FB01122B25FEFB01122B256E
:1035700088FC01122B259FFC01122B25ACFC0112AB
:103580002B25B6FC01122B2552FE01122B2547FFDD
:1035900001122B2590FF01122B257ADA05122B251B
:1035A00090DA05122B2523DB05122B254FDC0512A3
:1035B0002B2544DD05122B25E1DD05122B2521DE0F
:1035C00005122B259FDE05122B25FCDE05122B256F
:1035D0000CDF05122B2533DF05122B2586DF0512A4
:1035E0002B25F7E005122B25FCE005122B251CE10D
:1035F00005122B25FEC906122B252CCA06122B25D7
:1036000061CA06122B2563CA06122B2565CA06124B
:103610002B2576CA06122B2578CA06122B257BCAC3
:1036200006122B257AB906122B25E8B906122B258E
:103630000ABA06122B2542BA06122B2578BA0612B0
:103640002B256AA306122B25B1A306122B25D4A382
:1036500006122B2507A606122B2521A606122B25BE
:103660004CA606122B259A7F00122B25EAE20512A2
:103670002B25C3E305122B25A9E405122B25BAE45B
:1036800005122B25CBE405122B2517E505122B255A
:103690000BE705122B255FE805122B258FE8051295
:1036A0002B2556E905122B25B4E905122B25FFDA47
:1036B00002122B255ADB02122B2501DC02122B25CC
:1036C00076DD02122B2550DE02122B250DDF0212B1
:1036D0002B2524DF02122B2573DF02122B25D7DFC7
:1036E00002122B252CE002122B253FE002122B2583
:1036F000A0E002122B25F9E002122B2511E10212A3
:103700002B25A5E302122B25A9E402122B25E4E4C4
:1037100002122B2538E502122B25DFE702122B259A
:1037200025E802122B2598E802122B25E2E8021266
:103730002B25B6E902122B25F9E902122B2513EAF3
:1037400002122B255AEA02122B257AEA02122B25A5
:103750001FEB02122B2503EC02122B250EEC02129A
:103760002B255CEC02122B25B1EC02122B25F8EC78
:1037700002122B255CEE02122B2580EE02122B2565
:1037800005F102122B253CF102122B2544F2021204
:103790002B2568F202122B25D7F202122B259AF361
:1037A00002122B25D5F302122B253BF402122B25F6
:1037B00050F502122B2598F502122B25A2F50212C4
:1037C0002B25A5F502122B25AFF502122B25C2F5EC
:1037D00002122B254BF602122B2574F602122B2512
:1037E00087F602122B25B3F602122B25DAF6021207
:1037F0002B25FEF602122B2577F702122B25E9F76F
:1038000002122B2520F802122B252AF802122B2552
:1038100059F802122B256FF802122B258AF8021292
:103820002B25B8F802122B25D8F802122B2521F9E6
:1038300002122B255CF902122B2563FA02122B25AA
:10384000C1FB02122B25D7FB02122B25EEFB021225
:103850002B2500FC02122B259CC306122B25ADC381
:1038600006122B2536C406122B25008006122B25A6
:103870003E8006122B25CA8006122B25D581061202
:103880002B25F18306122B256E8406122B252DEA9B
:1038900005122B257CEA05122B251CEC05122B2585
:1038A000F0ED05122B2532EE05122B25FDEE05124B
:1038B0002B2505F005122B2527F005122B2583F06B
:1038C00005122B2504F105122B25595100122B2529
:1038D0007B5100122B25D35200122B251C530012B2
:1038E0002B25925300122B25105400122B257554B2
:1038F00000122B25B75400122B25265500122B251C
:10390000D15500122B25495600122B258E56001238
:103910002B259D5A00122B25A45C00122B25D75C69
:1039200000122B25295D00122B252C6000122B255F
:10393000A86000122B25566200122B258863001206
:103940002B25A06400122B25226500122B25026670
:1039500000122B256D6600122B25816600122B2587
:10396000636700122B25936800122B25AE6A0012A4
:103970002B25A76C00122B258A6D00122B25207099
:1039800000122B25C17000122B25C17100122B25AE
:10399000237500122B25337500122B257976001222
:1039A0002B25167700122B25407800122B25D17875
:1039B00000122B25FE7900122B25437A00122B25AD
:1039C000D77A00122B25DAD604122B257AD70412C7
:1039D0002B25E4D704122B25FDD704122B258CD8D8
:1039E00004122B25D0D804122B25EFD904122B2535
:1039F0002BDA04122B259EDA04122B25E9DA0412A5
:103A00002B2548DB04122B25F2DB04122B25DBDEF1
:103A100004122B25F8DF04122B2575E004122B2548
:103A200036E204122B25D6E204122B2575E304128C
:103A30002B25D8E304122B254DE404122B255CE53D
:103A400004122B253DE604122B2573E604122B25C8
:103A5000A6E604122B255AE704122B2586E704124A
:103A60002B2501E804122B2584E904122B25FFEAFB
:103A700004122B2554EC04122B25C7ED04122B2520
:103A8000D3EE04122B257AEF04122B25E8EF041253
:103A90002B2500F104122B25ACDA03122B2517DBA2
:103AA00003122B255FDB03122B25A3DB03122B252F
:103AB0000DDC03122B2556DC03122B2591DC03129F
:103AC0002B252BDD03122B2585DD03122B25DFDEB5
:103AD00003122B2568DF03122B2592DF03122B25FF
:103AE00097E003122B25A6E103122B25D8E1031240
:103AF0002B25C8E203122B25D9E203122B25F1E274
:103B000003122B25F1E303122B250EE403122B25C0
:103B1000D3E403122B25FDE403122B2514E5031235
:103B20002B253AE503122B2571E503122B2591E590
:103B300003122B25B8E503122B25D0E503122B2504
:103B4000AAE603122B2502E703122B2578E80312BD
:103B50002B2507E903122B252BE903122B2542E91C
:103B600003122B250DEA03122B25B0EA03122B2595
:103B7000D6EA03122B2506EC03122B2525EC0312A3
:103B80002B25A6EC03122B2513ED03122B2557ED45
:103B900003122B25E5ED03122B2550EE03122B25E6
:103BA00002EF03122B25F2F003122B25CAF10312A8
:103BB0002B251CF203122B2516F303122B2523F4BD
:103BC00003122B2534F503122B2542F503122B2566
:103BD00012F603122B25B2F603122B25F6F603126A
:103BE0002B250BF703122B250BF803122B25AEF810
:103BF00003122B2506F903122B25969F06122B255F
:103C00003EA106122B2504A206122B2559A206124C
:103C10002B25D6A206122B25EEC606122B25BD7B20
:103C200000122B25017C00122B25277C00122B254E
:103C30004D7C00122B25657C00122B257D7C00120B
:103C40002B25957C00122B25007D00122B25427D13
:103C500000122B25577D00122B255E7E00122B258E
:103C6000797E00122B25827E00122B258B7E00127E
:103C70002B25947E00122B259E7E00122B251B7F68
:103C800000122B25F87F00122B25D59206122B252A
:103C9000F19206122B25F69206122B25F9B7061281
:103CA0002B25CCFC05122B25E2FC05122B255EFEF4
:103CB00005122B2588FE05122B25CEFE05122B257D
:103CC000C7FF05122B25DFBD06122B2500CB0612E0
:103CD0002B25CDFF01122B25008002122B255780AA
:103CE00002122B25C38002122B254F8102122B2595
:103CF000058202122B254D8202122B2566820212AA
:103D00002B25898202122B25AB8202122B25E982F8
:103D100002122B25388302122B25638302122B25D6
:103D2000C18302122B25688402122B2510850212F2
:103D30002B258C8502122B25598602122B25A08655
:103D400002122B25EC8602122B25748702122B25DA
:103D5000AD8702122B25038802122B251F88021221
:103D60002B254E8802122B255A8A02122B25888B6E
:103D700002122B25B48B02122B25E88B02122B2565
:103D8000098C02122B25188C02122B25238C02126F
:103D90002B25D28C02122B25428D02122B25CD8D84
:103DA00002122B25D58D02122B25428E02122B25B5
:103DB0007E8E02122B25448F02122B2517900212A1
:103DC0002B256C9002122B250B9102122B2565914D
:103DD00002122B25AA9102122B25439402122B25A5
:103DE000869502122B25709802122B2554990212E7
:103DF0002B25389A02122B255D9A02122B256E9ADA
:103E000002122B25E09A02122B25779B02122B25FA
:103E1000EB9B02122B25DB9C02122B25009D02122C
:103E20002B25189E02122B25369E02122B25529E00
:103E300002122B25C59E02122B25D49E02122B2581
:103E40005C9F02122B2559A002122B2566A002129C
:103E50002B256FA002122B2551A202122B257DA328
:103E600002122B258DA302122B25C8A402122B258A
:103E700047A502122B2578A602122B25B4A6021202
:103E80002B258EA802122B254BAC02122B255FACE2
:103E900002122B2569AC02122B2573AC02122B25C2
:103EA0007DAC02122B2587AC02122B25A0AC02128E
:103EB0002B25AAAC02122B2521AD02122B252CADED
:103EC00002122B255BAD02122B2583AD02122B258E
:103ED0008EAD02122B25F3AD02122B25FDAD021281
:103EE0002B2508AE02122B252CAE02122B2550AE2C
:103EF00002122B25C2AE02122B250BAF02122B256C
:103F000027AF02122B2598AF02122B25E4AF021225
:103F10002B252DB002122B256BB002122B25ECB0F5
:103F200002122B2593B102122B2558B302122B2516
:103F3000BDB302122B25EBB402122B2511B50212D0
:103F40002B2559B602122B2593B902122B2591BBB2
:103F500002122B255CBD02122B25F5BD02122B256A
:103F6000F6BF02122B25ABC002122B25E4C00212B1
:103F70002B2554C102122B255EC102122B2587C3AB
:103F800002122B258AC402122B25C7C502122B252B
:103F90001EC602122B25C9C602122B2579C8021291
:103FA0002B25C6C902122B25E6C902122B253BCAB6
:103FB00002122B253CCB02122B2564CB02122B259F
:103FC000C3CB02122B25BBCC02122B2532CD021201
:103FD0002B2545CE02122B25B3CE02122B25B2CFB4
:103FE00002122B250CD202122B2535D202122B25C0
:103FF0009BD302122B251DD502122B2574D502123C
:104000002B2522D602122B25C7D602122B252AD702
:1040100002122B25E8D702122B257AD802122B2563
:10402000D9D802122B251BD902122B254CD90212EA
:104030002B25A3DA02122B25008003122B253280B8
:1040400003122B256B8003122B25348203122B25A0
:10405000788203122B254E8303122B25AD83031286
:104060002B25C38403122B250F8503122B259D8737
:1040700003122B25818A03122B25C88B03122B25B3
:10408000608C03122B256C8C03122B25B58C03122C
:104090002B25F78D03122B25ED8E03122B25178F61
:1040A00003122B256D8F03122B25C68F03122B2590
:1040B000399003122B256F9203122B25F1930312D3
:1040C0002B25DC9403122B25269603122B255E98B4
:1040D00003122B255B9B03122B256A9B03122B25B6
:1040E000FE9B03122B25A99C03122B25EC9C03128B
:1040F0002B25359D03122B25859D03122B25E99D2C
:1041000003122B255B9E03122B25779E03122B2572
:10411000A69E03122B25E59E03122B25E09F03127A
:104120002B258FA003122B250CA303122B253EA4B5
:1041300003122B2516A503122B2598A503122B2558
:10414000CDA903122B25FCA903122B2557AA031274
:104150002B258AAA03122B2502AB03122B2535AB84
:1041600003122B2596AB03122B25E6AB03122B254E
:10417000B3AC03122B256CAD03122B2530AE03120A
:104180002B25AAB003122B250CB203122B255DB3ED
:1041900003122B2581B403122B2584B403122B2583
:1041A000B3B403122B25ABB603122B256AB7031247
:1041B0002B2599B703122B25B7B803122B257FB9EE
:1041C00003122B2540BB03122B25B0BB03122B255A
:1041D000E2BB03122B2502BC03122B2571BC031278
:1041E0002B256ABD03122B258EBD03122B2501BE84
:1041F00003122B252AC003122B2589C003122B255D
:10420000DDC003122B250CC303122B25EFC30312B1
:104210002B2577C403122B255BC503122B25E5C57F
:1042200003122B25F9C503122B250DC603122B25CE
:1042300021C603122B2535C603122B2562C6031295
:104240002B2592C603122B254DC803122B2523C9FB
:1042500003122B25C7C903122B251CCA03122B25B9
:104260007FCA03122B25C8CA03122B25EFCA0312DB
:104270002B25B7CB03122B255DCC03122B25E3CDC9
:1042800003122B256ECE03122B25B5CE03122B2540
:1042900027CF03122B257CD003122B2525D1031207
:1042A0002B2559D103122B2571D103122B2514D2A2
:1042B00003122B2590D403122B2538D603122B255D
:1042C00056D603122B2574D603122B2540D7031282
:1042D0002B258EDA03122B25A78101122B25E981CC
:1042E00001122B25568701122B25A28701122B259F
:1042F000E88701122B25398901122B259E8901128D
:104300002B25E28901122B25488B01122B25A38E28
:1043100001122B25D68F01122B25659B01122B250F
:10432000F59B01122B25DF9E01122B2544A00112C3
:104330002B25A7A001122B25C3A101122B252DA3EC
:1043400001122B250CA401122B257AA601122B2574
:104350000CA801122B259DA801122B25BCA9011226
:104360002B2549AA01122B2553AA01122B257BAA22
:1043700001122B251EAB01122B2509AC01122B2596
:10438000D1AC01122B255EAD01122B2574AD0112AB
:104390002B2591AD01122B25BAAD01122B25E7ADCE
:1043A00001122B252BB001122B25FEB001122B255B
:1043B00042B101122B25C4B101122B2565B20112A5
:1043C0002B2597B201122B25DEB201122B2511B33A
:1043D00001122B2555B301122B25A4B301122B2555
:1043E000A9B301122B2505B401122B2549B40112E2
:1043F0002B2533B501122B2598B501122B25F6B5C7
:1044000001122B2575B601122B25EDB901122B25B2
:10441000F0BA01122B2586BC01122B25C9BF01124F
:104420002B256BC001122B25B4C201122B256FC3A3
:1044300001122B25AEC301122B2572C501122B25AB
:104440008FC501122B2598C501122B25A1C501127C
:104450002B25ACC501122B25CBC501122B25EFC78F
:1044600001122B254CC801122B2556C801122B25F1
:1044700060C801122B25C3C801122B251FC90112C8
:104480002B252CCA01122B258DCA01122B259ECB60
:1044900001122B25E7CB01122B25B1CC01122B25C4
:1044A000C8CD01122B258CCE01122B25D8CF01129D
:1044B0002B25DCD001122B25D5D101122B25EDD1D6
:1044C00001122B2524D201122B252ED201122B25CD
:1044D00038D201122B2543D201122B2561D20112B1
:1044E0002B25A9D201122B2507D301122B252ED360
:1044F00001122B2540D301122B25E9D301122B25C4
:1045000022D401122B2553D501122B25B0D501122F
:104510002B25A1D601122B25D7D601122B2547D743
:1045200001122B25C3D701122B2544D901122B25AB
:104530006BDA01122B252DDB01122B25FBDB01127F
:104540002B2580DC01122B252FDD01122B2517DEF8
:1045500001122B25B0DE01122B258CDF01122B2539
:10456000F4DF01122B25B3E001122B250FE101121C
:104570002B2573E101122B2539E201122B255CE278
:1045800001122B2516E301122B2538E301122B25EE
:1045900099E301122B25C9E501122B25C2E6011270
:1045A0002B256EE701122B258BE901122B25D4E96F
:1045B00001122B251FEA01122B257BEA01122B2564
:1045C000D9EA01122B25FDEA01122B2521EB01125C
:1045D0002B2556EB01122B257EEB01122B25C3EB6D
:1045E00001122B2521EC01122B257AEC01122B252F
:1045F00074ED01122B2520EF01122B2565EF01121E
:104600002B258EEF01122B2517F001122B258AF096
:1046100001122B2598F001122B25BCF001122B253D
:1046200012F101122B252DF101122B25E8F10112B7
:104630002B2514F201122B2557F201122B25BAF269
:1046400001122B25CAF401122B25F6F401122B2599
:10465000B1F501122B2595F601122B2529F7011230
:104660002B25A2C605122B25DAC605122B25FBC663
:1046700005122B253DC705122B25A1C705122B2599
:10468000ABC705122B25BBC705122B25F2C7051298
:104690002B259BCB05122B2563CD05122B2547CF50
:1046A00005122B25E9CF05122B2573D005122B25DA
:1046B000508004122B25F98004122B25D881041276
:1046C0002B25E48204122B25048304122B25268437
:1046D00004122B25D68504122B25438604122B2584
:1046E000148704122B251A8804122B259288041291
:1046F0002B25CD8804122B25268904122B256189B0
:1047000004122B25AA8904122B253E8A04122B257C
:10471000D48A04122B25A98B04122B257C8C04121D
:104720002B250A8D04122B25308D04122B255D8D2F
:1047300004122B258E8D04122B255B8E04122B2543
:104740006B8E04122B25BE8E04122B25CB8E0412E9
:104750002B25D88E04122B25E18E04122B25458F94
:1047600004122B25A38F04122B25EE8F04122B2568
:10477000099004122B25309004122B254D90041221
:104780002B25599004122B25EA9104122B25039214
:1047900004122B257F9204122B25929204122B25B2
:1047A000A29204122B25469304122B25B2940412D4
:1047B0002B25C59504122B25659604122B256F9683
:1047C00004122B25EE9604122B25FF9604122B259E
:1047D0003E9704122B256C9704122B25399804124E
:1047E0002B25909804122B25C99804122B251F996C
:1047F00004122B253D9904122B258B9904122B258D
:10480000569A04122B25A49A04122B25F19A04120D
:104810002B25749B04122B259E9B04122B25D49BC5
:1048200004122B25E39B04122B25429C04122B25FA
:10483000BA9C04122B25FB9C04122B254B9D0412C1
:104840002B25769D04122B25909D04122B25AA9DC5
:1048500004122B257F9E04122B25899E04122B25E2
:10486000C49E04122B25D49E04122B25DD9E041217
:104870002B252E9F04122B25429F04122B2564A06A
:1048800004122B2577A004122B258EA004122B25B1
:10489000A3A004122B2536A104122B25AAA10412D1
:1048A0002B254FA204122B255AA204122B25BDA39F
:1048B00004122B25D9A304122B2525A404122B2581
:1048C00093A404122B25C5A404122B25DFA40412E3
:1048D0002B253FA504122B25DEA504122B2529A686
:1048E00004122B257CA804122B2514A904122B25B5
:1048F0008BA904122B25E8AB04122B2500AC041263
:104900002B2503AC04122B250FAC04122B2523AC52
:1049100004122B252BAC04122B2562AC04122B2580
:1049200056AD04122B25E0AD04122B2562AE041205
:104930002B25E2AE04122B25B9AF04122B25DBAFD9
:1049400004122B2574B004122B25D1B004122B2590
:10495000D4B004122B2501B104122B2516B1041278
:104960002B2585B104122B25D1B204122B25E4B3DB
:1049700004122B256FB404122B2582B504122B25AB
:1049800049B604122B257AB604122B25A0B60412C0
:104990002B25A9B604122B25D8B604122B2588B7CF
:1049A00004122B2538B804122B25ABB804122B2582
:1049B0004EB904122B25C1B904122B2500BA0412DA
:1049C0002B2549BA04122B257EBA04122B25EBC6DF
:1049D00006122B2583C306122B251DC306122B2579
:1049E0009AC206122B2563C506122B25AFC40612E8
:1049F0002B2597C406122B2587C406122B25E57F8D
:104A000000122B25F9FF01122B251FC606122B259C
:104A100081C506122B2570C506122B250FAE051277
:104A20002B255CAD05122B2590AC05122B25ECAA8D
:104A300005122B25B5AA05122B2587AA05122B25B1
:104A400034AA05122B258BA905122B25F3A80512D4
:104A50002B25CDA805122B2582A805122B2556A89B
:104A600005122B25CAA705122B25829F06122B257E
:104A700069A705122B25279F06122B25C29E061219
:104A80002B25039D06122B252F9C06122B25B69B4A
:104A900006122B25A89B06122B258DC706122B2547
:104AA0008AC706122B2524A705122B253FA605121F
:104AB0002B255DA505122B2505A505122B2577C7EE
:104AC00006122B2575A405122B2530A405122B25C3
:104AD00014A405122B25C2A205122B25B98E06128D
:104AE0002B2584A205122B2527C706122B255EA293
:104AF00005122B25E2A105122B2598BB05122B25AB
:104B000051BB05122B25F0BA05122B25C3BA05128D
:104B10002B2599BA05122B2565BA05122B253DBA0E
:104B200005122B25DDB905122B25C7B905122B253A
:104B30008CB905122B2503B905122B254AB5051290
:104B40002B2508B305122B25CDB005122B254FB010
:104B500005122B25F0AE05122B2500B005122B25D2
:104B60008DAF05122B254EAF05122B259F7B000024
:104B7000000080FB8F000100E91987000100E8199F
:104B800035000400A51C25000200A91C2600020017
:104B9000AB1C27000200AD1C28000100B71C290037
:104BA0000100B81C84000400B91C86000100BD1C73
:104BB0002A000100BE1C2B000100BF1C2C000100BC
:104BC000C31C2D000800CA192E000100C41C2F00B0
:104BD0000100C51C30000100C61C31000100C71CCB
:104BE00032000100D21933000100D3193400010052
:104BF000C81C36000100D41938000100C91C390056
:104C00000100C21C83000200DD1C63000100E519E5
:104C100064000100C01C65000100C11C6D000100A2
:104C2000E61971000800C21966000100DC1C43008F
:104C30000100CD1C44000200CE1C45000100D01C28
:104C400046000200D11C47000800DD1948000100A1
:104C5000D31C4B000100D41C04000100DF1CA10088
:104C60000100E21C37000100E11C88000100E01C8B
:104C70003C000100D5193D000100CA1C490002009A
:104C8000D51C67000100E7194D000200D71C4E003B
:104C90000100D91C4F000200DA1C3E000100DC19A3
:104CA00051000100D61952000100CB1C5300010035
:104CB000CC1C54000100D7190000000000000001C6
:104CC0003636010100010201000103010001040167
:104CD000060605020000070100340801000F090460
:104CE00001010D0100FF0E0800001702000019016C
:104CF00000FF1A0100011B0100FE1C0100081D023B
:104D000000001F0100012001000121020000230119
:104D1000000F2402000026010001270100082802DC
:104D200000FF2A0100072B0102402C0100002D0189
:104D300000012E0100012F0100FF30010B1D310881
:104D400000003A0100083B01000F3C0100013D0159
:104D500000FF3E04000042040000460400004A0434
:104D600000004E04000052040000560400005A04E3
:104D700000000103710301030103010301030103A7
:104D800022030203010310030003000300030003D6
:104D9000000300030003420300032403060300038F
:104DA0000003040312032503230325032303040341
:104DB0000403000300030003440300030003230370
:104DC000000365032100350381030003050300038D
:104DD0000003000300032503230301017101010106
:104DE00001011101010131010101010180011001E5
:104DF00061013B0014006301730172016201430110
:104E00000001130106013D013500040112010001FA
:104E100000010001000104010401330133013C01E0
:104E20004401320136000001000165010001350036
:104E30008101000105018201830100010302710269
:104E400030016002110270020102020202028002BD
:104E5000100261023A0041006302730272026202B0
:104E60004302000213023800000200020402120290
:104E700000020002000200020402040237003700B0
:104E80003C024402000239000002000265020002F6
:104E9000350281020002050282028302000203043D
:104EA0007104020460041104700402040204010489
:104EB0000204100461040004140463047304720403
:104EC0006204430400041304060400040004040400
:104ED00012040004000400040004510464000004EF
:104EE00000040004440400040004000400046504F9
:104EF00000043504810464000504000483040004F4
:104F000003007100300160001100700031022003C5
:104F10005004800010006100000014006300730062
:104F20007200620043000000130006000000000051
:104F30000400120000000000000000000400040053
:104F4000370037003C024400000000000000000071
:104F500065000000350081000000050000008300AE
:104F6000000036000100060000000F0000000000F5
:104F7000000000000000000003FFFF00000403FF2A
:104F8000FF0000FFFF0FF4010005C404032000012F
:104F900000000B000000000000000003010F0000F3
:104FA0000000000000000000000000000000000001
:104FB00000000000000000000000000000000000F1
:104FC0000000053A130063391F0069391F806F39EB
:104FD0000100053A0200EB380300F1380400F7380D
:104FE0000500FD3806000939300027393100213924
:104FF000320033393300393935003F39340045390F
:1050000036004B391100573914005D3915001B3932
:10501000FFFF00000A000000020000000400000082
:105020000800000010000000200000004000000008
:1050300080000000000100000002000000040000E9
:1050400000080000001000000020000000400000E8
:10505000011D43065343084D430B6B4310E73F0AC2
:105060007D430223430541430729430C05430D11AA
:105070004364BF3DFF000007ECFDFDFDECDCDCCC34
:10508000BCACAC9C9C8C7C7C6C6C5C5C5C4C4C3C90
:105090003C2C2C1C1C03EAF5E5D5D5C5B5A595958A
:1050A0008585757565655555454535352525151530
:1050B0000500160F00000B150B020002220F330033
:1050C000000E5A6967426565416C6C69616E636583
:1050D000303901030507090B0D0F00020406080A09
:1050E0000C0D00011916181616182303003030177E
:1050F000181921301B1D1F30303016181920231AA3
:105100001C1E3000393D3F373C3C362C442D0003FB
:105110004A49434E181A2505020C0E020B040B0ACD
:105120000708000F020402010101010902E803005F
:105130000000BE040A0000E8030E0000007F001E0D
:10514000050303000404100A0C10080C28000904CD
:105150000903010C05081F08FFC082C08390194095
:10516000E4F0A3F07C197D1A7A597B1812353112BC
:105170003DEF124035123DF502667A74F512259323
:1051800074F5122C0BE9FF8A08EBFE8C09E9705BC1
:1051900074026A703E790812383D750A00780A1266
:1051A0002B7EE509F50A780A122B7EEEF50A780ABD
:1051B000122B7E90187512299D901CBDE0F97CDDA4
:1051C0007D19901CDD12651E123E197407122B8D7D
:1051D0000252A274016A60030252A7790812383D94
:1051E0007B00EEFAF9123E5B0252A274016F600876
:1051F00074026F60030252A7EA600574036A704785
:10520000790212383D901CBDE0F9901875122E32CB
:10521000123E07E9F8901884E0A2E34010E9700D0F
:10522000901944E004F0640470031252C1740365E1
:10523000087071901945E0F9740129F0E9C39405EB
:1052400040621252C1805D74016A705B74016F79B3
:105250000A702E12383D7401122E61E4F0740212AD
:105260002E617403F004122E61E4F0A3F0A3F0A306
:10527000F07408122E61E4F0AA18AB1912432F80C3
:105280003612383D901CB312299D7A007B20125CA7
:1052900073122B8D901CBDE0F9901875122E3212EE
:1052A0003E3DE9F8E8601090810612299D7A017B65
:1052B00000125C73122B8D740B122B8D7F0302284E
:1052C00019901875E4F0A374F8F0A374FFF0A374B8
:1052D00007F02274F6122593E9FFEAFE7AD1F9125B
:1052E00033998A828B83E5824583702A7A027B0018
:1052F00012337BEA4B700E7A107B00901879E0F93C
:105300001233BD80148A828B8374D1F0EFA3F0EE48
:10531000F91233878003EFA3F002552174F71225A9
:105320009389089004D1127821FF901CA0E0F470BA
:1053300003A3E0F470319005E4E0901CA0F0A3E436
:10534000F080248E828F83A3126382600F8E828FFF
:1053500083A3A312637FFAA9081238D38E828F83A6
:10536000126248E8FEE9FFEE4F70D8901CA0E0F40E
:105370007003A3E0F4600A901CA0E0FAA9081238B8
:10538000D312443D901843125A971244377F0102BA
:10539000281974F0122593890B8C0C750900750877
:1053A000007410122E611262487412122E61126A79
:1053B00092FD804712545CF50EA3E0F50FAE08EEA7
:1053C0002EFEE433FFEA2EF582EB126729650E709C
:1053D00004A3E0650F7019AE09EE2EFEE433FFEC76
:1053E0002EF582ED3FF583E50EF0A3E50FF00509FC
:1053F000050AE50AC3950C40BB0508E508C3950BF3
:105400005005750A0080EBA90980007F0802281961
:1054100074F4122593890B7D00740C122E611262B4
:105420004880010DEDC3950B502E750A00800205D2
:105430000AE50AC39C50ECED25E0FEE433FFEA2EBA
:10544000F582EB3F126C8B12545C65087004A3E08C
:10545000650970DB7901800279008014AE0AEE2EB6
:10546000FEE433FFE82EF582E9125C5D22122B8DFB
:105470007F0402281974F612259312550B7003A3AA
:10548000E06D70177508827509187808122B7AEE8E
:10549000FA123A0B7402122B8D801A7508027509E4
:1054A000807808122B7A8A0889097808122B7A12D8
:1054B00054F9122B8D806A74F612259312550B70D5
:1054C00003A3E06D701775088F7509187808122B03
:1054D0007AEEFA123A117402122B8D801A750803B3
:1054E0007509807808122B7A8A0889097808122BA6
:1054F0007A1254F9122B8D8028EE240E125C5AFD7C
:105500007C80126731123A2F740422EAFEEBFF12FC
:105510006748FCE439FD901843E06C227402122BBA
:105520008D7F0202281974F612259374FE122C0B3B
:10553000EAFEEBFF851882851983E41255CA1268CA
:1055400083FBECFA88828983A3A3E0F975090075CF
:105550000800600574FF697005750882803E901828
:1055600043E06A7003A3E06B701BAA18AB19124BDF
:1055700021E9FA851882851983126A9D70037508DE
:10558000838A0980179019E8E0600464017005754A
:1055900008818008E06402700375088085188285A0
:1055A0001983126A92FDA908EEFAEFFB123A17E589
:1055B000096014851882851983126A9D600985180F
:1055C000828519831270BA02551CF0A3F01276FA84
:1055D0002274F2122593EAFEEBFF750800750900AC
:1055E000126744F50AE439F50B12443DEA650A7086
:1055F00003EB650B7012124B0FE914F50879017A71
:105600000C7B19124B098003750980EE240E12677A
:1056100026F50C780C122B7E750C0C750D19780C78
:10562000122B7A7808122B7E780A122B7AE509F56C
:10563000087808122B7E12650D126726F97A057B11
:1056400080123A1D740702795F74F6122593E9FF00
:105650007E0080328A828B83E0F508A3E0F8E4C8FC
:10566000F9E50828E439F509EE25E0F8E433F9EC2A
:1056700028F582ED39F583E508F0A3E509F0EA2481
:1056800002FA50010B0EEEC39F40C902552174E887
:1056900012259374FC122C0B8A168B17751100744B
:1056A00002122E61E4F0A312688B1255CA3517124C
:1056B0005C6BF50B850A82F583127AC5FEE439FF2F
:1056C000850A82850B83A3A3E0FA850A82850B8372
:1056D000A3A3A3E0F9EAF508E439F509EEFAEFFB34
:1056E0001244D9E964016016EEFAEFFB1244D9E9DD
:1056F0007038901843E06E7003A3E06F602C127452
:1057000061122B7EE4F508F5097808122B7A7808E7
:10571000122B7E9018431229A57508807808122B49
:105720007E125A65122B8D025A44850A82850B839C
:10573000A3A3A3A3E0F510E50A2405F50A5002058A
:105740000BE51060281279D67402122E61125A9756
:105750007402122E61126A9D60137402122E61127D
:105760005A5BA9101239038A0A8B0B80037510004B
:10577000850A82850B8312797060241279D6851888
:1057800082851983EAF0A3EB126AA3E849601085C9
:105790001882851983125A5BA90F12390380037589
:1057A0000F009004D18052850A82850B83A3A3A3A6
:1057B000A3A3A3A3A3E4F0A3F0AA0AAB0B851482CE
:1057C000851583A3A3E0F812637FF912338785124E
:1057D00082851383E0C0E0A811740C28F582E434BC
:1057E00019F583D0E0F00511A2005007AA12AB13FF
:1057F000123423851482851583E0F514A3E0F51592
:10580000E514451570030259C1851482851583A3DB
:1058100012638260DE851482851583A3A3A3A3A3EC
:10582000A3A3A3E0A2E050CB851482851583A3A394
:10583000A3A3126A9D851482851583A3A3601E12FB
:105840006383FA7901851482851583A3A3A3A31228
:105850005A4E1227798A128B13D200800F125A4E99
:10586000A3A3A3E0F512A3E0F513C200E5124513CC
:1058700070030257E8851282851383A3E0650870E0
:1058800004A3E06509600F74FF6508700474FF6588
:105890000960030257E8851282851383A3A3A3A39B
:1058A000A3A3A31229A5851282851383A3A3A3A36F
:1058B000A3A3E0FC7404122E6112651EA910123815
:1058C000E57402122B8DE9703C851282851383A347
:1058D000A3A3A3A3A3A3A3A3A31229A5851282858F
:1058E0001383A3A3A3A3A3A3A3A3A3E0FC74021203
:1058F0002E6112651EA90F1238E57402122B8DE974
:1059000070030257E8E50F2510C333240AFA7B0021
:1059100012337B8A0A8B0BEA4B70030257CE8A82C2
:105920008B8374D2126C958A828B83A3A3E8F0A335
:10593000E912793FA3E510127ACFE50FF0E5106088
:105940002CEA240AFAE4350BFB850A82850B8312C4
:105950005A927402122E61125A85122B76AC10ECF8
:105960002CFCE433FD127193122B8D800D8A828BF7
:1059700083A3A3A3A3A3E4F0A3F0E50F700302574E
:10598000A7A810E828F8E433F9E50A28F8E50B3968
:10599000F9E8240AFAE439FB850A82850B83A3A37C
:1059A000A3125A92851882851983125A85122B7672
:1059B000AC0FEC2CFCE433FD127193122B8D0257CB
:1059C000B9E5116025127461122B7E75080C7509FA
:1059D000197808122B7AE511F5087808122B7E90B9
:1059E00018431229A57508008029EEFAEFFB12442E
:1059F000D9E9702A127461122B7E75080C75091989
:105A00007808122B7A7508007808122B7E901843BC
:105A10001229A57808122B7E125A65122B8D74025A
:105A2000122E61126A9D60087402122E611270BA01
:105A3000851882851983126A9D60098518828519E7
:105A4000831270BA7404122B8D7F10022819125A17
:105A50005222E0F8A3E0F583888222E0FCA3E0FD77
:105A6000AA0AAB0B22E5162402FCE43517FDE51665
:105A7000240FF582E43517F583E0F97A067B80126E
:105A80003A1D740722E0F50CA3E0F50D750E0078C1
:105A90000C22A3A3A3A3A3EAF0A3EBF02274F112B8
:105AA000259374F4122C0B8A088B09ECFEEDFF741D
:105AB0000B122E617403F0122BE31235311265F6CE
:105AC0007403122BE312352BE9600A125C6260103A
:105AD000E06401600B8518828519837484025C0E72
:105AE0008E828F83A3A3A3A3A3A3A3A3E06013F435
:105AF0006010125C627016EE24141267266003F4C4
:105B0000700B8518828519837482025C0E1277E50A
:105B1000E064217002A3E06003025BE585188285E2
:105B20001983748CF0125C626003025BCF74011203
:105B30002BEBEE240BFAE43FFB124161E960030218
:105B40005BCF12382B8A0A8B0BEA4B7003025C0F77
:105B50008E0C8F0D750E00780C122B767C157D0047
:105B6000127193122B8D850882850983A3A3E50A00
:105B70002415FCE4350BFD7409122A9E127416C01C
:105B8000E0E50A241E125C47D0E012609FC0E0E509
:105B90000A241F125C47D0E0F0E50A2420125C477B
:105BA0007405F0EE240BFE50010FFAEFFB124A438E
:105BB0007D007C007900EEFAEFFB1239D59081066A
:105BC00012299D7A007B10125C73122B8D80731248
:105BD0005C4F122B7E125C7E1241437401122B8D9E
:105BE000E9702C8014125C4F122B7E125C7E1241E5
:105BF000497401122B8DE9700D851882851983E493
:105C0000F01237FB80098518828519837488F01299
:105C10007416F50A780A122B7E7401122BDB880A9F
:105C2000890B780A122B7AE508240CF582E43509F1
:105C3000125C6B4480F50B780A122B7A1265D8122D
:105C40002B8D740C026FA9F582E4350BF58322EEDF
:105C50002414125C5AF50A780A22F582E43FF5838F
:105C6000E022EE2413125C5A640322F583E0F50A65
:105C7000A3E022901879E0F91234E3740422EE24B0
:105C80000BFCE43FFD8E828F83A3A3A3A3A3A3A356
:105C9000A3A31274518E828F83A3A3A3A3A3A3A350
:105CA000A3E0F922C082C08374F3122C0B85188202
:105CB000851983E4F004122E61125A977403122E90
:105CC00061AA82AB83123CF3AA18AB19123D2F7460
:105CD0000D122B8D02667A74F612259312671FF847
:105CE000A3E0125D1AF890188AE058F508A3E0596D
:105CF000F509E5084509601F7808122B7A901843CA
:105D00001229A5EE240E126726FD7C0012672D12C3
:105D10003A297404122B8D0255218882F583125D75
:105D20002222E0FAA3E0F9EA2274EA12259374DB56
:105D3000122C0B8A148B157512007513001276F64F
:105D40003515F583126383F50EAC18AD197A007B17
:105D500000799C123E6D7A047900123D59EAF50CE7
:105D6000851882851983E02AF0F8E50EC398400370
:105D7000025F4DE0C3950EF509C394044003750915
:105D800003E50975F01AA4FAABF012341D8A128BE0
:105D900013EA4B7003025F50750D00AE12AF13850E
:105DA0000E08025E2D7C087D0079FFEE240AFAE4DD
:105DB0003FFB123363850A82850B83A3A3A3A3E071
:105DC000702D850A82850B83126A9D700C12762ACB
:105DD000F0EE241812762D8010125FD5F0901A8BF9
:105DE000E014C0E0125FB8D0E0126008E4803490A4
:105DF0001A8BE004C0E0125FB8D0E0125FFBC394DE
:105E000003EE4003025EB61276EB7402125FFB648F
:105E1000017003025EC3EE2415125FD8F0EE241663
:105E2000125FD8F0EE241AFE50010F050DE50DC3E8
:105E300095094003025EEEE508C3950C4003025E3F
:105E4000CCAA087B00123DA78A0A8B0B0508901A82
:105E500078125FE1850A82850B83126248125FB077
:105E6000F583E8F0A3E9126018850A82850B83A305
:105E7000A3A3A3A3A3A3A3A3A3E0C0E0125FA6D000
:105E8000E0F07401122E61E4F0850A82850B831222
:105E900062487402122E61E812782F7401122BE30B
:105EA000123D1DE964016003025DA57404122E61B8
:105EB000125FC6025DB5125FD6125FFB640360031A
:105EC000025E16EE241512762D025E1CE50CC395BB
:105ED0000E4005750800801DE50EC3950CF5088081
:105EE00014125FD5F0EE241AFE50010F050DE50DDA
:105EF000C39509505B740E122BEBAA087B007987BF
:105F0000123E6D05087418122E61125FE1741012B2
:105F10002E61125FC6EE2412F8E43FF9740E122EC1
:105F20006112651E88828983EAF0A3EB126008740F
:105F300003126018741D122E61E0C0E0125FA6D03B
:105F4000E012790CE849709912762A809775090059
:105F5000750A00780A122B7E7812122B7A780912B1
:105F60002B7EE50EF5097809122B7E7405122E6141
:105F7000E0FD7C00E51412649B3515FBE5141276F8
:105F80001B3515F583E0F9123A657405122B8DE582
:105F90001245136007AA12AB131234237425122B77
:105FA0008D7F0E022819EE2419F582E43FF5832235
:105FB000EE2412F582E43F22125FBC22EE2418F593
:105FC00082E43FF58322AC82AD83EE240AFAE43FFB
:105FD000FB12353122EE2414F582E43FF58374017F
:105FE00022126CA28E828F83E8F0A3E9F07C8C7D74
:105FF0001AEE12649B3FFB12353122F0850A82852E
:106000000B83A3A3A3A3E02212766E7402F0EE2406
:1060100016F582E43FF58322F0EE2417F582E43F83
:10602000F5837402F0125FBC74FFF02274F612253F
:106030009374F9122C0B1276F23509127B838518B2
:1060400082851983122E4A8E828F83A3A3A3A3E095
:10605000C0E07404122E61D0E0127921F8740512A8
:106060002E617401F07406122E617401F090184DC7
:10607000F090185604127710FAA3E0FB90184E1215
:106080005A97E890185712609F90184CF0AA18ABD6
:1060900019123E0DE96003123E13740702551EF0FB
:1060A000E508240F12741E2274F212259374FF1255
:1060B0002C0B7508007E007F0012435F8A0A8B0B51
:1060C00012622880080508126234126248E849709A
:1060D000F49019E8E06007640160030261A01262B5
:1060E000288006126234126248E849603388828947
:1060F0008312651E901A78E06A7003A3E06B600A51
:1061000012623412651EEA4B70D98882898312624A
:1061100048901A78E0687003A3E06970030261A0F8
:106120007A167B001278A46077901A781262488AF7
:10613000828B83E812782F901A6D126D84F01244CE
:10614000C1E98E828F83A3A3A3A3A3F0901CBEE01A
:106150008E828F83A3A3A3A3A3A3F07C8C7D1AEECE
:10616000240B125FCDAA18AB197941123C21851876
:1061700082851983E0600890184312624880047891
:10618000FE79FF8E828F83A3A3A3A3A3A3A3E81208
:10619000782FEE12623C3F12624C8E0A8F0B05087C
:1061A000901857E0F8E508C398500479008027E577
:1061B00008C398F9C39406400279057800800DE57C
:1061C0000A12623C350B125C6BF50B08901857E015
:1061D000FAE8C39A40E97509007809122B7E780A1B
:1061E000122B7AE9F5097809122B7E901857E0F501
:1061F000097809122B7EAD087C007A4E7B18901826
:106200004CE0F9123A5F7405122B8D9019E8E060AA
:10621000046401700BEE4F6007EEFAEFFB123423BB
:10622000123E13740102795F12435F8A0C8B0DA832
:106230000CA90D22E812623C39F583222414F58260
:10624000E422851882851983126CA222F583E50A5F
:10625000F0A3E50BF02274F012259374FF122C0BBF
:106260008A0A8B0B7E008E0E8E0F1276F6125C4A17
:10627000126383FFAC18AD197A007B00799D123E42
:106280006D851882851983E0F8EFC3984003026397
:106290002AE0C39FFEC3940B40027E0AEE75F0070E
:1062A000A4FAABF01264938A0E8B0FEA4B607975F7
:1062B0000C00801A850882850983A3A3A3A3A37475
:1062C00003F0E5082407F50850020509050CE50C64
:1062D000C39E5056AC08AD09E50C2FFAE43400FB20
:1062E000798B123E6D850882850983A3A3A3A3A39E
:1062F000E014600814601314601F80B8850882855C
:106300000983A3A3A3A3A3E480B785088285098397
:10631000A3A3A3A3A3740180A8850882850983A3EE
:10632000A3A3A3A3740280997E00750800780812C5
:106330002B7E780E122B7AEEF5087808122B7EEF62
:10634000F5087808122B7E7405122E61E0FD7C00A2
:10635000E50A12649B350BFBE50A12761B125C4AB8
:10636000E0F9123A6B7405122B8DE50E450F6007AC
:10637000AA0EAB0F1234237401122B8D02540B1290
:106380005A54A3125A52E02274EE12259374FE124C
:106390002C0B8A0C8B0D7510007511001276F635DA
:1063A0000DF583126383F50AAC18AD197A007B00F2
:1063B00079A312414F126242C3E50A98E4995074DE
:1063C000851882851983A80AE0C398FEA3E094008B
:1063D000FFC3EE9404EF940040067E037F00800428
:1063E000EE4F6050EEFAEFFBEA75F015A4FAA8F054
:1063F00075F015EBA4281264928A108B11EA4B6099
:1064000033750B00750E00801FAC08AD09A80AE5B6
:106410000E28FAE43400FB79A212414FE508241556
:10642000F50850020509050EC3E50E9EE49F40D90C
:10643000EEF98005750B8B79007508007808122B32
:106440007E7810122B7AE9F5087808122B7EE50A7F
:10645000F5087808122B7E7405122E61E0FDAC0B56
:10646000E50C12649B350DFBE50C12761B350DF522
:1064700083E0F9123A717405122B8DE51045116015
:1064800007AA10AB111234237402122B8D7F0A025B
:106490002819FB12341D8A088B09222402FAE422EF
:1064A00074F612259374FF122C0BEAFEEBFF1264B4
:1064B000F912651E8A82F583A3A3A3A3A3A3A3A3B2
:1064C000E0F9123E31E9851882851983F0750800DC
:1064D0007808122B7E7401122BDB88088909780852
:1064E000122B7A7508357509807808122B7A126597
:1064F00001122B8D740102551EEA1276FB3FF583C3
:1065000022790112650DFAE43F1265EF22EE2402B2
:10651000FCE43FFDEE240F22851882851983127456
:10652000512274F412259374FA122C0B1276F21283
:106530007185127821FFEEFAEFFB123CF9E9600F4A
:106540001265F6EEFAEFFB12352BE96401700A745E
:1065500001122E61E4F0A380097401122E61EEF0A5
:10656000A3EF12794CF8A2E650087403122E61745E
:1065700001F0E8A2E750087404122E617401F0746F
:1065800005122E61E4F004122BE3123E61E9851836
:1065900082851983F090810A122E3212445B7A00B0
:1065A0007B001244677A007B00124461750A007810
:1065B0000A122B7E7401122BDB880A890B780A12CF
:1065C0002B7A750A34750B80780A122B7A1265D8EB
:1065D000122B8D740602546D7901E5082402FCE447
:1065E0003509FDE508240FFAE435091265EF22FBB1
:1065F0001239C97405221244378A0A8B0BAC0AADD2
:106600000B2274F612259374FF122C0B12671FF8DD
:10661000A3E08882F583E0F509A3E0F508A9091253
:106620003E1FE9851882851983F09019E8E0700B08
:10663000740165087005A909123B2BEE240B126743
:106640002670277508007808122B7E7401122BDB48
:10665000880889097808122B7A75083675098078B8
:1066600008122B7A126501122B8D0264F4C082C0CD
:10667000839019E8E07003123B31D083D082022B63
:106680002274F412259374EF122C0BEAFEEBFF1226
:106690006744F508E439F509901843E06A7003A3EC
:1066A000E0697052A818A919880A890B780A122B78
:1066B0007A750A11750B00780A122B7A7C007D001E
:1066C0007A817B001234A77404122B8DE970277530
:1066D0000A00780A122B7E7401122BDB880A890BC0
:1066E000780A122B7AAC08AD0912672D123A23747E
:1066F00003122B8D8024750A11750B80780A122BDA
:106700007A7808122B7AEE240E126726FD7C84120A
:10671000672D123A2F7404122B8D741102546DEAF6
:10672000FEEBFFEA2413F582E4125C5D221267316E
:1067300022EE2402FAE43FFBEE240FF582E43FF55B
:1067400083E0F92212674822EA2413F582E43FF538
:106750008312701B8882F583E0FAA3E0F8E4C8F99D
:10676000EA282274F112259374EB122C0BEAFEEB4B
:10677000FF1276F6126883FAE4CAFBEC2AF5089059
:106780001843E06C7003A3E06B6003026828888202
:106790008983A3A3E09410500F88828983A3A3E088
:1067A000851882851983800885188285198374105D
:1067B000F0E0C0E07404122E61D0E0127810A982DB
:1067C000AA83890C8A0D750E00780C122B7674073B
:1067D000122E61E0FC7D007408122E61AA82AB8348
:1067E000127193122B8D7404122BDB880A890B789B
:1067F0000A122B7A750A11750B00780A122B7A7C13
:10680000007D007A817B001234A17404122B8D74F8
:1068100004122E61E09018826005E0D2E48003E06B
:10682000C2E412688BE48008851882851983748419
:10683000F0E0C0E07401122E61D0E0F07402122E7C
:1068400061E508F07403122E61E508F012687C3FE0
:1068500012746A122B7E7402122BDB880889097865
:1068600008122B7A7508147509807808122B7A792A
:1068700003126503122B8D7415026FA9EE240EF519
:1068800082E4223F127834FCA3E022F0851882854E
:1068900019832274F612259374E0122C0BEAFEEB96
:1068A000FF901A7AE064086008E064046003026AFA
:1068B00077AC18AD191239B19019E8E0640270276D
:1068C0001244377402122E61AC82AD8312352BE96B
:1068D0006015126A7C851882851983E0687003A3AD
:1068E000E0697003026A7712460B7402122E61ACE3
:1068F00082AD83126518124509E964017003026ACA
:10690000777418122BE31244497402122E61AC8280
:10691000AD837418122BE312352BE9602D1244431A
:106920008A088B09A808A909851882851983E06857
:106930007003A3E0696013126242901A6EE8127845
:106940002F7A6E7B1A794B123C279019E8E060048D
:1069500064017067126A7CEE241112672668700366
:10696000A3E06960567402122E61AA82AB83123DC5
:10697000838B09A909EA4960268A828B83A3A3A392
:10698000A3E06401600D8A828B83A3A3A3A3E064C8
:1069900002700C7402122E61AA82AB83123D8F909A
:1069A0001B08126A9D60149019DCE06401700C12DF
:1069B0006518901B09125A5512277979001265182B
:1069C000123FB1901A78126A92FD1265181245C3EF
:1069D000740B122E61E4126AA3740C122E61E81279
:1069E000782F740B122BE3123D1DE9603F7C087D6C
:1069F0000079007418122BE3123363740E122E61A7
:106A0000AC82AD837418122BE312352BE9601D7430
:106A100002122E61AC82AD83740E122E61AA82AB7B
:106A200083123CF3740B122BE3123D2F7402122ECF
:106A300061AC82AD83740E122E61AA82AB83123CCC
:106A4000F3740B122BE3123D23E9602B740C122E0E
:106A500061126248851882851983E0687003A3E09B
:106A6000696014126242740C122E61E812782F745D
:106A70000B122BE3123D2F742002551E12443D8A47
:106A8000088B09A808A90922FAE433FB12341D90E7
:106A90001942E0FCA3E022F582E438F583126CA2EF
:106AA000E84922F0851882851983126CA22274E8C5
:106AB00012259374F7122C0B8A168B177F008F0800
:106AC0008F091239B78A128B13EA4B7003026C716B
:106AD0007E00800DEE75F00CA4F8126C76123D8FDE
:106AE0000E851282851383E0F8EEC3984003026B93
:106AF000AF750CFF750DFF750EFF750FFFEE75F08E
:106B00000CA4F8A9F0126C76123D83EA4B60D18A8E
:106B1000828B83A3A3A3A3E06401600D8A828B838D
:106B2000A3A3A3A3E0640270B7126D54700C126D9E
:106B30007E122DD4126D48122BF3EE75F00CA4F8D2
:106B4000A9F0E51228F582E513126D6F122AFD40B7
:106B5000837A0E7B0012341D8A0A8B0BEE75F00CC3
:106B6000A4F8A9F0126C7EAC82AD831279A6780CE1
:106B7000122DF2E50A240C125C47E4F0A3F0E508BC
:106B80004509700E850A10850B11851008851109BD
:106B90008019E510240CF8E43511F9888212624C52
:106BA00088828983E0F510A3E0F5110F026AE0EF17
:106BB0007003026C6A7408122E617402126C95855F
:106BC0001882851983E812782F7E00EF75F00CA4E7
:106BD000FAABF012341D8A0C8B0DEA4B7003026C79
:106BE0006A8051850810850911EE75F00CA4F8A98A
:106BF000F0E50C28F50AE50D39F50BAC08AD09AA4E
:106C00000AFB1274FFA3A3A3A3A3A3A3122E0E85B2
:106C10000A82850B83A3A3A3A3A3A3A3A3122E4A33
:106C20000EE510240CF582E43511126C8BAA10AB22
:106C300011123423E508450970A975080078081277
:106C40002B7E75081F7509807808122B7A780C1234
:106C50002B7AEFF97405122BEBE516240FFAE435C5
:106C600017FB1239FF7405122B8DAA12AB131234C5
:106C7000237409025A46126C7EAA82AB8322E51263
:106C800028F582E51339F583A3223BF583E0F50867
:106C9000A3E0F50922F0851682851783A3A3126C61
:106CA000A22212701BF92274F01225931239B78AAE
:106CB000088B09AE08AF09EA4F7003026D457508ED
:106CC00000806F750CFF750DFF750EFF750FFFE5EA
:106CD0000875F00CA4F8A9F0126D61123D83EA4B1F
:106CE000604E8A828B83A3A3A3A3E06401600D8A14
:106CF000828B83A3A3A3A3E064027034126D54704B
:106D00000C126D7E122DD4126D48122BF3E508750E
:106D1000F00CA4F8A9F0EE28F582EF126D6F122A9C
:106D2000FD500DE50875F00CA4F8126D61123D8F51
:106D300005088E828F83E0F8E508C3984085EEFA57
:106D4000EFFB12342302540BEA2417F582E43BF5DF
:106D500083780C22EA241BF582E43BF583E064018E
:106D600022EE28F582EF39F583A3AA82AB8322397C
:106D7000F583A3A3A3A3A3A3A3A3A3780C221278B0
:106D8000B6780C221279B8A3A32274F11225937459
:106D9000F6122C0BEAFEEBFF750800901942126AFE
:106DA0009D70457A377B0012341D901942125A9714
:106DB000F9EA4960197C377D007900123363EEFCF3
:106DC000EFFD90194212651E123981E9700B85188A
:106DD000828519837488026F1C1277F112749C7477
:106DE00001F0127441026FA7E8242EF582E439F510
:106DF000837402F0EAFCEBFD127427123981E9700A
:106E00000C8518828519837488F0750801750A0C41
:106E1000750B19780A122B7A1270AEF582E438F5E8
:106E2000831229A51277F1242812740EFC1270A87F
:106E3000126FC82414126FB1122B8D126FBF127013
:106E400007243112740E603A1274E9126A88CC2455
:106E500032126FF96020750C0C750D19750E0078E3
:106E60000C122B761274E9FCE433FD1270A2126F3F
:106E7000EC122B8D800C8518828519837488F0752F
:106E80000801780A122B7A12709CF582E438F58397
:106E90001229A51277F1241112740EFC12709612A9
:106EA0006FC8242B126FB1122B8DE9F81277F124E1
:106EB00034127007243412740E602E1274E0126AB9
:106EC00088CC2435126FF96042750C0C750D19755C
:106ED0000E00780C122B761274E0FCE433FD12776E
:106EE000F12435126FEC122B8DE508A2E04025123B
:106EF0006FBF12740E70089019421274AC60157B4B
:106F0000007A007900123987026FA78518828519E7
:106F1000837488F08518828519837486F074091249
:106F20002E617402127805126FE5122E61E8F0A34B
:106F3000E912780512746C122B7E7401122BDB8817
:106F40000889097808122B7A750820750980780855
:106F5000122B7A79017406122BEBEEFAEF1265EF21
:106F6000122B8D127492703C7409122E61740212ED
:106F7000750E126FE0122E61127512122B7E7401C3
:106F8000122BDB880889097808122B7A750820757E
:106F900009807808122B7A79017406122BEB12748F
:106FA00057122B8D12397B740A122B8D7F07022802
:106FB00019F582E438F583E0F91238DF7404229081
:106FC0001942126FD6243122F582E43812744F121E
:106FD0006FD322901942126FDA22E0F8A3E0C822A0
:106FE000F5838882A3A3126CA2740122F582E4388F
:106FF00012744F123357740322F582E43CF583EA8E
:10700000F0A3EBF0EA4B22F582E438F5831270121C
:10701000C822E9F012701822901942E0F8A3E02289
:10702000C082C083901942126A9D6067E82435F5DA
:1070300082E439126A9B60081277F124351270B429
:107040001270A2126A9760061270A21270B41270C7
:107050009C126A97600612709C1270B41270A8128B
:107060006A9760061270A81270B41270AE126A9716
:1070700060061270AE1270B4127096126A976006B3
:107080001270961270B49019421270BA901942E4BC
:10709000F0A3F002667A126FD3242C22126FD3244D
:1070A0001222126FD3243222126FD3241522126FB0
:1070B000D3242922F582E438F58312745112342343
:1070C0002274F1122593EAFEEBFF8C088D09750AF4
:1070D000018C0C8D0D750E00780C122B767C177DB3
:1070E00000127193122B8D12765AE5082411127139
:1070F00082E060271279E41271B0601CE508241266
:107100001271A4122B76E5082411127199125FB145
:10711000126FF0122B8D8003750A00E508241412FB
:107120007182E060251279E4EE24151271B360419A
:10713000E50824151271A4122B76E50824141271A7
:1071400099127177126FF0122B8DE50AA2E0401CA4
:10715000125FB0126A9B6006125FB01270B81271B3
:1071600076126A9B60061271761270B8A90A026FD5
:10717000AC750A0080DAEE2415F582E43F22E508BA
:10718000240BF582E43509F583227D00EE2404FA10
:10719000E43FFB12335774032212741E25E0FCE413
:1071A00033FDEE2212741EF50CA3E0F50D780C22CF
:1071B000EE2412F582E43FF583EAF0A3EBF0EA490E
:1071C0002274EE12259374ED122C0B890B8A0E7526
:1071D0000C00750D00750AFF7510FF7511FF75081D
:1071E00000750900851882851983E412750EF9E887
:1071F0004960167403650B60067402650B700FE03E
:10720000C8243012740E6B600579000274097C8DFD
:107210007D397A007B001240477401650B700A8546
:1072200018828519837485803DE50B6006740365BB
:107230000B7019901942127472F07403650B702967
:10724000E50E6029851882851983801A7402650B02
:10725000701BE50E90194270051274728008127747
:10726000F41274897402F08004E50B601E127478C5
:1072700070191274A56005126FC2800A1274AC6096
:107280000A1277F1243412740E14F01274A56018E7
:10729000126C8D1274E912798ACA24321274BD24D8
:1072A0001D127434242580261274AC602A90194271
:1072B000E02417F508A3E03400F5091274E0127910
:1072C0008ACA24351274BD2406127434240EF58241
:1072D000E43AF583E0F50A7409122E61740212682B
:1072E0008BE0600302737EE5084509700302737E3C
:1072F00012747870047E2280027E218508828509BE
:1073000083126FE4122E61E812782F901946E0C0C4
:10731000E01277F12430F582E438F583D0E0F074A0
:1073200012122E617403F0AC0CAD0D740A122BE333
:107330001274FFE0F50C780C122B7E780A122B7E6B
:10734000740C122BDB880C890D780C122B7A7810B8
:10735000122B7AE5082406F50CE43509F50D780CB6
:10736000122B7A127416F97409122BEBEEFA7B00C9
:10737000123A3B7408122B8D12744102740712707A
:1073800018126FE0122E61127512122B7E74011208
:107390002BDB880889097808122B7A750820750973
:1073A000807808122B7A79017406122BEB1274572D
:1073B000122B8D127492704C1277F12419F582E41D
:1073C00038F583126FE6122E61E8F0A312700D24D7
:1073D00018F582E43812746A122B7E7401122BDBCA
:1073E000880889097808122B7A7508207509807831
:1073F00008122B7A79017406122BEB12742712658E
:10740000F0122B8D12397B7901741302648AF58294
:10741000E438F583E022E508240E12741E22F5827A
:10742000E43509F583E022901942E02417FAA3E03D
:107430003400FB22F50CA3E03400F50D901942E076
:10744000227C8D7D39901A1712745112404722F513
:1074500083E0FAA3E0FB229019421274511265F006
:1074600022E516240EF582E43517F583E0F5087859
:107470000822127482740122901942127482E0640C
:107480000122126FDA12748922242FF582E438F572
:107490008322126FD312749CE0640222242EF582A0
:1074A000E438F583221274EF901942221274B0224C
:1074B000126FDA2434F582E438F583E022F582E4B1
:1074C0003AF583E028F8A3E039F9E824FEF582E9EB
:1074D00034FFF583E0F510A3E0F511901942E022A6
:1074E0009019421274B025E0221274EF25E0229028
:1074F0001942126FDA2431F582E438F583E0221262
:10750000750322123531850882850983A322127002
:107510001322E8F0A3127012F5838882A3E0F50825
:10752000780822C082C0837B007A8579011239876E
:1075300002667A74F4122593ECFEEDFFEA240F1232
:10754000790012793A1262488C828D83A3A3E812E3
:10755000782FEA240E1279001255CB126C8A850816
:1075600082F5831279F312782EE5082402F508508B
:10757000020509FCAD09EE240612764AC0E0126845
:107580007C3FF583D0E0F0E5082409F508500205BA
:1075900009F582850983127991F9EE12761B3FF580
:1075A00083EA12782F12765A850882850983A3A36D
:1075B000E0F8EE241112770150020509E860191273
:1075C00076211271B06011EE241212763D24111250
:1075D00076358A088B098007EE241112762DF08506
:1075E0000882850983E0F81276EAE81278C4858279
:1075F00008858309601EEE2414126726127621EE98
:1076000024151271B3600DEE241512763D24141268
:107610007635800412762AF0025470240FF582E445
:1076200022F81279DA8B0BA90B22EE2414F582E4EE
:107630003FF583E422125C5AF912390322125C5A94
:10764000FCA3E0FDAA08AB09EE22FAE43FFB1275A9
:1076500003A3A3A3A3A3A3A3E022EE2412F582E431
:107660003FF583E4F0A312766EE4F0A3F022F0EE8F
:107670002415F582E43FF5832274F6122593ECFE7F
:10768000EDFF1276F6126C8AAC08FDEEFAEF127678
:107690004D8E828F83A3A3A3A3A3A3A3A3F0E50886
:1076A0002409F50850020509F582850983127996A7
:1076B000A3F0A3E9127710F8EE2413127701500219
:1076C00005097403687013AC08AD09EE240B12763B
:1076D0004AC0E01276EAD0E0800C850882850983F2
:1076E00012797BF0A3E9F0025521EE12623C3FF5DE
:1076F00083228A088B091276FA22EA2413F582E49F
:1077000022F582E43FF583E8F0E5082403F508223A
:107710001278C8A3E02274F2122593EAFEEBFF75FB
:107720000A00EA2410126726C3940C400D1264F973
:107730001277F4240B12740EF50AA80AE828F8E46C
:1077400033F9E8240D12796770030277DEEE1267D1
:1077500024FEA3E0FF8E82F583E0F88A828B8312F9
:107760007805AE82AF837076EEFCEFFDEA2403125B
:1077700077F850010FF5828F83125D1E8508828590
:10778000098312782E12717EE4F0E50A6050E50854
:10779000240DF8E43509F98E828F83A3A3E0C0E0BD
:1077A00012717ED0E0127926C0E01277E5D0E0F0C9
:1077B000EE2404FE50010F850A0B8E828F83126A1D
:1077C00092FBEC88828983125A98E82402F85001CF
:1077D00009EE2402FE50010F150BE50B70DCAA0820
:1077E000AB09027962E508240CF582E43509F583DA
:1077F00022901942126FD622FAE43509FB12353174
:10780000EE2408FE2212780922F08E828F83A322B2
:107810001278142212781822F088828983A3A3A3F5
:1078200022E0FEA3E022A3E0F9EA8C828D83A3F09C
:10783000A3E9F022F58312701BF98882F583E02218
:1078400074F11225931278B2E0F508A3E08508825E
:10785000F583E0F50BA3858208858309A3A3E0F5F2
:107860000A12789D60308A828B83E50BF08508824E
:10787000850983E0FA1279BEE50A1278C4A3A3A9A8
:1078800082AA83890C8A0D880E780C122B76AC0A9A
:1078900012718A122B8DEEFAEFFB026FAC2404FA00
:1078A000E43400FB12341D8A0C8B0DAE0CAF0DEAD4
:1078B0004F221278B6221278BA22EA2413F582E413
:1078C0003BF583221278C822F0850882850983A3BC
:1078D0002274F7122593EA2413F8E43BF98882F521
:1078E00083127991F5838A8212790612790C888243
:1078F000F583A3E0FA88828983A312782602538D48
:10790000F582E43BF583E08C828D83221279131299
:107910006CA222F08882898322FAE439FB12341D9A
:1079200022127954E022127809A3A3E0221278BA35
:10793000E0FEA3E08E82F583E0221279ECA322120E
:10794000794322F08A828B83A3A3A322127954A3C2
:10795000A3A3E022F08E828F83A3A3A3A3A322126A
:107960002B8D7F06022819FAE439126492EA4B2221
:10797000E0F50FA385820A85830B22127991F9EE37
:10798000240BF582E43FF583EA22F8E433F99019F9
:1079900042E0FAA3E022125D228E828F83A3A3A38A
:1079A000A3A3A3A3A322123531850A82850B83A347
:1079B000A3A3A3A3A3A3A322E08A828B8322A3E091
:1079C000F8E4C8F9EA8E828B83A3F0A3E9F08E82F3
:1079D0008B83A3A3A3221279DA2225E0FAE433FBF6
:1079E00012341D221279DA8B0DA90D22F08A828BB6
:1079F00083A322125D228C828D83A3A3A32274F61B
:107A00001225938C088D09127A3CFF125D1A8C8224
:107A10008D8312782FE82402FE50010FFCEFFDE564
:107A20000812649B3509FB1235318E828F83A3A324
:107A3000A3127B57A3A3A3A3F00255211278B61279
:107A4000701B2274F2122593127ABA75F00CA4A955
:107A5000F024011279198A0C8B0DEA4B60558A8249
:107A60008B83A38582088583098A828B83E50BF04B
:107A7000750A008037EEFCEFFDAA08AB091277FD0E
:107A800050010F7904127B90850882850983A3A396
:107A9000A3A3A3A3A3A3122E4AEE2404FE50010F16
:107AA000E508240CF50850020509050AE50AC39506
:107AB0000B40C2AA0CAB0D02796212792DF50BA313
:107AC000AE82AF8322127991F8E4C8F9EA28221233
:107AD0007943A3A3A3A32274F61225938C088D09DE
:107AE0001276F63B127B83850882850983122E4A23
:107AF0008E828F83A3A3A3A3E0F8850882850983E0
:107B0000A3A3A3A3F0C3940650098E828F83127B94
:107B10005C8040850882850983A3A3A3A3E064FE5B
:107B2000600E850882850983A3A3A3A3E0F47024D3
:107B30008E828F83127B57F0EE2406FE50010F8554
:107B40000882850983A3A3A3A3E0F47007127B6EC8
:107B5000F0A3E9F0025521127B5CA322A3A3A3A307
:107B6000A3E0850882850983A3A3A3A3A3228E8211
:107B70008F83125D22850882850983A3A3A3A3A313
:107B8000A3A322F583127821FF7904EE127B9022C1
:107B9000FAEFFB12336FEAF8EBF9ECFAEDFB227423
:107BA000F712259312494112485712473D790112A5
:107BB0003C1BE9FE79FF1233CFEEF9806574F712B2
:107BC000259374FF122C0B12493BE9FE8518828520
:107BD0001983E4F0AA18AB1979561230157A407B54
:107BE0000D79E2123015127CF060129019EEE0FA75
:107BF000A3E0FB1234239019EEE4F0A3F0EEF98039
:107C00001C74F7122593E9FE74E26E700B7C407DC4
:107C10000D1235317900800312300F800574011286
:107C20002B8D7F0102281974F71225938908EAFE2B
:107C3000EBFF74E269700BEAFCEBFD7A407B0D12FE
:107C40003531EEFAEFFBA90812301580D5C082C09D
:107C5000838A828B83A3A3A3A3A3A3A3A3E4F01289
:107C6000485D027E6BC082C0838A828B83A3A3A3FC
:107C7000A3A3A3A3A3E4F0124743027E6DC082C076
:107C8000838A828B83A3A3A3A3A3A3A3A3E4F01259
:107C90004749027E6B74F6122593EAFEEBFF8A8257
:107CA000F583122E0E9019EA122E4A127CF060040F
:107CB00079FC80238E828F83A3A3A3A3E064036057
:107CC000138E828F83A3A3A3A3E0700D127F3B606A
:107CD0001B127F51127F2580228E828F83A3A3A344
:107CE000A3A3A3A3E060ED127F6F70E8791A80E789
:107CF0009019EEE0F8A3E0F9E849227F0202281982
:107D000074F712259374FF122C0BEAFEEBFF851813
:107D1000828519837401F0AA18AB197952123015B3
:107D2000EE2415F582E43FF583E4F0EE2420F5829D
:107D3000E43FF583E4F0EEFAEFFB12474F790002DF
:107D40007C1DC082C083EA2413F582E43BF583E402
:107D5000F0124863027E6B74F11225938A088B0936
:107D60008C0A8D0BEA241C127E55FBEA241B127E22
:107D700055FA127E51F91247CD8A0C8B0DAE0CAF1D
:107D80000DEA4F7003027E4A85080C85090D750EB9
:107D900000780C122B767C117D00EA2423FAE43F54
:107DA000FB1233577403122B8DE508241F127E55E6
:107DB000F50CA3E0F50D780C122B76127E51FC7DAC
:107DC000008E828F83A3A3E0FAA3E0FB12335774E3
:107DD00003122B8DE508241350020509F50C8509C3
:107DE0000D780C122B767C0B7D00EE2418FAE43F04
:107DF000FB1233577403122B8DE50A450B60408E3E
:107E0000828F83A3A3A3A3E060358E828F83A3A375
:107E1000127CF3602A8E828F83A3A3E0FAA3E0FB97
:107E20008E828F83A3A3A3A3E0F9850A82850B83A7
:107E3000122779E96009EEFAEFFB123381800BEE2D
:107E4000FAEFFB1247C779008002791A7F070228F0
:107E500019E508241EF582E43509F583E022C08285
:107E6000C0837C007D00123C5180027900D083D019
:107E700082022B227900027C22C082C083122EBF94
:107E800080E9C082C083122EC580E2C082C0831206
:107E90002ECB80D974F7122593122ED180D674F48C
:107EA0001225938A088B09ECFEEDFF7B007A00799E
:107EB000001247CDEA4B605EEA242EF582E43BF5E2
:107EC000837402F0EA2423F582E43BF583E508F0AD
:107ED000A3E509F0EA242BF582E43BF5837402F074
:107EE000EA242CF582E43BF583EEF0A3EFF0EA24DC
:107EF0002FF582E43BF583E4F0EA2430F582E43B9D
:107F0000F5837431F0A3E4F0EA2420F582E43BF534
:107F100083E4F01247C77F04022819C082C083128D
:107F2000487B027E6D8E828F83A3A3A3A3A3A3E4C9
:107F3000F0EEFAEFFB1249897900227A1B7B0012DE
:107F4000341D8B09A9099019EEEAF0A3EBF0EA4978
:107F5000227C1B7D0079001233639019EEE0240B24
:107F6000F8A3E03400F9127F90E8F0A3E9F022755D
:107F7000F021A4FAABF012341D8B09A909127F90ED
:107F8000EAF0A3EBF09019EEEAF0A3EBF0EA492255
:107F9000EE2416F582E43FF5832274F612259375DC
:107FA0002900752A00752B008A2C8B2DEA90620B14
:107FB000F08A088B0974047808122DE3E5089062B2
:107FC00007F08A088B0974097808122DE3E5085434
:107FD0003E906209F0758B00C2E843AC20439A02E0
:107FE0007F020228197404F5D574E3F5D47404F5FE
:107FF000D374EBF5D2022B22851A87C2AF022B2253
:108000000000000000000000000000000000000070
:108010000000000000000000000000000000000060
:108020000000000000002403540049002000430029
:10803000430032003500330031002000550053006A
:108040004200200043004400430024035400650024
:10805000780061007300200049006E007300740016
:10806000720075006D0065006E0074007300A53C21
:10807000A548DB424140D740B73691389D357F3522
:10808000E9490000000000000000000000000000BE
:1080900000000000000000000000000000000000E0
:1080A00000000000000000303132333435363738FC
:1080B00039414243444546000000000000000000F2
:1080C000FFFFFFFFFFFFFFFFFFFFFFFFFFFFFFFFC0
:1080D000FFFFFFFFFFFFFFFF0000000000000000A8
:1080E0000008000400020001020502000801748279
:1080F000003A003B0000000000000000000000000B
:10810000000200020603E803000000000000000077
:10811000FF00FFFFFFFF03000000E9FFFFFF00007B
:1081200000FF09433886965118000400000019E04A
:10813000FCFFF8FF0000E71F0300805101003C0036
:108140000000100E00009F0200006AAEE7FF08006A
:108150000000FA000000040309041F000000FEFFF5
:10816000FFFF9751180060EA0000E2040000580287
:108170000000BC0200003200000000F8FF076400AD
:108180000000E90300000B0000000A0000001027B7
:108190000000000000000048000001000000300066
:1081A0000000000000000A74F7122593E9901AC538
:1081B000F0901A7AE4F0123327901ADDE4F0A3F07D
:1081C000901AC6F0A3F01245AB9019E8E060046481
:1081D000017006123D53123F1B12332D901A01E419
:1081E000F0A3F0123C5D02B40074EC12259374D736
:1081F000122C0BEAFEEBFF54806068901AC5E0F980
:108200001233938A088B09EA4509604F7C0080018C
:108210000CEC75F003A4F8A9F0745028F5827450A2
:1082200039F583E493F4602CE493F88508828B831A
:10823000E06870DCAA08EC75F003A4F8745128F526
:1082400082745039F583E493C0E0740193F583D0D0
:1082500082122779AA08AB09123381EEFAEF648003
:1082600002872DEF5420601E1243F58A088B09EA1D
:108270004509600A124311AA08AB09123381EEFACC
:10828000EF642002872D9019E8E06402705FEEA28F
:10829000E0501F901A7FE0640F701179001242E1E4
:1082A000E96009901CA5122E321242F9EE64010217
:1082B0008644EF5440603690187CE0640670287461
:1082C0000BF0901CBDE0F9750801750900750A00F6
:1082D000750B00901A6DE07808122ADEAA08AB0927
:1082E000AC0AAD0B123E3D9019D80286EBEE54203D
:1082F00070030286157A207B00901AC5E0F91234CB
:10830000F5EA4B4C4D701A901AD9122E0EE8494AD4
:108310004B700E750C01750D00750E00750F008009
:1083200061750C00750D00750E00750F0012350794
:108330008A088B098C0A8D0B901AD9122E0EE849E7
:108340004A4B602A901AD97808122AFD400E750C03
:10835000FF750DFF750EFF750FFF801285080C85E8
:10836000090D8C0E8D0F901AD9780C122BF3740115
:10837000780C122BC2E50C450D450E450F7003021B
:10838000853C7C0079047A007B001243BF8A088B0D
:108390000902846985188285198374FFF0740112BB
:1083A0002E6174FFF07402122E6174FF12A320FA82
:1083B000A3E0FB7403122BEB12D1B812441FE96443
:1083C00001600302844BE508240D12B0034480F8D9
:1083D000A3E0F97424122E61E8F0A3E912C511A3F9
:1083E000A3A3E0C0E07426122E61D0E012CFC0A398
:1083F000E0540860167424122E61A3E04401128731
:1084000050C0E07428122E61D0E0F0E50812ED5C57
:10841000350912CF99601CE508240F12CC88A3E01F
:10842000C812C4D938F583E0F87412122E61E8F04E
:10843000A3E4F090810A12299D7404122BEB7407B7
:10844000122BE3123E7F7404122B8D85088285095E
:1084500083A3A3A3A3A3A3A3A3A37406128750F982
:108460001243A1850A08850B09E508450970030236
:10847000853C7C007904AA08AB091243BF8A0A8BA9
:108480000B850882850983A3A3A3A3E0F510A3E0CD
:10849000F511E4F512F513780C7910122DB4402380
:1084A000E5082404F8E43509F9850C10850D1188D8
:1084B000828983C3E09510F0A3E0951112F1DF707B
:1084C000A2800E850882850983A3A3A3A3E4F0A359
:1084D000F0850882850983A3A3A3A3A3A3A3A3A3D1
:1084E000A3E06401850882850983A3A3A3A3A3A3B2
:1084F000702BE0540460030283948508828509830D
:10850000A3A3A3A3A3A3A3A3A37406F07AB7850888
:10851000828509831289331242F3028463A3A3A3E1
:10852000A3E06003028394850882850983A3A3A343
:10853000A3A3A3A3A3A37401F002846312438F7CBB
:108540000079017A007B001243BF8B09EA4509607C
:108550000C7A207B00901AC5E0F91233BD850C0A15
:10856000850D0B7C0079047A007B001243BFEA4B37
:10857000701580558A828B83A3A3A3A312E69BE583
:108580000898E5099940098A828B83A3A312874240
:108590007C0079041243BF8B0DA90DEA4970D5C345
:1085A000E50A9508E50B95095013C3E508950AF50A
:1085B00008E509950BF509E508450970147A207B53
:1085C00000901AC5E0F91233BD901AD9129B4C8065
:1085D0003FE50825E0F508E50933F509E4F50AF576
:1085E0000B7808122B727A207B00901AC5E0F912E2
:1085F00034E37404122B8D123507EAC0E0EBC0E0BF
:10860000ED901AD9FBECFAD0E0F9D0E0F8122E4A3E
:10861000EE6420802FE0600764016003028706EEAD
:1086200054106008123F57EE64108018EE544060FA
:1086300008123FCFEE6440800BEE5480600B123E78
:1086400025EE6480FAEF02872DEF5401600B12458E
:1086500081EEFAEF640102872DEF54086047123F64
:10866000279019D2E0640170349019D3E0602EF5A0
:1086700008E4F509F50AF50B908106780C122DD463
:108680007808790C12242E7808122B727A007B0855
:10869000901AC5E0F91234E97404122B8DEEFAEF4A
:1086A000640802872DEF54106012901AD7E060051D
:1086B000E4F0123F27EEFAEF64108071EF5440604F
:1086C00045901AFE12CF9B60369019DCE064017071
:1086D0002E901AFF12C8BD122779901B0412CF9B4F
:1086E000600612C8BD12277990810612299D7A0072
:1086F0007B40901AC5E0F91234E97404122B8DEE18
:10870000FAEF64408027EF5402600A12457BEEFACC
:10871000EF64028018EF5404601612CE6F79019056
:108720001A7812CC9C123E9DEEFAEF6404FB800492
:108730007A007B007429122B8D7F0C0228198E82FF
:108740008F83A3A312874822E0F508A3E0F509224E
:1087500012C515A3E022C082C08374EA122C0B7CE0
:10876000167D007900AA18AB191233637408122E13
:10877000617402F0901A6E129B1F12879674091290
:108780002E6112CCAB7413122E61E412CFD2123CC4
:108790004B741602D58BE8F0A3E9F0901A7812D545
:1087A0004E2274F712259374DA122C0BEAFEEBFFBB
:1087B000EE4F602DAC18AD1912441F7406122E61D5
:1087C000E0601E7417122E61E0FD7401122E61E04C
:1087D000FCEEFAEFFB79001242B7E9600479A4805D
:1087E000027900742602B3FD74F4122593EAFEEBBD
:1087F000FF8E828F83A3A3A3A3A3A3E05440601999
:1088000012E2FD12CC9C1244D9E960077AFF7BFF8B
:108810000288DD12E2FD0288D09019E8E06007646A
:108820000160030288C5901A65E0A2E14003028856
:10883000C512B44312CD9BA3A3A3A3E0FA888289F7
:1088400083A3A312D91A8E828F83A3A3A3A3A3A366
:10885000A3E054106004794080027900750AFE7527
:108860000BFF780A122B7A1289211229A5AC08ADC8
:108870000912E2FD12CC9C123F2D7404122B8DE5DF
:10888000086A7003E5096B600B12BF5A6A7003A394
:10889000E06B703F750A00780A122B7E79028E8297
:1088A0008F8312B504FCA3E0FDAA08AB0912451B97
:1088B0007401122B8D7508CDAA0812892F1242F36C
:1088C000E9604C80579019E8E0640270E8901A6EF5
:1088D00012CC9C74FE6A700374FF6B60D812E2FDC8
:1088E00012E16D1244D9E98E828F83600B12BC783D
:1088F00012F4B1E4F0A3800312F49FF07CE77D4210
:108900008E828F8312CC9C123C51E9F50870A9EE3F
:108910004F60097901EEFAEFFB12439BA908028F21
:10892000D1EE128926222411F582E43FF583228EAE
:10893000828F8312F488E0F92274F6122593E9FEFF
:10894000EAFF7A0F7B0012337BEA4B601F8A828B2F
:1089500083740CF0EEA3A3F0EF8A828B8312B1B97B
:10896000901AC5E0F91233877900802FEEF912438F
:10897000C58A088B09A808A909E849601C8882896A
:1089800083A3A3A3A3A3A3A3A3A3740612ED62E0EE
:10899000F9123FE1EEF91243A1791002C91A74F4F9
:1089A0001225938A088B098C0A8D0B901A7FE0643C
:1089B0000F702CEA4509450A450B6023901A7AE0AE
:1089C00064086005E0640470167808122B727A015E
:1089D0007B00901AC5E0F91234E37404122B8D0267
:1089E0008FD174F2122593EAFEEBFF8C0A8D0B896E
:1089F00008740E122E6112E6A0850C82F583E4F055
:108A0000A312CE64F5838882E0F91244B5E96026AA
:108A100012CC8F1244D9E96402701B8E828F83A31B
:108A2000A3A3A3A3A3A3A3A312BAE5850C82850DD8
:108A30008312CCAB800375080012B4FB14602E14B3
:108A4000604314606414606C146048147003028AFC
:108A5000D424FE7003028AEE147003028AF71470A5
:108A600003028B0A147003028B18028B2E780C12EF
:108A70002B7AAC0AAD0BEEFAEFFB123F3F740212F9
:108A80002B8D028B13AC0AAD0BEEFAEFFB123F45B8
:108A9000028B3812CC8F1244D9E96003028B2EEE80
:108AA000FAEFFB123F93028B38A908EEFAEFFB12A4
:108AB0004521805F12B97964027073E508700A126B
:108AC000E2237003A3E069706FEEFAEFFBA90812CE
:108AD00044A9803F12E2237003A3E069705012B9E9
:108AE0007964027049EEFAEFFB124491804AEEFA83
:108AF000EFFB12459F804112E2237003A3E06970EF
:108B00002DEEFAEFFB12452D802EEEFAEFFBA908B1
:108B1000124539E9F50880209019DCE064017009FC
:108B2000EEFAEFFB124545800F750800800A7508C4
:108B3000007AD37B00123873A9088007A90A74034E
:108B4000122B8D7F0602281974F412259374D61205
:108B50002C0B8A088B098A828B83A3A3E0F912432A
:108B6000C58A0A8B0BAE0AAF0BEE4F7003028C7AEC
:108B7000850882850983A3A882A983E0C0E012CC7E
:108B800076D0E012E6ADE064F160338508828509B5
:108B900083A3E064CD6027850882850983A3E06410
:108BA0001A601B850882850983A3E064E9600F854C
:108BB0000882850983A3E064E16003028D72901945
:108BC000E8E0600764016003028C9B8E828F83A3C0
:108BD000A3A3A3A3A3A3E054087003028C9B8E82DB
:108BE0008F83A3A3A3A3A3A3A3A3A37405F09019A6
:108BF000E8E0600464017053850882850983A3E07E
:108C000064E96047901AFA12CF9B600612C8BD1241
:108C10002779901AFC12CF9B6031901A65E0A2E18F
:108C2000502912D18EA3A3A312B9B78882898312C7
:108C3000CC9C1245DBEA4B6012850882850983A330
:108C4000E0F9901AFC12E3011227798E828F83A338
:108C5000A3A3A3A3A3A3A3A3E0640270108E828F97
:108C600083A3A3A3A3A3A3A3A3A37406F08508824D
:108C7000850983A3A3E0F91243A112438F9019E859
:108C8000E064027011901CABE0F508A3E0AA08FBB9
:108C9000E4FCFD1242F9742A028FCE790012439B44
:108CA000E97003028D729019E8E0600764016003C7
:108CB000028D47901A65E0A2E14003028D4712CF72
:108CC000967003028D478E828F8312CC9C7404129F
:108CD0002BEB12D1B812441F850882850983A3E0CB
:108CE00064E97023128E7C122B7E850882850983AD
:108CF000A3E0F50A780A122B7E128E8912CC9C1200
:108D000044557402122B8D740D122E6112CF8C12E9
:108D1000F10A12CCAB7409122E61E0600479408034
:108D2000027900740F122E6112B9B7740D122E6100
:108D300012CC9C123F39E9600E8E828F83A3A3A3CD
:108D4000A3A3A3E04420F0EE2404F50AE43FF50BCE
:108D50008E828F8312B010E0F9850A82850B831210
:108D6000CC9C123339850A82850B83EAF0A3EB028F
:108D70008BED850882850983A3E0C0E07402122E82
:108D800061D0E012A80012E109E508240B12B0033B
:108D9000C0E07403122E61D0E012E970E0AA18ABB3
:108DA000197031123E799019E8E06004640170276F
:108DB0007402122E61E0701F12E2FD12CC9C12446C
:108DC000D9E97039901AFA12CF9B603112C8BD12DE
:108DD000277980031244AF7402122E61E064E970B7
:108DE0001C128E7C122B7E750AE9780A122B7E12D9
:108DF0008E8912CC9C1244557402122B8D9019E866
:108E0000E0600764016003028C4B901A65E0A2E108
:108E10004003028C4B8E828F83A3A3A3A3A3A3A39F
:108E2000A3A3E06402703C8E828F83A3A3A3A3A3B9
:108E3000A3E05404602D12E2FD12CC9C1244D9E947
:108E40008E828F83700F12E30174FFF0A312A9B01A
:108E50007405028C6CA3A3A3A3A3A3A3A3A374036D
:108E6000028C6C850882850983A3E064E9600302B3
:108E70008C4BEEFAEFFB124557028C4B8E828F83A0
:108E800012DA50750A01780A22E508240C12BF791B
:108E9000E0F98A828B83A3A3A3A3A3A3A3A3A31212
:108EA000D9122274F4122593EAFEEBFF75080075BF
:108EB00009008E828F83A3A3A3A3A3E0603B750860
:108EC0000812CC8F79FF1240E38B0BEA450B601040
:108ED00075082C8E828F83A3A3A3A3A3E0D2E0F016
:108EE0008E828F83A3A3A3A3A3E054036401600332
:108EF000028FAD430811028FADEE241812B97C60C9
:108F000049EE241A12B97C6003F4701D12E223703A
:108F100003A3E0697006750822028FAD901A7AE00B
:108F200064046003028FAD801CEE241BF582E43FD5
:108F300012B9C5241A12B97CFAEE2419129BDC125C
:108F40003FA5E97068750901806312CC8F1244D97E
:108F5000E96402700375080112E2237003A3E0695B
:108F60007006E508D2E1F508E50860158E828F836A
:108F7000A3A3E07006E508D2E58004E508D2E6F593
:108F80000812CC8F1244D9E964017006E508D2E0DA
:108F9000F5088E828F83A3A3E0601212B4FBF9124E
:108FA00044B5E964016006E508C2E0F5089019E8F7
:108FB000E0600464017012E508A2E1400CE509A23A
:108FC000E04006E508D2E7F50802891C7418122B68
:108FD0008D7F0402281974EC12259374C3122C0B94
:108FE000EAFEEBFF85188285198374FEF0A304F076
:108FF0007510007511007509009019E8E0640270A1
:10900000248E828F83A3A3A3A3E06019901CA912CE
:10901000CF9B6011901CA9E0F50AA3E0AA0AFBE42B
:10902000FCFD1242F97405122BEB8E828F83A3A3F1
:10903000A312CF8E12CC9A12441FE970030294122D
:1090400078017407122E61E0C39402400278007424
:1090500009122E61E0C3940240027800740E122EB1
:1090600061E064F87003A3E0F47003029412740EDC
:10907000122E61E064F97003A3E0F470030294120D
:10908000740E122E61E064FA7003A3E0F470030220
:109090009412740E122E61E064FB7003A3E0F4706E
:1090A000030294127408122E61E0F9901A68E069C4
:1090B0006003029412E8A2E040030294129019E8BF
:1090C000E06402700B7429122E61E06003029412B6
:1090D00012BADC7424122E6112B9E6241C12BADF13
:1090E0007412122E6112CCAB740B122E61E0601D53
:1090F000741C122E61E0FD7406122E61E0FC8E825B
:109100008F8312CC9A79011242B7E9703D7405122F
:109110002BE312430BE9F508740B122E61E0702F5C
:10912000901A62E06029742255086422602174421A
:109130005508644270147422122E61129AF8600F5E
:109140007422122E61129AFE60057ACF029414E9FD
:10915000A2E6506C9019E8E060046401701B901A5C
:1091600065E0A2E150137422122E6112B504122A96
:109170002A01010B97910012947422122E6112B5EC
:109180000424FD601214600F24FD600B24FD6007B1
:1091900024FE60030294127422122E61129B377017
:1091A0000F7422122E61A312C8BDA3E0640D6010DB
:1091B0007405122BE3124515E964017003029AE16C
:1091C000EE242DF582E43FF58312A3137003A3E090
:1091D000697021750A00780A122B7E780A122B7E9C
:1091E000EE242F129BDC129B0412CC9C124455746B
:1091F00002122B8D740B122E61E070030292A312E7
:109200009B0412CC9C1245DB8A0A8B0BEA450B703F
:109210000302933A7406122E61E0F88E828F83A3C4
:10922000A3E028F8A3E03400F9E8240D129AE6F848
:109230008A828B83A3A3A3E068600EE88A828B8373
:10924000A3A3A312B1A7129B4C79047406122E613A
:1092500012A663E02AF8A3E034008882F583A3AA6B
:1092600082AB8312336F8A0C8B0D8C0E8D0F850AA7
:1092700082850B83A3A3A3A3780C122AFD400302CB
:109280009AE190819A780C122D4D850A82850B8384
:10929000A3A3A3A3E50CF0A3E50DF0A3E50EF0A3B3
:1092A000E50FF09019E8E0640260030293E7901A7A
:1092B0007AE064046008E064096003029AE1E5086A
:1092C000A2E54003029375EE242F12B97CC0E0742E
:1092D00002122E61D0E0129B5DC0E07403122E6179
:1092E000D0E0129B55C0E07404122E61D0E0F074FF
:1092F00016122E61E0640170267410122E61129B0A
:10930000147003A3E0697017740E122E6112CC9CC6
:109310001244D9E9640270077416122E61E4F01247
:109320009B4212299D7406122BEB7409122BE31237
:109330003E7F7404122B8D029AE1901ABFE0640103
:1093400060030292A37422122E61129AF87009E54A
:1093500008A2E650030292A37412122E61E0F47088
:1093600003A3E0F4600CEEFCEFFD7405122BE31296
:109370004317029AE1A2E64003029AE17422122EF8
:109380006112D19B7016741C122E61E0640270543D
:109390007405122BE379001244A980487422122E1E
:1093A00061129AFE7014741C122E61E06404703411
:1093B0007405122BE312449D802A7422122E61122E
:1093C0009B37700C79007405122BE3124521801431
:1093D0007422122E6112B506640C70087405122BEB
:1093E000E3124551029AE1E0600764016003029ACA
:1093F000E1901A65E0A2E14003029AE17429122E7D
:1094000061E060267410122E6112CC9C123D71E94D
:10941000700A7AD37B00123873029AE18E828F83AE
:10942000A3A312E301A3E0C2E5F07416122E61E0DB
:10943000601DEE2402F8E43FF9E8FAE9FB12D1A13D
:1094400014F012D1A1F87416122E61E8F07006E53E
:1094500008C2E7F508E508A2E35061751110A2E221
:109460005018740A122E61E054E3F0740A122E614F
:10947000E0131313541FF8E0802CA2E4502A740A5E
:10948000122E61E01313543F5407F8600974076803
:10949000600B18E87007C3E508C2E7F508E8333346
:1094A00054FCF8E054E348F0740A122E61E0C0E086
:1094B0008E828F83A3A312B0EED0E0F0901A7AE0F0
:1094C00064046008E064096003029598740E122E2B
:1094D0006112E2307003A3E069601F740E122E6106
:1094E00012CC9C1244D9E96402600F740A122E61F6
:1094F000E0540364016003029AE17407122E61E0F4
:109500007041EE242F12B97CC0E07402122E61D09B
:10951000E0129B5DC0E07403122E61D0E0129B55F7
:10952000C0E07404122E61D0E0129B3D12299D749C
:1095300006122BEB7409122BE3123E7F7404122BDC
:109540008D80527422122E6112D19B7016741C12DF
:109550002E61E06402703E7405122BE37900124420
:10956000A980327422122E61129AFE7014741C1299
:109570002E61E06404701E7405122BE312449D807A
:10958000147422122E61129B37700A79007405122E
:109590002BE3124521029AE174615508700302968B
:1095A0009FE508A2E0506D12B9AE7405122BE312CC
:1095B0003FD5E9705C12444FE9F5097416122E612B
:1095C000E0700F7410122E61129B147003A3E069F7
:1095D0006042A90912B9AE7405122BE3123FDBE910
:1095E0006024E508A2E3500C85188285198374FF76
:1095F000F0A3800C740E122E61129B1FE8F0A3E9F9
:10960000F0751004800EE508C2E5F50875090080C4
:109610000353089FE508A2E5503FEE242F12B97CC2
:10962000C0E07402122E61D0E0129B5DC0E07403B2
:10963000122E61D0E0129B55C0E07404122E61D04E
:10964000E0129B3D12299D7406122BEB7409122B1C
:10965000E3123E7F7404122B8DE508A2E64003025C
:109660009974A818A919880A890B780A122B7AA963
:1096700009129AEF122BE31242FF7402122B8DE9AA
:10968000F50970030299747422122E6112B50464F4
:1096900001600302997474104510F51002997474F6
:1096A00007122E61E06401705D7422122E6112B502
:1096B000046405701EA818A9198808890978081279
:1096C0002B7A129AED122BE31242FF7402122B8DA9
:1096D000029AE17422122E61129B377029740E12C5
:1096E0002E6112CC9C123D71E9601BA818A9198843
:1096F0000A890B780A122B7A129AED122BE3124286
:10970000FF7402122B8D7416122E61E070257407FF
:10971000122E61E06401700C7422122E61E0F812C6
:109720009B37600CEEFCEFFD7405122BE312431720
:10973000029AE1124395E96003029AE1741D122E28
:1097400061E070030297ED7420122E6112B9B774B4
:109750001F122E61E0FA741E122E61E0F9123FA56D
:10976000E9607D741F122E61E0701E740E122E616E
:10977000129B1F12F4C1FAA3E0FB123D7D8B0BEA92
:10978000450B600302996E80517420122E6112CC39
:109790009C741F122E61E0F9123F9F851882851973
:1097A0008312E16D7808740D122E61E0600278106A
:1097B000740C122E61E06004740828F8740A122EEA
:1097C00061E0600108088E828F83A3A3E028FAA3DA
:1097D000E034008A82F583E014F075104002996E3F
:1097E0007508007808122B7E790B029927740E12E7
:1097F0002E6112CCA07409122E61E060030299421E
:10980000E508A2E350030299427407122E61E06456
:1098100001607A790085188285198312CC9C123FE9
:10982000F98A0A8B0BA80AA90BE849601C8882896F
:1098300083A3A3A3A3A3E06401605288828983A3C6
:10984000A3A3A3A3E064026044EE242D12B9B18562
:10985000188285198312CC9C1245DB8A828B83E5A2
:10986000824583600FA3A3E0F91245F9E96005C3BF
:10987000940840197410122E6112CC9C123D71E9AB
:10988000700302991D7409122E617404F07800E8C7
:10989000F5097809122B7E741E122E61AC82AD83FD
:1098A000740F122E6112CC9C740A122E61E0F91210
:1098B000400B7401122B8DE9600F7510208E828F82
:1098C00083A3A312B504543FF0741D122E61E0600F
:1098D00023740E122E6112B9B7741E122E61AA8261
:1098E000AB8312441985188285198312E16D744087
:1098F0004510F5107407122E61E0640160157900BF
:109900007410122E6112B9B7740E122E6112CC9C13
:10991000123FABE508A2E350377940803575080067
:109920007808122B7E7902740F122E6112B9B77467
:1099300011122E6112CC9C12451B7401122B8D0248
:109940009AE1E508A2E3400302988D784002988FDF
:1099500079007410122E6112B9B7740E122E6112B2
:10996000CC9C123F39E9600674204510F510124472
:109970004FE9F509851882851983E064FE7003A319
:10998000E0F470037509009019D5E06401600302EA
:109990009A27EE241312B97CF47003A3E0F4700349
:1099A000029A27740E122E61C3E094F9A3E094FF8B
:1099B000507512BADC7410122E61E0687003A3E0D7
:1099C0006960647410122E6112CC9C123D7D8A0A6B
:1099D0008B0BA80AA90BE849604D88828983A3A351
:1099E000A3A3E06401600D88828983A3A3A3A3E0FD
:1099F000640270337430122E61740112E6B7F8A35A
:109A0000E0F9743B122E6112CCAB7430122BE312CE
:109A10003D29E960127433122E61AA82AB83123D94
:109A20008FE960031237FBE508A2E74003029AE1E1
:109A3000E5097003029AE18E828F83A3A3A3A3E0BA
:109A4000FA7B0012341D8A0A8B0BEA450B70030265
:109A50009AE1EE2404F512E43FF5138E828F83A37E
:109A6000129B29122B76851282851383E0FC7D00E0
:109A70001233577403122B8D7407122E61E0C0E06D
:109A8000742B122E61D0E0F0742E122E61E4F0A33C
:109A9000F0742B122BDB880C890D780C122B7A7545
:109AA00008007808122B7E7810122B7AE509F50849
:109AB0007808122B7E12B9701229A585128285139F
:109AC00083E0F97408122E6112B9B7AA0AAB0B121F
:109AD000440D7408122B8DE96007AA0AAB0B1234EF
:109AE00023743D028736F582E412EEF522790012E6
:109AF000B97412B9BB74072212B51E64062212B5DE
:109B000020640722EE242BF582E43FF58312B9CBC3
:109B100012B9752212D54EEE241312BF61682212BB
:109B2000D54E85188285198322A3E0F50CA3E0F5B4
:109B30000D750E00780C2212B520640322F0129BE2
:109B40004222EE2425F582E43FF58322E4F0A3F0DF
:109B5000A3F0A3F022F0EE243112BF6122F0EE2434
:109B60003012BF612274F4122593EAFEEBFF8C08D9
:109B70008D099019D2E0600F12E2237003A3E0690F
:109B80007005123F278052790012CC8F123FF98A5C
:109B9000828B83E58245836035A3A3A3A3A3A3E0BF
:109BA0005418602AE508241C12CC881229A5E5085F
:109BB000241312CC881229A5EE2418129BDC129BC8
:109BC000E112CC9C1240117404122B8D800B790091
:109BD000129BE112CC9C123F51028FD112BF61F94E
:109BE000228E828F83A3A3A3A3A3A3A3A3A312B9AB
:109BF000CB12CC7B2274F012259374EA122C0B8AC0
:109C00000A8B0BEA2402F50EE4350BF50F0A0AFB6A
:109C1000123D838A088B09AE08AF09750801850AD1
:109C200082850B83A3E0F509750C01AC0EAD0F74B2
:109C30000B122E61AA82AB831235317413122E617E
:109C400074FEF0A304F07415122E617402F074080F
:109C5000122E61E4F0901CE3E0700EEE4F700AE506
:109C60000970067508C3029E31901A7AE064086094
:109C7000067508C2029E2D850A82850B83A3A3A3C5
:109C8000A3A3A3A3A3A3A3E0A2E1500EA2E35005C4
:109C9000750C04800C750C038007A2E35003750C4F
:109CA00002EE4F7003029D408E828F83A3A3A3A375
:109CB000E06404600D8E828F83A3A3A3A3E06403FA
:109CC000700C7404650C602C7403650C60268E8225
:109CD0008F83A3A3A3A3E06402600D8E828F83A36E
:109CE000A3A3A3E0640170317402650C60067401E3
:109CF000650C70188E828F8312CC9C1244F7E97029
:109D00003F12A9A6122E6112CCAB80348E828F83B3
:109D1000A3A3A3A3E06402600D8E828F83A3A3A3F9
:109D2000A3E06401700A8E828F8312CC9C123F6F75
:109D3000E50A2402FAE4350BFB123D8F7E007F001A
:109D40007413122E61E064FE7003A3E0F4704612F7
:109D50003D35E97040E509601B901CEC12CC9C126B
:109D600044F7E9700F901CEC12A9AA122E61E8F0DA
:109D7000A3E98020850A82850B83A3A3A3A3A3A3C1
:109D8000A3A3A3A3E05402F9123F637413122E613C
:109D9000EAF0A3EBF07413122E61E064FE7003A3EB
:109DA000E0F470067508C7029E2DE509F50D780DE3
:109DB000122B7E850A82850B83A3A3A3A3A3A3A34F
:109DC000A3A3A3E0F9E50A2402FCE4350BFD741417
:109DD000122E6112CC9C123EA37401122B8DE970DD
:109DE0004CA90CE50A2402FCE4350BFD7413122E79
:109DF0006112CC9C123D5F8A0E8B0FAE0EAF0FEE40
:109E00004F601F74026509700D8E828F83A3A3A318
:109E1000A3A3E0D2E3F07415122E61E4F0750800FC
:109E2000800B7413122E6174FEF0A304F0E5097028
:109E300009AA18AB19123C33800AFCA90CAA18AB6A
:109E400019124497E9FCEE4F6053E50960208E82B9
:109E50008F83A3A3A3A3A3E0D2E6F07402650970E5
:109E60000D8E828F83A3A3A3A3A3E0D2E5F0850A7E
:109E700082850B83A3A3A3A3A3A3A3A3A3A3E0A26D
:109E8000E6500D8E828F83A3A3A3A3A3E0D2E7F0B5
:109E90008E828F83A3A3A3A3A3A3E004F0E508709D
:109EA0003BEC60337D007A017B10123333EE4F6060
:109EB0000CE50A2402FAE4350BFB123D8F741312F1
:109EC0002E61E064FE7003A3E0F4600B7413122EA5
:109ED0006112CC9C123F6F741602D93CFC80C57491
:109EE000F712259374F7122C0BEAFEEBFF901A7A07
:109EF000E06403600DE064016008E064096003024F
:109F0000A02E8E828F83A3E06003029FEC7C007DF5
:109F1000007A027B0012333312A0338A828B8312C1
:109F2000BAE5901A6B12CCAB7953123C27901A7A8F
:109F3000E064096009901A7812CC9C1245D5851806
:109F400082851983740112CFD27942123C27901A6C
:109F50007A7404F07401122BE3794A123C217401E3
:109F6000122BEB7A707B1A12353190187CE0640B5F
:109F700070057406F0800B7900901A7812CC9C1250
:109F80003E9D9019E8E060046401701F901A6EE035
:109F900064FE7003A3E0F4602A79007401122BEBD5
:109FA000901A6E12CC9C123D5F8018E06402701310
:109FB000901A6B12B9B77A037B0012333312A8924E
:109FC000123333901A65E0A2E35004D2F08002C24B
:109FD000F012CFC87952123C279019E8E064027061
:109FE0004A901CA5122E321242F9803FFC7D007A65
:109FF000037B101233339019E8E06402701B901851
:10A000007CE0640B7003740AF09019D6E4F0FA7BDC
:10A0100040901AC5E0F91234EF8E828F8312A03D72
:10A0200012CC9C123E9D901A7AE4F012436574099A
:10A0300002B3FDEE2402FAE43FFB22E0F8A3E0F9CC
:10A04000901A7822C082C083901A0112CF9B701F91
:10A05000901A7AE014600924FC600A14600C800FE6
:10A06000901A0C8034901A08802F901A0A802AE8DF
:10A07000496008901A0212A674700C8A828B83A31E
:10A08000E0F9123E85801D901A0112D1A56402707C
:10A090000512456F800E901AF812CF9B600612C809
:10A0A000BD12277902C58874F412259374FE122C10
:10A0B0000B8A088B097A007B04901AC5E0F91234E8
:10A0C000EFAA18AB197950123C217A0F7B0012339A
:10A0D0007B8A0A8B0BAE0AAF0BEE4F60208508829D
:10A0E000850983A3E07016901A78E0F47003A3E06A
:10A0F000F4603B12A30D7003A3E069603185088210
:10A10000850983A374EA12A7F8123C277A6E7B1A9A
:10A11000794B123C277A787B1A7950123C277A6D5A
:10A120007B1A79E1123C27EE4F700302A1B78E82B1
:10A130008F837402F0901A78E0F47003A3E0F46067
:10A140000A12A30D7003A3E069704F851882851968
:10A150008312A03BE8F0A3E912A7F8123C21901A61
:10A160006B12B02112CCAB7A6E7B1A794B123C2168
:10A170007A6D7B1A79E1123C21750A00780A122B5C
:10A180007E780A122B7E901C5912A03E12AD5712F7
:10A19000CC9C1244557402122B8D8508828509834C
:10A1A00012A1BCA3F0901A7A7403F0EEFAEFFB90C0
:10A1B0001AC5E0F91233877402028FCEA3E08E82B3
:10A1C0008F832274F412259374E8122C0BEAFCEBB3
:10A1D000FD8C828D83A3A3A3A37808122DD47808C5
:10A1E000122D94901A7B7808122D277F7F7E7F791D
:10A1F00000901A7B7808122DD4E97808122BC2E55A
:10A2000008A2E050297800901AC68014850882853B
:10A210000983A3A3E069700108E508241412CC881F
:10A2200012AA4170E7E8C39F5004E8FFE9FE09E97C
:10A23000C3941B40BC8C828D83A3A3A3A3122E0EB8
:10A24000E8494A4B6079EC2404F508E43DF50985BA
:10A250000882F583122E0E901A7B122E4A7C187DEE
:10A26000007900AA18AB1912336385088285098327
:10A27000122E0E851882851983122E4A7404122E0E
:10A28000617401F0901A81E0C0E07405122E61D073
:10A29000E0F07407122E61E412CFD2123C3F806AC4
:10A2A000901A7812CC9C123ED38A0A8B0BA80AA96A
:10A2B0000B901A7812A31C687003A3E069602D90BC
:10A2C0001AC612AA41602585088285098312A31344
:10A2D0007003A3E069700C850882850983A3A3E05D
:10A2E0006E60BDE508241412CC8880D6EE901A6DFD
:10A2F000F0124347E96013901A7AE4F0901A0E12B4
:10A30000CF9B600612C8BB122779028FCC851882BA
:10A3100085198312D54E901A78E06822E8F0A3E9F7
:10A3200012A32422F0850882850983E02274F412A6
:10A33000259374E8122C0B8A828B83A3A3A3A3A377
:10A34000A3A3A3A312DA4C7C00901A7B7808122DE9
:10A35000D4EC7808122BC2E508A2E0502FECF8EA02
:10A360002812BAD4F8901CEBE0C398501F7508016E
:10A37000750900750A00750B00EC7808122ADE7862
:10A3800008122D94901A7B7808122D270CECC39498
:10A390001B40B6901A7B122E0EE8494A4B604E7C49
:10A3A000187D007900AA18AB19123363901A7B123A
:10A3B0002E0E851882851983122E4A7404122E617E
:10A3C0007401F07407122E617401F0901A81E0C0DC
:10A3D000E07405122E61D0E0F07407122E61E412D1
:10A3E000CFD2123C3F901A7A7406F0801C901A7AF1
:10A3F000E4F0FCFD7A047B10123333901A0E12CF76
:10A400009B600612C8BB122779028FCC74F5122507
:10A410009374D1122C0B8A088B098A828B8312BC0D
:10A4200070741C122BEB8A828B83A3A3A3A3A3A318
:10A43000A312A66C12CC93124377741C122E61E007
:10A44000702C850882850983A3A3A3A3A3A3A3A338
:10A45000E0C3940B40188E828F83A3A3A3A3A3A36E
:10A46000A3A3E06402700712CC76E0F4600302A6B6
:10A470005E901A7AE06402700302A543E0640670FD
:10A480000302A543901A0112CF9B600812A67470B4
:10A490000302A577901A7AE064086008E06404601B
:10A4A0000302A65E741E122E6112A663A3A3A3A3C9
:10A4B00012BC70901A01E0F849600712D1AB640237
:10A4C0006077901A78E06E7003A3E06F600302A6D5
:10A4D0005E74016A60167423122E61AC82AD837AB9
:10A4E0008C7B1A12352BE9600302A65E7A007B0290
:10A4F000901AC5E0F91234F5EA4B4C4D600302A600
:10A500005E901A7B122E0E851882851983122E4AB0
:10A51000901A81E0C0E07404122E61D0E0F074055E
:10A52000122E617401F07406122E61740212CFD2E1
:10A53000123E0DE9600302A65BEEFAEFFB124569DD
:10A5400002A65E901A0112CF9B702C750800780845
:10A55000122B7E7808122B7EEE2410F582E43FF554
:10A560008312CF8FA3A3A3A3A312B9D412CC9C129E
:10A5700044557402122B8D8E828F8312BAE57407B4
:10A58000122E61E8F0A3E912A9B012BAE57409121B
:10A590002E6112B9E612BF6BC0E0740B122E61D0AF
:10A5A000E0F012CC76128744740F7808122DE37411
:10A5B0000C122E61E508F07420122E61E0C0E074E8
:10A5C0000D122E61D0E0F07422122E61E0C0E07412
:10A5D0000E122E61D0E0F0741D122E61E0C0E07406
:10A5E00010122E61D0E0F0741E122E61E0C0E074F3
:10A5F0000F122E61D0E0F0EE241012B97CC0E0748E
:10A6000011122E61D0E0F07421122E61E0C0E074CE
:10A6100012122E61D0E0F0742E122E61E0C0E074B0
:10A6200013122E61D0E0F07423122E61A982AA8346
:10A6300089088A09750A007808122B767C087D0043
:10A640007417122E61AA82AB831233577403122B34
:10A650008D7407122BE3123E978003123E13742F62
:10A6600002B66DE0FA8E828F83A3A322A3E0F98A5B
:10A67000828B832212D1AC64012274F71225937469
:10A68000C9122C0B124587901A7AE06408601F905B
:10A690005156E493901A5CF0905156E493901A5AF4
:10A6A000F0901A83740112A7EFA30412A7EF7C2382
:10A6B0007D0079007414122BE3123363901A8BE03F
:10A6C0007009741E122E6174018006741E122E61B0
:10A6D000E412A800740FF0901CEA12CFD27946124F
:10A6E0003C277401122E61E4F0901CBEE0C0E074BF
:10A6F00002122E61D0E0F0901A68E0C0E0740312FC
:10A700002E61D0E0F07404122E61E4F07405122E74
:10A7100061E4F07407122E61E4F0901A8BE0C394A8
:10A720000F500CE0C0E07406122E61D0E080077478
:10A7300006122E61740FF07C8C7D1A7408122E6143
:10A74000AA82AB831235317C037D0079FF7410122D
:10A750002E61AA82AB83123363901AC4E0C0E07406
:10A7600013122E61D0E012CBDC7401122BE31243E2
:10A77000717AC87B1A7945123C27124485901A7F5A
:10A78000E0C0E0741C122E61D0E0F0901A80E0C0AE
:10A79000E0741D122E61D0E0F0901A6DE0C0E074FC
:10A7A0001A122E61D0E012879A7418122E6112CC00
:10A7B000AB7420122E61E4F0901A82E0C0E0741FA6
:10A7C000122E61D0E0F07434122E61E4F07429127C
:10A7D0002E61E412A7F8123C277A6E7B1A794B128D
:10A7E0003C277414122BE3123C45743702B3FDF07E
:10A7F000A3E4F0A3F0A3F022F07A6B7B1A79532242
:10A8000012A80422F085188285198322C082C08391
:10A810008A828B83A3E0901A7A6004E4F0807074DB
:10A8200008F0901A8BE07028901A0E12CF9B6008E7
:10A83000790012C8BD122779901A7812B9B77A0533
:10A840007B00123333901A7812CC9C1245D58018B5
:10A850007900123E91901A6B12B9B77A067B0012FA
:10A86000333312A892123333901AFE12CF9B601F1B
:10A870009019DCE06401701790810612299D7A001E
:10A880007B40901AC5E0F91234E97404122B8D0252
:10A89000C588901A6E12B9BB7A047B002274F41238
:10A8A000259374EA122C0B8A088B09EA2402FAE435
:10A8B0003509FB123D838A0A8B0BAE0AAF0BEE4FB4
:10A8C000700302A9A18E828F83A3A3A3A3E06401D6
:10A8D000602A8E828F83A3A3A3A3E06402601D8EEF
:10A8E000828F83A3A3A3A3E0640360108E828F836F
:10A8F000A3A3A3A3E06404600302A9A1E5082402C2
:10A90000FCE43509FD740B122E61AA82AB8312356B
:10A910003112A9A6122E6112CCAB7415122E6174DD
:10A9200001F07408122E61E412CFD2123C39E9FC16
:10A930007D007A077B001233338E828F83A3A3A31B
:10A94000A3A3E0C2E012A9B0740112E97F5001098B
:10A950007A027B00122337E88E828F83A3A3A3A3FE
:10A96000A3A3A3A3F09019DCE0640170349019D67E
:10A97000E06402702C8E828F83A3A3A3A3E0640102
:10A98000600D8E828F83A3A3A3A3E06402701212D2
:10A99000B970122E0E12C25F122E4AEE241B12CF75
:10A9A000827416028FCE8E828F8312D54E7413223C
:10A9B00012A9B42212C295A3A3A3A32274F2122552
:10A9C0009374F8122C0BEAFEEBFF8C0A8D0B890DA9
:10A9D0009080C8AC18AD197408122A9E750C00EE50
:10A9E000FCEFFDAA18AB1912352BE97003750C01A9
:10A9F000901AC6801AEEFCEFFDE508240BFAE43548
:10AA000009FB12352BE97023E508241412CC8812B7
:10AA1000AA416024E50CA2E040DB85088285098319
:10AA2000E0650A7004A3E0650B70DD850882850986
:10AA300083A3A3E0650D70D0AA08AB097408028B4C
:10AA400040128748E508450922C082C083901AC693
:10AA500002C58574F7122593901AC612F105800C71
:10AA600012D7B412BC73123423EEFAEFFBEA4B7028
:10AA7000EF901AC6E4F0A3F002B40074F412259328
:10AA8000EAFEEBFFEE241312B97C6403700CEE2493
:10AA90000BFAE43FFB123D83800EE06402707C12EF
:10AAA000CC7612CC9C123D7D8A088B09E5084509BD
:10AAB00060698E828F83A3E0700F85088285098389
:10AAC000A3A3A3A3A3A3E4805164F1600A8E828FA1
:10AAD00083A3E064E17027850882850983A3A3A38B
:10AAE000A3A3A3E06401701685088285098312CCB4
:10AAF0009C123F6FEE240BFAE43FFB123D8F85085A
:10AB000082850983A3A3A3A3A3A3E0600E85088283
:10AB1000850983A3A3A3A3A3A314F0028FD174F187
:10AB20001225938A088B09ECFEEDFF890A8A828B35
:10AB30008312DBEF8A828B8312A1BC12ABF08A8274
:10AB40008B83A3A3E0C454F0FA88828983E04A127D
:10AB5000AC0012A1BC12ABFAE0333354FCF88E8285
:10AB60008F83E04812ABFAA3E033333354F8F88E06
:10AB7000828F83E04812ABF08508828B83A3A3A366
:10AB8000A3A3A3E0A2E0E4331313FA88828983E04D
:10AB90004AF0E5082407F50CE43509F50D750E00BB
:10ABA000780C122B767C087D00EEFAEFFB123357FF
:10ABB0007403122B8DEE2408FE50010FE508240FBC
:10ABC000F50CE43509F50D780C122B767C037D002D
:10ABD000EEFAEFFB1233577403122B8DE50AC39480
:10ABE0000F400A12CC8412A1BDA3A3A3F002E95125
:10ABF000F0EEF8EFF9A30EAF832212AC00A3A3226C
:10AC0000F08508828B83A3A32274F1122593EAFEB8
:10AC1000EBFF890A8C088D098E828F83E08C828DF0
:10AC20008312BF9CAE82AF83E012C34B12C535C402
:10AC300012C34B12ACC8E012C35212C533A2E2E4F5
:10AC4000338C828D8312C532131313541F12C34BDE
:10AC500012C531A2E7E4338C828D83A3A3A3A31290
:10AC6000ACC88E0C8F0D750E00780C122B767C08FC
:10AC70007D00E5082407FAE43509FB123357740315
:10AC8000122B8DEE2408FE50010F8E0C8F0D780CC8
:10AC9000122B767C037D00E508240FFAE43509FBCE
:10ACA0001233577403122B8DE50AC3940F40118E93
:10ACB000828F83A3A3A3E0C0E012CC84D0E0800401
:10ACC00012CC84E4F002E951A3A312BFA00EAF831B
:10ACD0002274F51225938A088B098A828B83A3AE8E
:10ACE00082AF83E0F9123EBB8E828F83E064EB601B
:10ACF00024850882850983A3E064E16018850882C1
:10AD0000850983A3E064F1600C850882850983A32B
:10AD1000E0641A7009850882850983A3E4F0901C19
:10AD2000A5122E321242F9750A01780A122B7E857D
:10AD30000882850983A3E0F5087808122B7E790044
:10AD4000901A7812AD5712CC9C1244557402122BF3
:10AD50008D12438F02B67012B9BB901A6E22C08258
:10AD6000C083E9901AD87003E480027401801EE069
:10AD7000F902C588C082C0837CE77D428A828B83CA
:10AD800012CC9C123C5102C588EAF0A3EBF002C53C
:10AD90008874F6122593901AD8E0701B7C00790114
:10ADA0007A007B001243BFEA4B600C8A828B8312CD
:10ADB000CF9B60031242ED02C91AC082C08379049E
:10ADC0001243B9E9F8905154E493C398401079FFC5
:10ADD0001243B9E9F8905153E493C39850047901B0
:10ADE0008002790002C58874F01225938A088B09C5
:10ADF000890B750C008A828B83A3A3A3A3A3A3A3AF
:10AE0000A3E0F91243C58A0E8B0FAE0EAF0F750A81
:10AE100001EE4F600302AED285088285098312B02D
:10AE200010A3A3A3A3A3A312C05912CC9C1243AD99
:10AE30008A0C8B0DAE0CAF0DEE4F700302AFFB8E84
:10AE4000828F83A3A3A3A3E4F0A3F0E508240CFA64
:10AE5000E43509FB8A828B83E0C0E012E975D0E01B
:10AE6000F0E508240D12B00812DBBD12CCAB124481
:10AE7000E5EE240F12E167E508241112B0081289EB
:10AE80002212CCABE508241312B003C0E012B97053
:10AE9000D0E0F0750C01EE240612BF51E0547FF0B3
:10AEA000A3E054FC12E6ADE05404600302AF499005
:10AEB0001CB7E0F50875090074077808122D148E88
:10AEC000828F83A3A3A3A3A3A3E04508F0A3E04537
:10AED00009F08E828F83A3A3A3A3128742740778FD
:10AEE00008122DE3E5085407FCE50B606C8E828F99
:10AEF00083A3A3A3A3A3A3A3A3A3740212C536127F
:10AF0000B2D7600B901A6612B021A3A312CCABEC9F
:10AF1000700302AFC4EE240612F453547FF508A365
:10AF2000E054FCF509EC24FFF50EE434FFF50F7452
:10AF300007780E122D14E508450EF8E509450FF9BE
:10AF40008A828B8312CCAB807B8E828F83A3A3A358
:10AF5000A3A3A3E0448002AED1EC7005750A008083
:10AF6000638E828F83A3A3A3A3A3A3E05420600CCA
:10AF7000123375EA547F7900245F80198E828F83A3
:10AF8000A3A3A3A3A3A3E05410601A123375EA5439
:10AF90000F7900240A5001098E828F83A3A3A3A3F3
:10AFA000F0A3E9800D8E828F83A3A3A3A37401F085
:10AFB000A3E412A9B07404F07A207B00901AC5E0D3
:10AFC000F91233BDE50CA2E0503412B9D0A3A3A30B
:10AFD000A3A3A3A3A3A3E0F9EEFAEFFB1243B3E903
:10AFE000601C12ED5B3F12CF99600912B52E12CC96
:10AFF0009C123423EEFAEFFB123423750A00A90ADF
:10B0000002D93F12BF79E02212BF7912D54EEE224B
:10B01000A3A3A3A3A3A312B9BB850882850983A315
:10B020002212D54E8E828F83A3A32274F41225930D
:10B0300074F7122C0B7E001243C5EA4B700302B06A
:10B04000E78A828B83A3A3A3A3A3A3A3A3A3E06400
:10B0500006600302B0E78A828B83A3A3A3A3A3A302
:10B06000A3E0FF8A828B8312B0EEE0C0E074081286
:10B070002E61D0E012B51512CCA11243E3EF5408B3
:10B08000606385188285198312B9B77A007B001234
:10B0900043A78B0BEA450B704C12F5AD123C697C53
:10B0A000007D007A007B0080288E828F8312B50499
:10B0B000F47003A3E0F4602D901A7812B9D812CC82
:10B0C0009C123C63E9641A601C7C007D00EEFAEF80
:10B0D000FB1243A78A0A8B0BAE0AAF0BEE4F70C967
:10B0E0007900123C6F7E01EEF97409028FCE12BC1A
:10B0F0007C12B0F5222408F582E438F58322C08260
:10B10000C083EA4B7005901ADD80068A828B83A388
:10B11000A312B30B60258A828B83A3A3A3A3A3A34B
:10B12000A3E0540860E5EC4D60158A828B8312B56C
:10B13000046C7003A3E06D70D280047A007B00027F
:10B14000C58874F2122593EAFEEBFF890A8C088DFC
:10B15000097A147B0012341DEA4B603F8A828B838C
:10B16000A3A3A3A3A3A3A3A3A3E412B50AA3E50ADD
:10B1700012B1A7A3A312DD2A8A828B83A3A3A3A360
:10B18000E4F0A312B52812B1B912E105EA12ED5CA0
:10B190003BF583E4F012B19EF0A3F0028B43A3F0E1
:10B1A0008A828B83A3A32212B1AB2212B1AF22F009
:10B1B0008A828B83A3A3A3A322A3F012F4743BF58A
:10B1C00083E4F02274F4122593EAFEEBFF89088CE5
:10B1D0000A8D0BEE4F700302B260740165087012A5
:10B1E00079011243B9E9F8905155E493C39850227C
:10B1F000801674046508701479041243B9E9F89054
:10B200005154E493C398500A79118056740265082A
:10B21000704E8E828F83A3A3A3A3A3A3A3A3A3E5AE
:10B220000812B9E012DBCAE4F0A3F0901ADD12CFE5
:10B230009B60178003E0F8A312CDA2A3A312B30B67
:10B2400088828983A3A370ED8003901ADD12E1093F
:10B250007A207B00901AC5E0F91233BD7900800294
:10B2600079C1028FD1C082C083E9F87900901ADDDC
:10B27000801D8A828B83A3A3A3A3A3A3A3A3A3E07C
:10B2800068600574FF687001098A828B83A3A3122A
:10B29000B30B70DE02C58874F7122593EA4B700574
:10B2A000901ADD80068A828B83A3A312B30B6020E1
:10B2B0008A828B83A3A3A3A3A3A3A3A3A3E0697000
:10B2C000E4EC60108A828B83E012B2D770D78004DE
:10B2D0007A007B0002B40012F4A9E0540422C08278
:10B2E000C083901ADD80068A828B83A3A312B30BDE
:10B2F00060128A828B83A3A3A3A3A3A3A3A3E06961
:10B3000070E580047A007B0002C58812D1D0EA4B38
:10B310002274F7122593EAFCEBFD901ADD80068A71
:10B32000828B83A3A312B30B60248A828B8312B512
:10B33000046C7003A3E06D70E68A828B83A3E0C87F
:10B3400012BC6912D92BA2E0E43370D380047A00D6
:10B350007B0002B40074F21225938A0A8B0B8C0CCA
:10B360008D0D750800750900EA450B6030901ADDF7
:10B3700080068E828F83A3A312BC73EE4F601EAC37
:10B380000CAD0DEEFAEFFB850A82850B831227794F
:10B39000E9640170DDEEF8EFF988088909AA08ABC5
:10B3A00009028B437900022B2274F7122593901A1D
:10B3B000DD12BAE57C007D00800DE8FCE9FD8882A5
:10B3C0008983A3A312BAE5E8496030EA687002EB0A
:10B3D0006970E7901ADD12CC9CE86A7002E96B880C
:10B3E000828983A3A3700812BAE5901ADD8009123E
:10B3F000BAE58C828D83A3A312CCAB8003122B8D74
:10B400007F0102281974F7122593EAFEEBFFEE4F35
:10B41000602F1243DD12B44312CC9C1234238E826F
:10B420008F8312CC9C12342312ED5B3F12CF9960B4
:10B430000912B52E12CC9C123423EEFAEFFB123413
:10B440002380BD12CFA1F5832274F61225938A8240
:10B450008B8312B504F508A3E0F509901ADD12BA42
:10B46000E57D007C00802F88828983A3A3A3A3A30A
:10B47000A3A3A3A3E0640570140C12DBE6F5838E8E
:10B4800082E065087004A3E0650970010D88828977
:10B4900083A3A312BAE5E84970CD905151E493F823
:10B4A000EDC398500890515012EEE3400F8A828B02
:10B4B00083A3A3A3A37401F0A3E48010901A66E011
:10B4C000F812A66CA3A3A3A3E8F0A3E912B528740D
:10B4D0000512B50AE0440812B515F47003A3E0F4B0
:10B4E0006011901A7812D90E12CC9C123C63E96458
:10B4F0001A70057901123C6F02C91AEE241DF582FB
:10B50000E43FF583E0F812B5202212B50E2212B105
:10B51000AFA3A3A322F08A828B8312B51E22E0F888
:10B52000A3E0F5838882E02212B50EA3A322EE12D7
:10B53000CD8722C082C083EAFCEBFDEC4D6017ECA6
:10B5400024FBF582ED34FF12CF99700712B58DE020
:10B55000F4600712338179058030901AC5E0C0E0AD
:10B5600012B58DD0E0F0905147E493F97ADF7B1A61
:10B570001233B7E9640170107A007B20901AC5E09D
:10B58000F91233BD79008002790402C588EC24FFEA
:10B59000F582ED34FFF5832274F4122593A2AFE413
:10B5A00033F508C2AF901ADF12BC73EE4F603AEE6B
:10B5B00024FBF582EF34FF12CF997A007B20901A9A
:10B5C000C56007E0F91233BD8005E0F91233C3E42A
:10B5D000F50AF50B780A122B7AEEFCEFFD7ADF7B89
:10B5E0001A1233B17402122B8DE508A2E092AFEE6D
:10B5F000FAEFFB028FD174F51225938A088B097537
:10B600000A00901ADD12DBEA805A8E828F8312B50F
:10B610000465087004A3E06509703D8E828F83A3E2
:10B62000A3A3A3E4F0A312C2A6540460118E828FD8
:10B6300083A3A3A3A3A3A3A3A3E0F9123FE18E8254
:10B640008F83A3A3A3A3A3A3A3A3A37406F07AF059
:10B6500012892F1242F3050A8E828F83A3A312BA96
:10B66000E5E8FEE9FFEE4F70A1A90A8003122B8DD9
:10B670007F0302281974F012259374D4122C0BEA5C
:10B68000FEEBFF750B00750A007508FE7509FF12C9
:10B690004395E9600302B963EE241512B97C604456
:10B6A000901CD4E0C43354E0F8E0333354FC48C079
:10B6B000E012D73DD0E012B9E012CC9C79FF1240E5
:10B6C000E38B0DEA450D600F750B017508FF12CF76
:10B6D0008612CE5CD2E0F09019E8E060046401705C
:10B6E00003750A408E828F8312CC9A1244D9E96086
:10B6F0000312B988EE241312B97C700D90277BE4F5
:10B7000093C0E012B970D0E0F08E828F83E0A2E7A0
:10B71000500454038019EE241412B97C7012901A4C
:10B7200057E0C0E012F449D0E0F0901A57E004F07E
:10B7300012F4657016901CC0E0600D901A62E07003
:10B740000A8E828F83E0700312CD779019E8E06053
:10B75000046401704B901A65E0A2E15043E50BA22E
:10B76000E040218E828F8312CC9A1244D9E9603056
:10B770008E828F83E0600DEE240B12B4FEF912442A
:10B78000B5E9601C12B994700302B915EE241312C6
:10B79000B97C6401600302B91512B52EE054FBF0C8
:10B7A0008E828F83E06401700DEE240B12B4FE6470
:10B7B00002700312B9A112B994600302B87BE50BC1
:10B7C000A2E0500302B87B9019E8E06007640160D2
:10B7D0000302B87B901A65E0A2E1400302B87BE562
:10B7E0000AF50B780B122B7EEE2406FCE43FFD8E4F
:10B7F000828F8312CC9AEE2412129BDC12400B74BF
:10B8000001122B8DE9600612B98812B99A8E828FC7
:10B8100083A3A3A3A3A3A3E0603CEE2402F50CE45E
:10B820003FF50D850C8212B9C52407FAE43FFB12DF
:10B8300044198A088B09850C82850D83E0650870A0
:10B8400004A3E06509700C8E828F83A3A3A3A3A336
:10B85000A3E4F012B9A18E828F83E06401600BA98A
:10B860000A12B9D412CC9A123FABA90A12B9D0125B
:10B87000CC9A123F39E9600312B99AAC18AD19EEAF
:10B88000FAEFFB1244138A0A8B0B74FE65087004EE
:10B8900074FF6509700312873EEA450B700302B915
:10B8A000678E828F83E0C0E07401122E61D0E0F0D9
:10B8B0007404122E6112E109EE241E12BADF740222
:10B8C000122E6112CCAB7401122BDB880C890D781F
:10B8D0000C122B7AEE242012B980122B7E12B52E78
:10B8E0001229A5EE240E12B980122B7E901A6B122B
:10B8F00029A57408122E61E0F9AC08AD0912440DB7
:10B900007408122B8DE9FE74106E705DAA0AAB0BE1
:10B910001234238054EE241312B97CC0E074171241
:10B920002E61D0E012F4BA740F122E6112B9E6241F
:10B930000412F45812BAE57411122E61E8F0A3E96A
:10B9400012BFC1C0E07418122E61D0E012E96B1270
:10B95000A66D12B9B77406122BE3123FDBE9600340
:10B9600002B7A0791180047E10EEF9742C02D93C44
:10B9700012B97422EE12CDBF22EE241712BF61223B
:10B9800012BF61F50C780C22EE2412F582E43FF52B
:10B9900083E4F02212B9A854402212B9A84420F03E
:10B9A0002212B9A84440F022EE12CD8BE022EE2400
:10B9B00013F582E43FF58312B9BB2212B9BF22E02E
:10B9C000FCA3E0FD22F58312B9CB2212B9BFEE220F
:10B9D0008E828F83A3A3A3A312B9BB8E828F8322EF
:10B9E00012DBD622A3A3E8F0A3E9F0EE22C082C0C6
:10B9F0008374D7122C0B9080007403122BEB7426E7
:10BA0000122A9E8A828B83A3A3A3A312BAE5740E83
:10BA1000122E61E8F0A3E912D547740C122E6112C0
:10BA2000BAE9240D12BAD4C0E0741A122E61D0E023
:10BA3000F012D7BE12BAE37420122E6112BAE924B2
:10BA40001512BAD4C0E07408122E61D0E0F0EA24D6
:10BA50001CF582E43B12BAE37412122E6112BAE9A9
:10BA6000241112BAD4C0E07409122E61D0E0F0EAB9
:10BA7000241212BAD4C0E07407122E61D0E0F0EAAA
:10BA8000241EF582E43B12BAE37424122E6112BA2A
:10BA9000E9242012BAD4C0E07426122E61D0E0123C
:10BAA000A80074FFF07401122E6174FFF07402128A
:10BAB0002E6174FFF090810A12299D7404122BEB01
:10BAC0007407122BE3123E7F7404122B8D790074DD
:10BAD0002902D58BF582E43BF583E022EE2413F5B1
:10BAE00082E43FF58312D54E22E8F0A3E9F0EA2282
:10BAF00074EE12259374EC122C0B8A0E8B0F8C08AB
:10BB00008D09890C750A107A217B0012341D12D51B
:10BB100091E849700302BC62750B007C217D0079BD
:10BB200000851882851983E0FA1233637429122E76
:10BB30006112BC739019E8E060046401703EAA08C9
:10BB4000AB09123D7D8A108B11A810A911E849603C
:10BB50002388828983A3A3A3A3E06401600D888264
:10BB60008983A3A3A3A3E064037009EE5440700487
:10BB700074044FFFEF54046003750B01901A7812A0
:10BB8000CC9C85188285198312BC782409F582E43F
:10BB90003812E16B7426122E6112BAE57411122E5E
:10BBA00061E8F0A3E912BC8112F46B12BC8112B0FF
:10BBB000F5740212F4C5F8A312C8BD12DE9412BCCB
:10BBC0008112F47BE50CF07428122E61E0F50885F3
:10BBD000188285198312F484E50812BC8112BC69AD
:10BBE000F583E50EF0A3E50FF07406122E6112E165
:10BBF000097408122E61E508F0742C122E6112E30C
:10BC000001C082C083740C122E61AC82AD83D083DC
:10BC1000D0827405122A9E742B122E61E0C0E0744B
:10BC200013122E61D0E0F0A90BAA18AB1912439B96
:10BC3000E9640170219019E8E0600464017012E584
:10BC40000BA2E0500CA9081243C5EA4B6003124353
:10BC5000E9750A00800C85188285198312CC9C1224
:10BC60003423A90A741402C2AC241FF582E43822DA
:10BC7000A3A3A312DBEAFF2212BC7C2212D5ABC81D
:10BC80002212D5A0C82274EE122593EAFEEBFF8C97
:10BC9000088D098E828F83A37408F0EE241612B9E2
:10BCA0007C60088E828F83A37410F012B9796009CA
:10BCB0008E828F83A3E02408F0EE241512B97C60F5
:10BCC000088E828F83A3E004F08E828F83A3A3A3C8
:10BCD000A3A3A3E060198E828F83A3A3A3A3A3A32E
:10BCE000A3E0C3332402F88E828F83A3E028F012EE
:10BCF000BF5A6005750B0E8003750B009019E8E0C4
:10BD00006402701E9019DCE0640170168E828F83CD
:10BD1000E06401600D9019D6E0600712BF4774011E
:10BD2000800412BF47E412BF9CE012BF6928250BB4
:10BD30008C828D83F012BF5A6013901A63E0F9125F
:10BD400042BDE9F8850882850983E029F0850882EB
:10BD5000850983E0C39475400975080075090002E0
:10BD6000BF40E0FA7B0012341D8A088B09EA4509BE
:10BD7000700302BF408E828F83E0FA901A6812BF70
:10BD8000957402780C122D14EA450CFAAB0DEE24D2
:10BD90001212B97C5403F50C750D007406780C1260
:10BDA0002D14EA450CFCEBFDEE241512B97C600461
:10BDB000780180027800EE2416FAE43FFBE8F9ED02
:10BDC00049FD12BF5AF50C7409780C122D14ED457B
:10BDD0000DFD8A828B8312BF95740B780C122D1483
:10BDE000ED450DFDEE241712BF8F740C780C122D4B
:10BDF00014ED450DFD8E828F83A3A3A3A3A3A312ED
:10BE0000BF95740A780C122D14ED450DFDEE242318
:10BE100012BF8F740D780C122D14ECF8ED450DF94E
:10BE2000E8850882850983F0E9A3F0EE240212BFB9
:10BE30005112C06312BFB7F0EE240412BF5112BFFB
:10BE40008112BFB7A3A312CDB512BF81A3A3A3A331
:10BE500012BFC1850882850983A3A3A3A3A3A3A3BB
:10BE6000F0750A088A828B83E06015EE241812B9F7
:10BE7000B1E5082408FAE43509FB123531750A10DA
:10BE800012B9796019EE241A12B9B1A80AE5082886
:10BE9000FAE43509FB1235317408250AF50A8E8259
:10BEA0008F83A3A3A3A3A3A3E06057EE2407F510F9
:10BEB000E43FF511851082F583E0C0E012BF70D039
:10BEC000E012BFA7E0C0E00812BF72D0E012BFA727
:10BED000129B29122B76851082851183E025E0FCC8
:10BEE000E433FDA80AE50828FAE43509FB123357C4
:10BEF0007403122B8D851082851183E0C333250ACC
:10BF0000F50AEE241512B97C6008C0E012BF70D0AB
:10BF1000E0F012CC76129B2A122B7612BF6AFC7DBF
:10BF200000A80B8E828F83A3E0FAE5082AFAE43595
:10BF300009FBEA28FAE43BFB1233577403122B8DFA
:10BF4000AA08AB0902C2AFEE2423F582E43FF583D1
:10BF500022F8E43FF9888289832212BF5E22EE2410
:10BF600011F582E43FF583E022F8EE12DBC1E02216
:10BF7000A80AE5082812BF7922F582E43509F5837D
:10BF80002212BF8522E0850882850983A3A322F5BA
:10BF900082E43FF583E0F50C750D002212BFA0226C
:10BFA000F08E828F83A322F0050A8E828F83A3A353
:10BFB000A3A3A3A3A3A322A3A312E6BD12BF85A399
:10BFC00022F0EE241412BF612274F412259374FD42
:10BFD000122C0B8A088B09ECFEEDFF7401122BDB8F
:10BFE000880A890B780A122B7A7402122BEBEEFA6C
:10BFF000EFFB123F877402122B8DE9705385188274
:10C0000085198312C063F07401122E61E0F812C02A
:10C0100059A3A312F4C1602914850882850983A35A
:10C0200012F4C512DA457401122E61E028F8A3E07B
:10C0300039F9E824FEF582E934FFF58312F1058031
:10C040000C850882850983A3E4F0EEFAEFFB8004F7
:10C050007AFE7BFF7403028FCEA3E0F98508828508
:10C06000098322E08508828509832274EE122593D4
:10C070008A0A8B0B8910ECFEEDFF750F017C267D83
:10C08000007900EEFAEFFB123363E510C394085019
:10C090000302C1F88E828F83E510F0EEFCEFFD8580
:10C0A0000A82850B8312C503124425E96003750FCC
:10C0B0000012C4E58E828F8312C53DEE12C4D93FB3
:10C0C00012C527C0E0128921D0E012C51FC0E0EEE2
:10C0D0002412F582E43FF583D0E012BF9C7408126D
:10C0E000C28DA3A3E06018E50A2408F8E4350BF933
:10C0F00012B97012CCAB8E828F83A3E02408F08E2D
:10C10000828F83A3A3A3A3A3A3A3A3E060178E821C
:10C110008F83A385820885830912C4F812D73D1244
:10C12000A31C2408F0EE241912B98BEE241B12B9BB
:10C130008BA312C28DE0600F12C2748E828F83A314
:10C14000A3A3A3A312C2A0EE241812B97C70030209
:10C15000C1E812C274FAEE2419F582E43FF583EACD
:10C1600012C2A0F8E50A28F582E412F5A7F812DC5D
:10C17000FEE812C2A0E8C39AEE5068241912B97CF6
:10C18000F8905148E493C398500575110C8008EE5F
:10C19000241912B97CF5118E828F83A3E0F8E50A89
:10C1A00028F50CE4350BF50D750E00780C122B7686
:10C1B000AC11EC2CFCE433FD7A277B0C1233577462
:10C1C00003122B8DEE241BF582E43FF5837427F0D8
:10C1D000A3740CF0E511C333F8850882850983E068
:10C1E00028800412CD6EE4F08E828F83A3E0F88E57
:10C1F000828F83E0C398500479008061A3E0FAE560
:10C200000A28F8E4350B12C269E8F0A3E912C53632
:10C21000C39AC0E012C25FD0E012C2A6603DEE2415
:10C2200017F8E43FF9880889098882F583E024F249
:10C23000F0EE241D12BF51E0240EFAA3E03400FBFF
:10C240008882898312E16D901A63E0F91242BDE998
:10C25000F8850882850983E0C398F0A90F8050EE25
:10C260002417F582E43FF58322F9EE241DF582E4DC
:10C270003FF583228E828F83A3858208858309E020
:10C28000F8E50A28F582E4350BF583E02212C29125
:10C290002212C29522F08E828F83A3A3A3A3A3228E
:10C2A00012A32404F02212C291A3E022122B8D7F4C
:10C2B0000A02281974F41225938A088B09EA12C31A
:10C2C00052A3A3F0EA1313543F12C34BA3A3A3F04A
:10C2D000EAC4131312C35212C3657409780A122DEB
:10C2E000E312C359A3A3A3A3A3A3F0EB12C35B124E
:10C2F000C364740A780A122DE3E50A5401C0E0EC25
:10C300002418F582E43DF583D0E012C369740B78FC
:10C310000A122DE312C35912C362740C780A122D4B
:10C32000E312C359A312C362740D780A122DE3E518
:10C330000A5401C0E0EC2424F582E43DF583D0E00A
:10C34000F0740E7808122DE302891C540F8C828D34
:10C35000832254038C828D8322E50A54018C828DC2
:10C360008322A3A3A3A3A3A3A3F08A0A8B0B22C0B7
:10C3700082C08379008A828B83A3A3A3A3A3A3E0B3
:10C38000901A62600EE070238A828B83A3A3E07010
:10C390001A8016E060158A828B8312CC93901A6BF8
:10C3A000E06A7003A3E06B6002790102C58874F251
:10C3B0001225938A0A8B0B890C8C088D098A828B33
:10C3C0008312C50312442512C4E5850882850983BA
:10C3D00012C53DE50812C4D9350912C527C0E0E5EC
:10C3E00008241112CC88D0E012C51FC0E012CC8402
:10C3F000D0E012CFAF740812C511E06017E50A242F
:10C4000008F8E4350BF9E508241312C4DD12CFAFA8
:10C41000E02408F0850882850983A3A3A3A3A3A32E
:10C42000A3A3E06017850882850983A312C4F4E5FD
:10C4300008241512C4DD12C5362408F0850882854B
:10C440000983A3A3A3A3A3E06019850882850983B8
:10C45000A3AE82AF8312C27F85088285098312C58D
:10C460003104F0AA08AB0912442BE9F50D7064857C
:10C470000882850983A3A3A3A3A3A312C063A37007
:10C480001AE0FAE50A2AF8E4350BF9E508241D124A
:10C49000CC8812CCABE50CC39A802C12C4F4E824EF
:10C4A0000EF8500109E508241D12CC8812CCAB907F
:10C4B0001A63E0F91242BDE9F88E828F83E0F9E554
:10C4C0000CC39924F2C398C0E0E508241712CC8865
:10C4D000D0E0F0A90D028B43EA12F4752212BF7965
:10C4E000E8F0A3E922850A82850B83A3A312C55332
:10C4F000E0F9EA22AE82AF83E0F8E50A28F8E435F5
:10C500000BF922E0FAA3E0F8E4C8F9EA28E439FBE1
:10C510002212C5152212CFB7A3A3A3A3A3A322124D
:10C52000C566A3A3A3E022F583E812C55FA3A3E039
:10C5300022A3A3A3A3A3F08E828F83E022A3A3A3AD
:10C54000A3A3A3A3A3A312C55F12C553A3A3E0F99A
:10C55000EAF822E0FA850A82850B83A3A3A322F0DE
:10C56000A3E912C56622F0850A82850B83A3A3A3E3
:10C57000A322C082C0837AED7B1A79E2123C217A31
:10C58000ED7B1A800312CC9CD083D082022B22C078
:10C5900082C083901A6B80EDC082C083901A6E8037
:10C5A000E4C082C083794A123C2180DC74F61225F3
:10C5B00093901AF5E0FE04F0EEF91243C58B09EAF8
:10C5C000450970EDEE60EAF902C91A74EE1225937E
:10C5D000EAFEEBFF8C0E8D0F890C750A00750B00BF
:10C5E0001245DB8A088B097412122E61E0F50D7476
:10C5F00013122E61E0F510EA45097017E51060038B
:10C6000002C6EDA90CAC0EAD0FEEFAEFFB1245FF22
:10C6100002C7ECE510700302C6B89019E8E06004A8
:10C620006401700E901AFA12CF9B600612C8BD12F8
:10C630002779E50D700E850882850983E4F0750B76
:10C640000102C7109019E8E060076401600302C7A7
:10C6500010901A65E0A2E1400302C710901AFC1284
:10C66000CF9B600CA90DAA08AB0912C8BD1227798F
:10C67000850882850983E0FA12E960500109C3EA5E
:10C6800098E499A2D265D033500985088285098340
:10C69000E004F0850882850983E0F8905141E49335
:10C6A00068706D750A01EEFAEFFB1240178508827B
:10C6B000850983A3E4F08058E50D701CEA2402127A
:10C6C000B003A80C28F8E4340013E813F070098ACA
:10C6D000828B83A3A37401F08A828B83A3A3E0F8E7
:10C6E000901C59E0C3985052750B01804D74016540
:10C6F00010701DE50D60199019E8E0600464017088
:10C700000F901A65E0A2E15007EEFAEFFB12401716
:10C710009019E8E06402702274016510701CE50D48
:10C72000901B0C6013E004F0901CB8E0F8901B0C18
:10C73000E0C3984005750A01E4F0E50BA2E092F031
:10C74000E50AA2E072F0400302C7EC9019E8E0604D
:10C750000464017041901A65E0A2E15039EEFAEFED
:10C76000FB123D7D8A088B09A808A909E8496026C3
:10C77000E50BA2E0500D88828983A3A3A3A3A3E0C5
:10C78000C2E0F0E50AA2E0506388828983A3A3A3F4
:10C79000A3A3E0D2E0F0E50AA2E050509019E8E04F
:10C7A00060046401701D901A65E0A2E15015EEFA74
:10C7B000EFFB123D6BE9600BEEFAEFFB7900123EE6
:10C7C000B58029901A6EE06E7003A3E06F701DEEC5
:10C7D000FAEFFB7901123EB59019E8E06402700CA3
:10C7E0007A017B00901AC5E0F91234EF02C2AF74EF
:10C7F000F41225938A088B098C0A8D0B90819A7804
:10C8000008122C62700E7A017B00901AC5E0F912B2
:10C8100033BD8035901CA57808122DF2EA450945F4
:10C820000A450B60187808122B727A017B00901A67
:10C83000C5E0F91234E37404122B8D800C7A017B6D
:10C8400000901AC5E0F91234EF028FD1C082C08384
:10C85000901CA902AD89C082C083901CAB02AD8937
:10C8600074F612259375085775091A7808122B7AF1
:10C870007C6E7D007A217B001234957402122B8D20
:10C88000E9F508123D47E942089019E8E0600464C0
:10C89000017006123DC5E942089004DA12CF9B6090
:10C8A0000912C8BD122779E94208124107E9FE12B0
:10C8B0003B91E9F8E5084E48F9805F79C4E0F583DB
:10C8C00088822274F612259312332D750857750944
:10C8D0001A7808122B7A75086E7509007808122BE1
:10C8E0007A7C007D007A217B001234A17404122B23
:10C8F0008D123D4D9019E8E0600464017003123D13
:10C90000CB9004DC12CF9B600612C8BD12277912AF
:10C91000410D123BA38003122B8D7F020228197454
:10C92000F612259374FF122C0B7E007508577509BB
:10C930001A7808122B7A7C6E7D007A217B001234E3
:10C94000957402122B8DE9600302CA047808122B39
:10C950007A75086E8E097808122B7A7C007D007A31
:10C96000217B001234A77404122B8DE9600302CAE4
:10C9700004901A6BE064FE7003A3E0F4700302CA33
:10C98000047E01901A7AE064086005E06404706F28
:10C99000851882851983EE12CFD27942123C277A0C
:10C9A000827B1A7943123C277A7F7B1A7947123CA3
:10C9B000277A707B1A794A123C277A6E7B1A794B58
:10C9C000123C277A787B1A7950123C277A6B7B1AB3
:10C9D0007953123C277A807B1A7954123C277A6D5E
:10C9E0007B1A79E1123C27901A65E0A2E35004D249
:10C9F000F08002C2F012CFC87952123C2780051293
:10CA0000332D7E00123D3B9019E8E0600464017014
:10CA100003123DDD9004DE12CF9B600612C8BD12EA
:10CA20002779124119EEF9740102C91774F612251B
:10CA300093E9FEA2E0502675085775091A78081286
:10CA40002B7A75086E7509007808122B7A7C007DA8
:10CA5000007A217B001234A17404122B8DEEA2E324
:10CA60005003123D419019E8E0600464017008EE43
:10CA7000A2E15003123DE3EEA2E2500E9004E01258
:10CA8000CF9B600612C8BD12277902C91A74F6122C
:10CA9000259374EC122C0B7401122BEB901CEAE022
:10CAA000F97AC87B1A1243777405122E61E4F07488
:10CAB00007122E61E4F07A04F9123D59905156E4C0
:10CAC00093F8C3EA98EB94005058123D35E9705240
:10CAD00090513B12CB7E60197A047903123D598A3A
:10CAE000088B09905156E493F890513B12CB885033
:10CAF000087405122E617401F090513512CB7E60DE
:10CB0000197A027901123D598A088B09905156E42D
:10CB100093F890513512CB8850087407122E617427
:10CB200001F0901CEAE0F97CC87D1A7401122BE335
:10CB30001243717AC87B1A7945123C277407122E6A
:10CB400061E070117405122E61E07009851882850C
:10CB50001983E480088518828519837401F0901C7C
:10CB6000E4E0F8901CE3E058F8851882851983E02A
:10CB70005812CFD27941123C27741402C917E4939A
:10CB8000F8740193F9E84922E493FA740193FBE8FD
:10CB9000C39AF8E49BF9C3E50898E509992274F76C
:10CBA00012259374ED122C0BE9FE901AC4F0AC1808
:10CBB000AD19901CEAE0F97AC87B1A124377741217
:10CBC000122E61EE12CBDCAA18AB191243717AC88F
:10CBD0007B1A7945123C27741302B3FDF0901CEACE
:10CBE000E0F97CC87D1A2274F4122593EAFEEBFF6B
:10CBF000901CECE064FE7003A3E0F470767A167B80
:10CC00000012337B8A088B09EA450960668A828BA9
:10CC100083740112C2A68A828B83A360047402808B
:10CC2000027401F0EA240AF8E4350912C26912F12B
:10CC30000AA312DD08F0A2E3400912CC7612CC9CC4
:10CC40001243FBEE241512B9B1E5082402FAE435CB
:10CC500009FB123531E508241312CC88E4F0AA0848
:10CC6000AB09901AC5E0F912338712CC7612D54081
:10CC700012CCAB028FD112CC7A22EE240BF582E4D7
:10CC80003FF58322E5082412F582E412BF7C228E50
:10CC9000828F83A3A3A3A3A3A3A3A3A312D1D02270
:10CCA000E0F8A3E0F9851882851983E8F0A3E9F09C
:10CCB0002274F212259374FD122C0B8A088B0989B9
:10CCC0000A8C0B7401122E61740412CFD21244BB71
:10CCD0008A0C8B0DAE0CAF0DEE4F700302CD5F12C0
:10CCE000CD94740712DD0EE5082413FAE43509FB30
:10CCF0008A828B8312CDAA8A828B8312CDA9E50802
:10CD0000241512CC8812DD0812DD15E508240BF875
:10CD1000E43509F912CD6DE8F0A3E912DEA812445A
:10CD20003712DCF612CDB57401F07403650A6006A3
:10CD30007401650A700712CD7E7404800412CD7EE2
:10CD4000E4F0901CEC12B02112CCAB7401650B70B6
:10CD50000312CD77EEFAEFFB123DFBE9F980027981
:10CD600010901CEC74FEF0A304F0028B3EEE24182D
:10CD7000F582E43FF58322EE128926E4F02212CDFB
:10CD8000867440F0A322EE12CD8B22240FF582E4AC
:10CD90003FF58322EE12F4753FF58312CD9F22E01A
:10CDA000F8A3E0F98882898322A3E088828983F04E
:10CDB000A308A9832212CDB922F0EE12CDBF2224FE
:10CDC00013F582E43FF5832274F4122593EAFEEB17
:10CDD000FF7A007B04901AC5E0F91234EF12CE6F8F
:10CDE000901A7A7409F01244378A088B09AC08AD9E
:10CDF0000912B97012CC9C12352BE96401705A7A71
:10CE00000F7B0012337B8A088B09EA4509604A8A46
:10CE1000828B83740212CE64F988828983A3E0FC3A
:10CE200088828983A3A3E0FBEC8A82850983A3A37C
:10CE300012E16E88828983A3A3A3E08A8285098395
:10CE4000A312CE5CFAA3E0FB794A123C27AA08ABF6
:10CE500009901AC5E0F9123387028FD1F0EE24153C
:10CE600012BF6122F0EE241D12BF61F8A3E02290F0
:10CE70001A0312D54E901CABE8F0A3E9F0901A0506
:10CE800012D54E901CA9E8F0A3E9F02274F4122503
:10CE90009374FD122C0B8A088B097401122E617495
:10CEA0000212CFD21244BB8A0A8B0BAE0AAF0BEE32
:10CEB0004F700302CF7A12F494E412CFAFA3A3A36E
:10CEC000E06401700888828983A37420F085088259
:10CED000850983A3A3A3A3A3E064017009888289C1
:10CEE00083A3E0D2E6F0850882850983A3A3A3A3E8
:10CEF000A3A3E06401700A88828983A3E0D2E7805B
:10CF00000512B970740112CFC0E064017021850868
:10CF100082850983A3A312CF9B600312CF7F85086C
:10CF200082850983A3A312B00B12CD6E12CCAB8500
:10CF30000882850983A3A3A3A3A3A3A3E06401702C
:10CF40000712F005F0A3E4F085088285098312CC6E
:10CF50009C1244D9E9600412CF86F0EE241712CF58
:10CF60008212443712DCF612A32012CF8D12B9E4DC
:10CF7000FAEFFB123DFBE9F98002791002C054EE92
:10CF8000241612DD1D2212B9A8440422E0F8A3E001
:10CF9000F98E828F832212CFA1F58312D54EE849F4
:10CFA000228E828F8312BC7C241FF582E4382212E9
:10CFB000CFB32212CFB722F0850882850983A3223E
:10CFC00012CFB3A3A3A3A322A2F0E43385188285D2
:10CFD0001983F0AA18AB192274F512259374F31271
:10CFE0002C0B890AEAFEEBFF7508007509007C0D21
:10CFF0007D007900AA18AB1912336312C26A12D1EC
:10D0000087741F58600C7AD37B0012387379000242
:10D01000D0D7E8A2E55008740C122E617401F0E834
:10D02000A2E75008740B122E617401F0E8A2E674B6
:10D030000A5008122E617401F08008122E61E0641B
:10D040000170138E828F83A3A3A3A3A3A3A3E06085
:10D0500032EE241380128E828F83A3A3A3A3A3A3F3
:10D06000A3A3E0601EEE2415F582E43FF58312AA27
:10D07000416010AC08AD097402122E61AA82AB8324
:10D0800012353112CC7612CCA0740A122E61E064F3
:10D0900001703B12CC8F1244D9E97039EE240B1287
:10D0A000BADF901A6EE0687003A3E0697027E508A4
:10D0B0004509601A1244378A088B09AC08AD097417
:10D0C00002122E61AA82AB8312352BE96007AA18DF
:10D0D000AB19123EAFA90A740D02B66D74F7122592
:10D0E0009374CD122C0BEAFEEBFF8E828F8312D14C
:10D0F000A5A2E0400302D18212D18EE054FE12EDCF
:10D100006D740D122BEB12D1B8124431E9707374A7
:10D110002A122E6112D19B70697C0D7D007900AAC4
:10D1200018AB191233637416122E6112CCA0742A34
:10D13000122E6112D187A2E55008740B122E617471
:10D1400001F0E8A2E75008740A122E617401F0E8B9
:10D15000A2E65004742080027422122E6112B9B724
:10D160007402122E61AA82AB831235318E828F83B4
:10D17000A3A3E0C0E0740C122E61D0E012CFD21253
:10D180003EA9743302B3FD12E305A3E0F8228E82B8
:10D190008F8312D932A3A3A3A3A32212B51E6404C2
:10D1A000228A828B83E0F812D1AB22A3E0C8240646
:10D1B000F582E438F583E022EA241EF582E43BF5AB
:10D1C00083E0F9EA241FF582E43BF58312D1D022F3
:10D1D00012F105FB22E9F87900740468600A740A08
:10D1E00068600574036870027901022B2274F612DC
:10D1F00025938A828B837424F0A3A37401F0123EDA
:10D20000018A088B09AE08AF09EE4F60108E828F3D
:10D210008312DEA6124437EE241A12E167EEFAEF0B
:10D22000FB02C91AC082C083901A6802AD6FC08227
:10D23000C083901CEB02AD6FC082C083E9901CEBF1
:10D2400002AD8DC082C083901AE17401F0E9A2E3BF
:10D2500050037403F0E9A2E15004E0D2E2F002C509
:10D260008874F612259379007C008A088B09780867
:10D2700012285FF8FF0796D294D294D294D294D217
:10D280008CD290D296D288D27C01800A7C0480060F
:10D290007C0280027C08901AE1E05C6004790280E4
:10D2A00005EC6002790102C91A74F4122593EAFEB2
:10D2B000EBFF8908123D838A0A8B0BA80AA90BE8A9
:10D2C00049604188828983A3A3A3A3E06036C39405
:10D2D00005503174016508601A88828983A3A3A36D
:10D2E000A3E06401600D88828983A3A3A3A3E06403
:10D2F00002700A8882898312CC9C123F6FEEFAEF8B
:10D30000FB123D8F028FD174F61225938A828B8394
:10D31000E07014A3A3A312CF9B600C8A828B8312AC
:10D32000CC9912416780047A007B0002C91AC0823E
:10D33000C083901A7AE0640870031244FD02C58825
:10D34000C082C0837C00EC75F003A4F8ADF0EDF969
:10D3500012D4167003A3E06B7018905145E493C08B
:10D36000E074E428F582741A3DF583D0E0F079C5C5
:10D3700080620CECC3940340CD7C00EC75F003A4F8
:10D38000F8A9F074E528F582741A129AE964FE701F
:10D3900003A3E0F4600F0CECC3940340DE7C00ECCC
:10D3A00012D3D77026EC75F003A4FCADF074E42C16
:10D3B000F8741A3DF988828983A312E16D90514572
:10D3C000E49388828983F0790080090CECC394038C
:10D3D00040CD79C702C58875F003A4F8A9F074E4BC
:10D3E00028F582741A12EEF522C082C0837C00EC0C
:10D3F00075F003A4F8A9F012D4167003A3E06B70C3
:10D400000912D3DE6004790180090CECC394034057
:10D41000DE790002C58874E528F582741A12EEF5EB
:10D420006A2274F212259374DD122C0BEAFEEBFFD4
:10D430007508009019E8E060076401600302D539BF
:10D44000901A6BE06E7003A3E06F7010EE4F7003E4
:10D4500002D52D75080112450302D539123D7D8A8A
:10D460000A8B0BEA450B700302D52D8A828B83A3AE
:10D47000A3A3A3E0640160108A828B83A3A3A3A368
:10D48000E06402600302D52D851882851983E412B9
:10D49000D547740B122E61E8F0A3E912CFD2123DEA
:10D4A00029E9700302D52D850A82850B8312D540A8
:10D4B00012CCAB7900123F63850A82850B8312DAA6
:10D4C0005B122E61AC82AD837418122E61AA82ABFE
:10D4D00083123531850A82850B8312BAE5742012D6
:10D4E0002E6112CCAB7422122E61E4F07C02850A0C
:10D4F00082850B83A3A3A3A3E0F9740D122BE3127F
:10D500004497850A82850B8312BAE57401122E6155
:10D51000E8F0A3E912CFD2123D2F750801E50A24E5
:10D520000CF582E4350BF583129B4C800C901A7835
:10D5300012B9C7FAEFFB1245C3A9087423028B4046
:10D5400012D54E901CEC2212B19F12D54E2212D54C
:10D55000ABF922C082C08374FE122C0B9019E8E054
:10D560006004640170237901123F6912D591901A09
:10D570006BE8F0A3E912CFD27953123C27851882C9
:10D5800085198312CC9C12378F7402122B8D02C521
:10D5900088851882851983EAF0A3EB12D5A0F922B9
:10D5A000F085188285198312D5AB22E0F8A3E0221A
:10D5B00074F412259374F3122C0B8A088B09ECFE79
:10D5C000EDFF750A12EA45097005790002D69C90B4
:10D5D0001A6BE065087004A3E06509701D124437FA
:10D5E0008A0A8B0BAC0AAD0BEEFAEFFB12352BE976
:10D5F0007005750A018003750A00851882851983F4
:10D60000E4F004122E6112DE9412CFD2123D1DE915
:10D61000602A7403122E61AA82AB83123CF9E9647A
:10D62000017019750A017403122E61AC82AD83EE8C
:10D63000FAEFFB12352BE96003750A009019E8E058
:10D640006004640170177412650A7011EEFCEFFD3E
:10D65000AA08AB09123D65E96003750A00EEFCEF0C
:10D66000FDAA08AB091245E1E9F8740A687005756E
:10D670000A01801D74A0687012EEFCEFFDAA08ABD1
:10D68000091245F3AA08AB091246057401650A7030
:10D69000097900AA08AB0912450FA90A740D028F77
:10D6A000CE74F6122593EAFEEBFF89089019E8E0A4
:10D6B00060046401701E1244FDE508F50978091242
:10D6C0002B7E790DEEFCEFFD7AFC7BFF12451B747F
:10D6D00001122B8D02C91A74F7122593EAFEEBFF93
:10D6E0008E828F83A3A3A3A3A3A3A3A3E060161298
:10D6F000D73D129BEE12CC9C124509E964017005DE
:10D7000012CC7680298E828F83A3A3A3A3A3A3A385
:10D71000E0602512B9AE12CC8F124509E9640170A0
:10D72000178E828F83A3A3A3A3A3A3A3A3A312CC27
:10D730009C1244F179018002790002B400EE2415B4
:10D74000F582E43FF5832274F212259374FD122CC6
:10D750000B8A088B09ECFEEDFF890B750A01740139
:10D76000122E61740412CFD21244BBEA4B60427491
:10D7700011122E61E0601412DE0DE412E30D8A82B4
:10D780008B83E0D2E7F012D7B4E4F012D7BE12CD0B
:10D7900099740312DA65EE88828983A3A3F0EF8877
:10D7A000828983A3A312B19E12DD2A123DFBE9F503
:10D7B0000A028B3CEA2414F582E43BF5832212F43E
:10D7C000743B2274F0122593EAFEEBFF890A750B75
:10D7D00001EE12DB273F12D92BF50C88828983A337
:10D7E000A3E0FA8882898312D91A12B97964046095
:10D7F0000A7AD37B0012387302D90AE50C122A2A5E
:10D8000002000215D8030BC2D8030CA8D80D80D88B
:10D810000EC2D8BFD89019E8E06007640160030227
:10D82000D8C2901A65E0A2E1400302D8C27900ABE9
:10D8300009123FF9EA4B603D8A828B83A3A3A3A31D
:10D84000A3A3E05418602E12CC761229A58A828BED
:10D8500083A3A31229A579008E828F83A3A3A3A3F8
:10D86000A3A3A3A3A312D90E12CC9C12401174043B
:10D87000122B8D802E7901AA08AB09123EC180427D
:10D880009019E8E0600464017038901A65E0A2E144
:10D890005030AB091244EBAA08AB091244F1E96419
:10D8A000C5701F750B00801A9019E8E060046401D0
:10D8B0007010901A65E0A2E150081237B38003752A
:10D8C0000A00EE2409F50EE43FF50FAC08AD09A9F6
:10D8D0000C850E82F58312CC9C123ED9850E828572
:10D8E0000F8312CC9C1244D9E9601F12BF5AC39413
:10D8F00002401712CC7612E2307003A3E069600A8E
:10D90000E50BA2E05004A90A80027900803112D907
:10D91000122212B9BF8A828B8322A3A3A3E0F8E468
:10D92000C8F9EA28F508E439F50922F58312D93255
:10D93000E02212D5ABF988828983A322122B8D7F36
:10D940000802281974EE12259374F5122C0B8A0A1A
:10D950008B0B890D8C0E8D0F7E01EE122E61740AD9
:10D96000F0741D122E61E0F50CE9700FE50CC33365
:10D97000240AC0E0EE122E61D0E0F0AA18AB191212
:10D9800044BB8A088B09EA4509700302DA3D12C4D8
:10D99000D8350912DBDB7409F0A3E50DC43354E07C
:10D9A000450C12DBF4AC0EAD0FEEFAEFFB12353185
:10D9B000EE2408FE50010FE50D702F7C00741E123E
:10D9C0002E6112DA4C801D12DA44EA28F8EB39F99C
:10D9D0008882898312DBEF8882898312A1BCF0A33D
:10D9E0000EAF830CECC3950C40DDE508241712CC78
:10D9F000887401F0124437E508241AF582E43509E9
:10DA000012DA59122BEBAA0AAB0B123D05E9601989
:10DA1000E508241612CC887401F07403122BDBE5A0
:10DA200008241812CC8812CCAB850882850983A300
:10DA3000A312DA63AA08AB09123DFBE9FEEEF97402
:10DA40000B02C2ACEC25E0F8E433F92212DA5022E2
:10DA500012D5ABF9E8FAE9FB22F583EAF0A3EBF083
:10DA6000740322E50AF0A3E50BF02274F01225936B
:10DA700074F8122C0B8A088B0912DB26350912DC8C
:10DA80006FF8741F58F50A880BA3AE82AF83EEFCC3
:10DA9000EFFDAA18AB19123531EE2408FE50010F24
:10DAA000AC18AD197A8C7B1A12352BE9607374E0CF
:10DAB000550B7066AA0AEA2AFA7B0012341D8A0CFA
:10DAC0008B0DEA450D605A7C00801D8E828F83127B
:10DAD000C50312DA44E50C28F582E50D3912E16B35
:10DAE000EE2402FE50010F0CECC3950A40DD780CC9
:10DAF000122B7A780A122B7E7403122BEB7900E535
:10DB000008240B12CC8812CC9C1245337403122BC0
:10DB10008DAA0CAB0D12342380077AD37B00123808
:10DB200073740802D93CEA241DF582E42274F012D1
:10DB300025938A0A8B0B890D8C088D099019081280
:10DB4000CF9B60757410122E61E0F50C12DA45E877
:10DB5000240EFAE439FB12337B8A0E8B0FAE0EAF24
:10DB60000FEE4F60548E828F8374D4F012DBCAA301
:10DB7000A3E50DF0AC08AD09EE2405FAE43FFB1275
:10DB8000353112DBBCE50CF07411122E6112E2F695
:10DB90007808122B76AC0CEC2CFCE433FDEE240E52
:10DBA000FAE43FFB1233577403122B8DEEFAEFFBAE
:10DBB00090190812E30112277902D93FEE12DBC156
:10DBC00022240DF582E43FF58322A3A3E50AF0A306
:10DBD000E50B12DBD62212BFA0A322F58312DBEAEB
:10DBE000FF8E828F832288828983E0FEA3E022E079
:10DBF0008E828F83F0A3AE82AF832274F6122593B8
:10DC000074F8122C0B890812DB263B12DC6FF974B6
:10DC10001F59F88909A3AE82AF837401687042EE80
:10DC2000FCEFFDAA18AB19123531EE2408FE5001A5
:10DC30000FAC18AD197A8C7B1A12352BE960297458
:10DC4000E05509701C8E828F83A3E0FA8E828F8349
:10DC5000A312C5058E828F83E0F9124563A908805F
:10DC6000097AD37B001238737900740802C917F55A
:10DC700083E02401FEA3E03400FF8E828F83E02244
:10DC800074F012259374FD122C0B8A0A8B0B8C08EE
:10DC90008D09890D750C017401122E61740312CF68
:10DCA000D21244BB8A0E8B0FAE0EAF0FEE4F603F09
:10DCB00012CD94740BF0A3E50D12DD0E7413122E29
:10DCC0006112DD0812DEA812443712DCF612DD15EF
:10DCD000EE2418F582E43F12DD288E828F83A3A301
:10DCE000E50AF0A3E50B12DE9B123DFBE9F50CA95A
:10DCF0000C740302D93C12DCFEEAF0A3EB22EE2402
:10DD00001AF582E43FF58322E08882898322F0A31A
:10DD1000A882A98322F0EE241612DD1D22F582E4EA
:10DD20003FF5837401F02239F58312DE94F02274FA
:10DD3000EF122593EAFEEBFF751000EE12DB273F92
:10DD400012DF7BF508A3E0F50912D73D12CC9C1237
:10DD50003D83EA4B700302DE088A828B83A3A3A370
:10DD6000A3E0700302DE08C39403400302DE08E56B
:10DD700008C3940F5004E50960057510018079EA25
:10DD80002412F582E43BF583E4F0E508702290501C
:10DD9000147808122D3A12DE0D7808122DF29050E8
:10DDA000147808122D3A12E7647808122DF280399F
:10DDB00075090074027808122D1474142508F58270
:10DDC000745012CC8B780C122D3A90813E78081248
:10DDD0002DD4780C790812242E12DE0D780C122D19
:10DDE000F212E764780C122DF2EA241BF582E43B70
:10DDF000F5837401F01237FB9019D6E0FCA91012DC
:10DE0000CC7612CC9C12454B7F09022819EA2417C4
:10DE1000F582E43BF5832274F012259374F5122CFD
:10DE20000B8A088B09890B8C0C750A017401122E60
:10DE300061740312CFD21244BB8A0E8B0FAE0EAFA9
:10DE40000FEE4F604812CD94740C12DA65A3E50C06
:10DE500012DEA8124437EE241AF582E43F12DA5992
:10DE6000122BEBAA08AB09123D05E9600E12CF7F19
:10DE70007403122BDB12CD6D12CCAB8E828F83A379
:10DE8000A312DE9412DE9B123DFBE9F50AA90A7487
:10DE90000B02D93CE508F0A3E5092212CDB97401C3
:10DEA000F0EEFAEFFB227401F0EE241712DD1D22D2
:10DEB00074F012259312DB263B12DF7BF8A3E0FE01
:10DEC000E8600302DF7874016E600874026E60031C
:10DED00002DF78EE9019D6F07508D6750919780822
:10DEE000122B7A7508017509007808122B7A7C00CC
:10DEF0007D007A517B001234A17404122B8D7402C0
:10DF00006E7075901CCCE0700A9050147808122D39
:10DF10003A8028F50874027808122D147414250824
:10DF2000F582745012CC8B7808122D3A90813E788D
:10DF30000C122DD47808790C12242E908116780CAE
:10DF4000122DD47808790C122524908106780C12B1
:10DF50002DD47808790C12242E9019D87808122D17
:10DF6000F29019D812299D7A007B40901AC5E0F9E9
:10DF70001234E97404122B8D02D93FF583E0240199
:10DF8000F8A3E03400F988828983E02274F6122530
:10DF90009374DA122C0BEAFEEBFF12CF9660508ED0
:10DFA000828F8312CC9CAC18AD1912D1B812441FC9
:10DFB0007409122E6112E2307003A3E0696030121E
:10DFC000E2FD1229A57508FE7509FF7808122B7A63
:10DFD000741C122E61E0F9740D122E6112B9B7741F
:10DFE0000F122E6112CC9C1240117404122B8D74EE
:10DFF0002602C91774F7122593E9FD7A007B009079
:10E0000019E8E06004640170407C00800B12E0A01D
:10E01000E02AFAA3E03BFB0C90515612EEE35029A4
:10E02000EC75F01CA4F8AEF0EEF912EF05F460E721
:10E03000740328F58274063912CF9960DAED60CD49
:10E0400012E0A0E4F0A3F080CE7C00800B12E08D03
:10E05000E02AFAA3E03BFB0C12EEE0502DEC75F049
:10E0600017A4F8AEF0EEF912F0847003A3E0F460A8
:10E07000E6746C28F58274093912CF9960D9ED6085
:10E08000CC12E08DE4F0A3F080CD02B400EC75F08A
:10E0900017A4F8EEF9746C28F582740939F5832217
:10E0A000EC75F01CA4F8EEF9740328F582740639B7
:10E0B000F5832274EC122593890CEAFEEBFF901A8B
:10E0C000C4E0C3950C503B12448B901AF612E10940
:10E0D000901A5EE0F508E4F509F50AF50B90817EEB
:10E0E0007810122DD47808791012242E7808122B6B
:10E0F000727A007B02901AC5E0F91234E3740412BC
:10E100002B8D0287398A828B83EEF0A3EFF0227485
:10E11000F6122593EAFEEBFF901AE28013888289BB
:10E1200083E06E7003A3E06F603A88828983A3A3C3
:10E1300012CF9B70E87A047B0012341D8A088B0989
:10E14000A808A909E849601C8882898312E109901E
:10E150001AE212CC9C88828983A3A312E16D901AE3
:10E16000E212CCAB02C91AF582E43FF583EAF0A3D0
:10E17000EBF02274F41225937E00901AE280070ED1
:10E180008A828B83A3A312B30B70F4EE25E0FAE42A
:10E1900033FB12341D8A088B09EA4509607F7C0035
:10E1A000901AE280228A828B83E0F50AA3E0F50BC5
:10E1B00012DA44E50828F582E50939F58312DA63B5
:10E1C0000C8A828B83A3A312B30B70D9901AC0124E
:10E1D000E2307003A3E0697808701C122B7AEEF528
:10E1E0000A780A122B7E7C8C7D1A7900901AC01254
:10E1F000CC9C124533801A122B7AEEF50A780A125B
:10E200002B7E7C8C7D1A7900901AC012CC9C124512
:10E21000277403122B8DAA08AB09123423123E1364
:10E22000028FD18E828F83A3A3A3A3A3A3A3A3A3AF
:10E2300012D54E901A6BE06822C082C08380128A89
:10E24000828B83A3A312BAE5901AE212CCAB1234EC
:10E2500023901AE212B30B70E602C58874F51225FA
:10E2600093901A7812BC73901AF612A03B12CCABA2
:10E270007AF67B1A7950123C27901AF612E2F68051
:10E280001312EBAD7004A3E06509600612EBBA123D
:10E2900045CF050A905149E493F8E50AC398502008
:10E2A000E50A75F017A4F8A9F012EA5B6E7003A3F3
:10E2B000E06F70CD746128F582740912DD2780D279
:10E2C000901AF612BC7390190A12CF9B60257A0639
:10E2D0007B0012337BEA4B601A8A828B8374D5F001
:10E2E000A3A3E412E6A80412E30D90190A12E301B5
:10E2F00012277902B670128748750A00228E828F23
:10E300008312E3052212D5ABF58388822212B1ABCA
:10E31000EEF0A3EFF022C082C083901A6BE064FE9F
:10E320007003A3E0F4600E901A65E0A2E1500612BB
:10E3300045E712458D02C58874F0122593901AB9ED
:10E34000E06053F50CE4F50DF50EF50F90810678BD
:10E3500008122DD4780C790812242E1233758A08ED
:10E360008B09A808A90990513DE49358F508A3E446
:10E370009359F509E4F50AF50B780C7908122CEE9F
:10E38000780C122B727A007B01901AC5E0F91234D6
:10E39000E97404122B8D02D93F74EE1225937E008E
:10E3A0007F008E0A8E0B123DAD750D00803BAA0DCD
:10E3B0007B00123DA78A088B09A808A909E84960D3
:10E3C0002688828983A3A3A3A3E060046404701752
:10E3D00088828983A3A3A3A3A3A3A3A3A3A3E0F9F0
:10E3E0001245F9E960010F050D905156E493F8E5E7
:10E3F0000DC39840B91245BD8A0E8B0F750C008075
:10E4000023AA0C7B001245C98A088B09A808A90910
:10E41000E849600EE8240F129AE6F91245F9E9601E
:10E42000010E050CC3E50C950EE4950F40D3EF2EBD
:10E43000FE700302E52F8E08750900740278081239
:10E440002D14AA08AB0912341D8A0A8B0BEA450B5E
:10E45000700302E52D750C008E08750900740278B2
:10E4600008122D14AC08AD0979FF123363750D0045
:10E47000805EAA0D7B00123DA78A088B09EA450938
:10E48000604C8A828B83A3A3A3A3E060046404701E
:10E490003D8A828B83A3A3A3A3A3A3A3A3A3A3E0E7
:10E4A000F91245F9E9F96026050C780A122B7AEE83
:10E4B000FD850882850983A3A3A3A3A3A3A3A3A384
:10E4C00012E5C012CC9C1245937402122B8D050DDF
:10E4D000905156E493F8E50DC3985006E50CC39FA0
:10E4E0004090750C00C3E50C950EE4950F5040AAC2
:10E4F0000C7B001245C98A088B09EA4509602AEAA3
:10E50000240F12B003F91245F9E9F9601C780A12D8
:10E510002B7AEEFDE508240E12CC8812E5C012CC51
:10E520009C1245937402122B8D050C80B87E007FDF
:10E5300062901A63E0600BF91242BDE9F87454C3AB
:10E5400098FF75F003EF84F50D94204003750D1FBF
:10E55000850A08850B09750C00EF6005750C207F96
:10E5600000E50DC39E5005850D0F80088E0FE50C4C
:10E57000D2E6F50CAC08AD09AA0CA90F124599E931
:10E58000F50EE50CA2E6401D150F7800800BE5089E
:10E590002404F5085002050908E8C3950F40EFE58B
:10E5A0000FCEC39EFEE97006E50CA2E650A8E50A70
:10E5B000450B6007AA0AAB0B123423A90E02C2AFA7
:10E5C000E0FC8508828509832274F2122593EAFE15
:10E5D000EBFF89088C098D0A7C007D00740E122ED9
:10E5E0006112CC9C750B00800DEAFCEBFDEA240463
:10E5F000FA50010B050BE50BC3950A400302E698A0
:10E600008A828B83E0F47003A3E0F4607AEC4D60BF
:10E610000C8C828D83C3E09EA3E09F50CC8A828BBA
:10E620008312E69BEE98EF9950BFEAF8EBF98882E7
:10E630008983E0F47003A3E0F46010E82404F85048
:10E640000109050BE50BC3950A40E3E8FCE9FDE889
:10E6500024FCF8E934FFF98882898312E6A08C82D1
:10E660008D83E50CF0A3E50D12E6B78C828D83A3B4
:10E67000A312E6ADA3A3A3E08C828D83A3A3A3F092
:10E68000C3EA98EB9940C412E1058A828B83A3A365
:10E69000E50912E6A8E508F0028B4312D54EC32225
:10E6A000E0F50CA3E0F50D2212B19FA32212E6B112
:10E6B00022F0888289832212E6BDA3E02212E6B10D
:10E6C000A32274F212259374FD122C0B89088A0977
:10E6D000ECFEEDFF750A0175F003E9A42402C0E029
:10E6E0007401122E61D0E012CFD21244BBEA4B600B
:10E6F0007012D7BE12CD997408F0741F55084509E1
:10E70000A3F0E82402F8500109750A0080338E82D4
:10E710008F8312DD0812DD0E8E828F8312CDA98EBB
:10E72000828F83A3A3E05407C4FC8E828F83A3A3AC
:10E73000A3E054074C12CDABEE2404FE50010F05AC
:10E740000AE50AC3950840C68A828B83A3A374FC9A
:10E75000F0A374FFF012E7647401F0123DFBE9F5D9
:10E760000A028B3CEA2413F582E43BF5832274F120
:10E770001225938A0A8B0B7508007AFE7BFF7CFEBC
:10E780007DFFE50A12DB27350B12D92BF509741F23
:10E790005509F50CE82402F8500109E509A2E74003
:10E7A00065E50A2417F582E412F5A7FE75F003E586
:10E7B0000CA424026E704FE50C600612DBE6FBEE43
:10E7C000FA750D00801DE05407F50EA3A882A983F9
:10E7D000EEFC901A6BE06E7003A3E06F7003850E81
:10E7E00008050DE50DC3950C502612DBE6FCE4CCC4
:10E7F000FDEE2CE43DFFE82402F8500109888289EF
:10E8000083E0548860C07AD37B0012387302E951E8
:10E81000E508700BA9091245A5E9700302E9511238
:10E82000E95612CC9C123D7D8A0C8B0DAE0CAF0DBF
:10E83000EE4F605A8E828F83A3A3A3A3A3A3A3E466
:10E84000F090514193F88E828F83A3A3A3A3A3A337
:10E85000A3A3E0C398402412E9605001097A027B27
:10E8600000122337E88E828F83A3A3A3A3A3A3A3BD
:10E87000A3F0E508C39407500205088E828F83A396
:10E88000A3A3A3A3A3A3A3A3E508F002E9517CFFDC
:10E890007DFF12E95612CC9C1245B18A0C8B0DAE4D
:10E8A0000CAF0DEE4F704F1245B78A0C8B0DAE0CAE
:10E8B000AF0DEE4F700302E9517C177D0079001215
:10E8C000336312E95612CF8C1287968E828F83A300
:10E8D000A3A3A3A3A3A3A312B9E412B52F74AA12EE
:10E8E000E97F5001097A027B0012233712DBBCE872
:10E8F00012E96B7401F0905141E49312BF69C3981F
:10E90000401912E9605001097A027B001223371284
:10E91000F00BE508C394075002050812EFF7E5086D
:10E9200012E970E4F012A033123CF9E97023850A71
:10E9300082850B83A3A3A3A3A3A3A3A3E06012E5F3
:10E940000A2415F582E4350B12B9C512A03412352C
:10E95000317F07022819E50A12F475350BF5832279
:10E96000905141E49379002401F822F012EFFB2248
:10E97000F012E97522EE240CF582E43FF58322F0D3
:10E98000905141E49379002401F82274F712259301
:10E99000E9FE74FE6A700374FF6B603474605E6439
:10E9A00060602DEEA2E5401CA2E6901A6B500DC3EC
:10E9B000E09AA3E09B5019790002B400C3E09AA347
:10E9C000E09B40F3901A6B12E69BEC98ED9940E7C0
:10E9D000790180E574F71225937E008008EE12EB32
:10E9E000B31245CF0E12EA1540F37E00EE75F00328
:10E9F000A4F8A9F074E428F8741A39F98882898394
:10EA0000A374FEF0A30412E6ADE4F00EEEC394038B
:10EA100040DA02B400905149E493F8EEC3982274AE
:10EA2000F71225937E0080010E12EA155026EE1291
:10EA3000EA6B6A7003A3E06B70EE12EA5B6C700322
:10EA4000A3E06D600A74FF6C700374FF6D70D912DF
:10EA5000EBBA80047A007B0002B40012EA5F2274F1
:10EA60006128F582740939F583E02275F017A4F85E
:10EA7000A9F012EA762212EED5E02274F61225935E
:10EA80007CFF7DFF7AFE7BFF1245B1EA4B703C753F
:10EA900008008032E50875F017A4F8A9F07466281C
:10EAA000F5827409129AE9600512EEFA701674572D
:10EAB00028FE740939FF8E828F8312CC9C12401776
:10EAC000EEFAEFFB050812EACE40C902C91A9051CE
:10EAD00049E493F8E508C39822C082C0837A007B9A
:10EAE000007C00801012F07C7003A3E0F460050A43
:10EAF000EA70010B0C12EEE040EB02C58874F412D0
:10EB000025938A088B09ECFEEDFF800B1245CFEEB2
:10EB1000FCEFFDAA08AB091245B1EA4B70EE028F7B
:10EB2000D174F71225937D007C0080020D0C12EE4B
:10EB3000E0501C12F07C7003A3E0F460F0EDF8EA02
:10EB4000684B70E8EC75F017A4F812EBBA80047A01
:10EB5000007B0002B40074F7122593EAFEEBFFEE8F
:10EB60004F60187C177D0079001233638E828F838B
:10EB700074FEF0A30412F012F0A3F002B40074F6D5
:10EB80001225938A088B097E00801AEE75F017A46F
:10EB9000F8A9F012EBAD7004A3E06509600612EB72
:10EBA000BA1245CF0E12EA1540E102C91A12EA5F05
:10EBB00065082275F017A4F8A9F0745728FA7409AB
:10EBC00039FB2274F41225938A088B09ECFEEDFFC1
:10EBD0009019E8E0600464017020901A78E06E708B
:10EBE00003A3E06F7014123D7D8A0A8B0BA80AA95B
:10EBF0000BE8496005E82408801AEEFCEFFDAA083E
:10EC0000AB091245B18A088B09A808A909E849602F
:10EC100009E8240DFAE439FB80047A007B00028FB6
:10EC2000D174F41225938A088B09ECFEEDFF750A66
:10EC300000750B00802FE50B12F06C123CF9E960B7
:10EC400022E50B12EA6B65087004A3E06509700306
:10EC5000750A0AEEFCEFFD12F07312352BE9600322
:10EC6000430AA0050B905149E493F8E50BC3985073
:10EC700004E50A60C1A90A028FD174F61225937EB9
:10EC800000805AEEFA7B00123DA78A088B09A8087B
:10EC9000A909E849604688828983A3A3A3A3E06405
:10ECA00001603988828983A3A3A3A3E06402602C56
:10ECB000E82407129AE6FA74012AF0901ABAE0C31F
:10ECC0009A501988828983A3A3A3A3A3A3A3A3A370
:10ECD000A3E412ED62A312ED6D1240170E9051568F
:10ECE00012EA18409E7E008059EE75F017A4F8AA2B
:10ECF000F0EAF912F0847003A3E0F460447457283A
:10ED0000F8740939F9E8240C129AE6F8740128F02D
:10ED1000901ABAE0C3985029EE75F017A4F8EAF9F2
:10ED2000745728F8740939F9E812ED5C39F583E471
:10ED3000F0E8240EF582E439F583E412ED6D12401B
:10ED4000170E12EA1540A27A00EA12D3D760021415
:10ED5000F00AEAC3940340F102C91AEE240FF582C7
:10ED6000E42212E6BDA3A3A3A3A3A3A32212E6B1A8
:10ED700012D1D02274F11225938A0A8B0BECFEED8E
:10ED8000FF750E007A007B017508FE7509FF740F90
:10ED9000122E6112E6A08011123375E50EF5F0EA2D
:10EDA00084E5F0FA750E007B007C00800712EED53A
:10EDB0001287440C12EEE0505CEC75F017A4F8AD2D
:10EDC000F0EDF912F0847003A3E0F460E612EA7249
:10EDD000650A7004A3E0650B60D912F0677003A3A5
:10EDE000E06F60CF12EA72650C7004A3E0650D60FD
:10EDF000C212EEFA60BDC3940850B8E0640760AD7B
:10EE0000EB050E70AEE50EC39A40A8745728F58244
:10EE1000740902EE9F9019E8E06007640160030244
:10EE2000EEA77C00800712EF151287440C90515614
:10EE300012EEE35072EC75F01CA4F8ADF0EDF9128F
:10EE4000EF1064FE7003A3E0F460E112EF10650AB6
:10EE50007004A3E0650B60D412EF106E7003A3E0A2
:10EE60006F60C912EF10650C7004A3E0650D60BC03
:10EE700012EEEA60B7C3940850B212EF0564016065
:10EE8000ABE0640260A612EEEA64076099EB050E3F
:10EE9000709AE50EC39A409474F328F58274053D88
:10EEA000F58312CC9C802BE50E6011EA700E740184
:10EEB000650E600302ED987A0102EDA474FE650808
:10EEC000700474FF65096006AA08AB0980047AFE25
:10EED0007BFF02E951745728F582740939F58322C2
:10EEE000905149E493F8ECC3982274FC28F582749D
:10EEF0000512EEF52239F583E022746528F5827457
:10EF00000912EEF52274F728F582740512EEF52247
:10EF100012EF15E02274F328F582740539F5832287
:10EF200074F51225938A088B09ECFEEDFF750A0033
:10EF30008002050A905149E493F8E50AC3985022EB
:10EF4000EEFCEFFDE50A12F06C12352BE960E3E50B
:10EF50000A75F017A4F8A9F0745728F582740912FD
:10EF6000DD2702B670E9F87907C3940D40047901F2
:10EF70008019E8C3940740047903800FE8C3940321
:10EF8000400479058005E870027900022B2274F0B4
:10EF90001225938A088B098C0A8D0B890C1245B7B0
:10EFA0008A0E8B0FAE0EAF0FEE4F60487C177D00C0
:10EFB00079001233638E828F8312DE9412F0121264
:10EFC000DA63E50C600712B52EE50C800312F0053C
:10EFD000F0901ABFE06401700612EFF7E4800512AA
:10EFE000EFF7740712E97F5001097A027B001223C0
:10EFF0003712F00B02D93F12EFFB22EE240EF582FE
:10F00000E43FF5832212CD86740122EE12DBC1E8C3
:10F01000F02212A9B4A32274F7122593EAFEEBFFA3
:10F02000750800803AE50875F017A4F8A9F012F009
:10F03000677003A3E06F601474FF6E700374FF6F5A
:10F04000701B12F0847003A3E0F4601112F07312CD
:10F050003CF9E97008E50812EBB31245CF05081238
:10F06000EACE40C102B40012EA766E2275F017A40F
:10F07000F8A9F0745928FA740939FB22EC75F017D5
:10F08000A4F8A9F012EA7664FE22C082C0837AFF57
:10F090007BFF12460502C588C082C083901AF874AF
:10F0A00017F0A37446F0901AFA741DF0A37446F09A
:10F0B000901AFC7423F0A3744602AD8D74F71225E8
:10F0C00093EAF8EBF9901A0112F105CA2406F582C9
:10F0D000E43AF583E0702B88828983A3A3A3A3A3DA
:10F0E000A3A3A3A31229A5901A0112F10A122E328A
:10F0F00088828983A3E0F9123ECD7402122B8D120F
:10F100003E1302B400E0FAA3E02212F105F5838A6F
:10F110008222C082C083901AC212F1D6F0901AC225
:10F1200012CF9B7005790112455D02C58874F612F5
:10F13000259374FC122C0BE9FE905143E493700864
:10F1400074E16E600302F1D1EA2408F8E43BF98827
:10F1500082898312F1D612F1DF700E901AC2E4F0A8
:10F16000A3F0790112455D8068901CE0E06062F8D0
:10F17000901AC212CC9CC3E89AE49B5054790012B6
:10F18000455D8A088B09AC08AD09ECF8EDF9E87526
:10F19000F064A4F8AAF075F064E9A42AF9901AC200
:10F1A00012CC9C12233FE8941AE994004023901952
:10F1B0000212CF9B601B901AC212CCA07402122EB6
:10F1C00061ECF0A3ED12CFD290190212E3011227E5
:10F1D00079740402C917E02401F0A3E0340022127C
:10F1E000E6B112D54EE84922C082C08374F8122CD1
:10F1F0000B9080D8AC18AD197408122A9EAC18ADCB
:10F200001912352BE96401700479008002790174C8
:10F210000802D58B74F6122593740C122E6112BC61
:10F2200073743A6E7001EF6006743B6E4F70237416
:10F230000A122E611229A58C088D097808122B7AE2
:10F24000EAFCEBFDEEFAEFFB1234A77404122B8DEF
:10F250008002790A02C91AC082C083901AFE74B370
:10F26000F0A3743DF0901B0074B9F0A3743DF090CE
:10F2700019D6E064017032901B027441F0A3744609
:10F28000F0901B047447F0A37446F0901B06744D75
:10F29000F0A37446F0901B087453F0A37446F090EA
:10F2A0001B0A743BF0A37446F0901B0212CF9B60C4
:10F2B0000612C8BD12277902C58874F4122593740A
:10F2C000E6122C0B8A088B097404122E617402F06A
:10F2D00004122BE31244BB8A0A8B0BAE0AAF0BEE6F
:10F2E0004F700302F44412F494746012CDB512DE30
:10F2F000A612443712DCF612B9E012DE9412BFC136
:10F300007012901A57E0C0E012F449D0E0F0901A61
:10F3100057E004F012F4657016901CC0E0600D9088
:10F320001A62E0700A8E828F83E0700312CD77AC90
:10F3300018AD19EEFAEFFB1244138A088B09EA455F
:10F3400009700302F43D7A217B0012341D74061209
:10F350002E6112E16D7406122E6112CF9B700302B2
:10F36000F4367C217D0079007406122E61E0FA12D9
:10F3700033637401122BE37950123C217401122E75
:10F380006112BAE57406122E6112F105CA2409F55C
:10F3900082E43AF58312CCAB901A6B12BAE574177B
:10F3A000122E6112CCAB7406122E6112BC7812F4CC
:10F3B0006BF07406122E6112B0EE740212F4BA747D
:10F3C00006122E6112F10A12CCAB7406122E6112D3
:10F3D000F49F12F4C5C0E07406122E6112BC7812BC
:10F3E000F47BD0E0F0EE240E12F453C0E074061269
:10F3F0002E6112F484D0E0F07406122E6112BC78F3
:10F4000012BC6912DD28EE240F12BADF740C122E22
:10F410006112CCAB8A828B83E0C0E0740E122E6145
:10F42000D0E0F07406122BE31243897406122E61A9
:10F4300012CC9C123423AA08AB09123423EEFAEF43
:10F44000FB123423741A028FCEEE2414F582E43FAB
:10F45000F5832212F458E022F8E43FF9E8FAE9FBD8
:10F460008A828B832212BF5E64012212F47538F502
:10F4700083740222EA240BF582E422241EF582E43E
:10F4800038F5832212F4882212BC7C240CF582E425
:10F4900038F5832212CC7A12CD9F7404F0A322E0B7
:10F4A00012F4A97401F0A3E422F8A3E0C812F4B1A5
:10F4B00022240DF582E438F5832212DBD612D54ED4
:10F4C00022E8F0A3E912A804E02274F61225937E44
:10F4D0000080187C047D0079FF8E088D0974027805
:10F4E00008122D1412F7051233630E90514012EAE0
:10F4F0001840E002C91A74F412259374F7122C0B09
:10F50000750800802285080A750B007402780A12BB
:10F510002D1474F6250AF582740C12F5A724FFF059
:10F52000A3E034FFF0050890514012EAD1506D85F8
:10F53000080A750B007402780A122D1412F59FF454
:10F540007003A3E0F460DE85080A750B007402788E
:10F550000A122D1474F6250AF582740C350B12CF9D
:10F560009970A27408122E617402F085080A750B56
:10F5700000780A122D1474F4250AFE740C350BFF62
:10F580008E828F8312CCA012F5AD123C697C047D73
:10F590000079FFEEFAEFFB123363808902B0E97461
:10F5A000F4250AF582740C350BF583E02212F71E60
:10F5B0002274EE12259374F7122C0BEAFEEBFF7502
:10F5C0000CFF7408122E6112F710123C63E9641AE2
:10F5D000700302F683750E00741B122E61780812F8
:10F5E0002DD4800B74FF650C7003850E0C050E90F6
:10F5F0005140E493F8E50EC3985048850E107511FC
:10F600000074027810122D1412F687F47003A3E030
:10F61000F460D1850E1075110074027810122D144B
:10F6200012F6876E7003A3E06F70C2750F0074024C
:10F63000780E122D1474F6250EF582740C350FF524
:10F64000838030E493650E702D74FF650C602E8509
:10F650000C0E750F007402780E122D1474F4250E22
:10F66000F8740C350FF98882898312E10988828940
:10F6700083A3A312DD2A7901740902C2AC12F5AD8D
:10F68000123C69790080F174F42510F582740C3510
:10F6900011F583E02274F412259374F7122C0BEA0F
:10F6A000FEEBFF7408122E6112F710123C69750808
:10F6B000008002050890514012EAD1504585080AA1
:10F6C000750B007402780A122D1412F59FF4700362
:10F6D000A3E0F460DE85080A750B007402780A1254
:10F6E0002D1412F59F6E7003A3E06F70C67C047D2D
:10F6F0000079FF8D0974027808122D1412F7051293
:10F70000336302B0E974F42508FA740C3509FB225E
:10F71000740212A804EEF0A3EFF012F71E22901A62
:10F720007812B9BFAA18AB192274EE1225938A0871
:10F730008B09ECFEEDFF750A00EE65087003EF65BE
:10F7400009600C12349B8A0C8B0DEA450D7006750E
:10F750000A0102F7E5EEFAEFFB12349B8A0E8B0FDB
:10F76000AC0EAD0FEC4D6007EEFAEFFB1234ADE4DA
:10F77000F50EF50F780E122B7AAC0CAD0DEEFAEFFC
:10F78000FB1234957402122B8DE96059AA0CAB0D53
:10F7900012341D8A0E8B0FEA450F6046780E122B2D
:10F7A0007A780C122B7A7C007D00AA08AB091234FF
:10F7B000A77404122B8DE9701D780E122B7A780C29
:10F7C000122B7A7C007D00EEFAEFFB1234A1740458
:10F7D000122B8DE96003750A01AA0EAB0F123423B8
:10F7E0008003750A10A90A02C2AF122398022B22C5
:10F7F000C082C08374FF122C0BAC18AD197A01794A
:10F800008712FE47C39403400F7402F07C007D0012
:10F81000FA79E2123591800CE4F0901CDFE0FA7B7B
:10F82000001236C37401122B8DD083D082022B229A
:10F8300074F012259374F5122C0B851882851983A8
:10F84000EAF0A3EBF0ECFEEDFF750820E97003028F
:10F85000F9E1901812E0F47003A3E0F47057EC4F54
:10F860006068740A122E617403F07402122BE312A2
:10F87000353190180BE0F5087808122B7E740312CE
:10F880002BEB7401122E6112FF3290180BE0F9126B
:10F8900041437401122B8DE9F50870197D007C003D
:10F8A0007900EEFAEFFB1239D590815212299D12A0
:10F8B000FAB2122B8D851882851983E0FCA3E0FD36
:10F8C000AA0879E112359102F9FF750802740A124B
:10F8D0002E617402F0122E6174FFF0A3F012FA0E82
:10F8E000A3A3A31229A588828983A3A3A3A3A3A367
:10F8F000A3A3A3E0FC7402122BE379011238E57490
:10F9000002122B8DE9602F7508007808122B7EE417
:10F91000F50AF50B780A122B7A7808122B7E7404FC
:10F92000122BDB880A890B780A122B7A12FA091239
:10F9300029A57901805712FA0E1229A58882898398
:10F94000A3A3A3A3A3A3E0FC7402122BE3790112E7
:10F9500038E57402122B8DE9700302F8B5750800C2
:10F960007808122B7E7401122BDB880A890B780A27
:10F97000122B7A7508017808122B7EE4F50AF50B34
:10F98000780A122B7A12FA091229A579007CFF7DD8
:10F99000FF740A122BE31239E17408122B8DE9F57A
:10F9A00008E508600302F8B5901A17E0F50CA3E02B
:10F9B000F50DE4F50EF50F780C122B727A007B2012
:10F9C00090181112FAB9122B8D851882851983E0CF
:10F9D000F8A3E0F9901812E8F0A3E9F08021124AA8
:10F9E000CD7C0085188285198312FF38124A6DEA92
:10F9F0004B70EB90815212299D12FAB2122B8D742A
:10FA00000B122B8D7F0802281912FB7FA32290185E
:10FA10000EE0F8A3E0F98882F583A3A3A3A3A3A330
:10FA2000A32274F712259374F7122C0B7408122E6C
:10FA3000617402F0851882851983EAF0A3EBF07DEA
:10FA4000007C00AA18AB19123A4D7409122B8D02D2
:10FA5000FCA774F4122593E9FE7A007B40901811FC
:10FA6000E0F91234EFEE700512FF8780407A011240
:10FA7000FF8974FF6E6036EEC3944140027E40EE13
:10FA8000F50875F0E8A4C508A8F075F003A428F8F7
:10FA9000E428F5093395E0F50AF50B7808122B7286
:10FAA0007A007B4090181112FAB9122B8D7F040254
:10FAB00028197A007B01901879E0F91234E3740474
:10FAC0002274F412259374F4122C0B8C088D09E91E
:10FAD000FF741B122E61E0FE74FE6A700374FF6BEC
:10FAE00070097408122E61E4F0801D851882851952
:10FAF00083EAF0A3EBF07408122E617402F0124452
:10FB0000D9E96004EEC2E4FE740A122E61E4F0A3A7
:10FB1000F012FB7FE0C0E07409122E61D0E0F074B7
:10FB20001C122E61E0F50A780A122B7E741B122B30
:10FB3000DB880A890B780A122B7A741B122E611249
:10FB400029A5EFF50A750B00780A122B7A780812AE
:10FB50002B7AEEF97C0B7D187409122BE3124B39CA
:10FB60007409122B8DE9FA600E741A122E61E0FCF2
:10FB70007D0079E0123591740C122B8D02FAAD12D2
:10FB8000FB832290180EE0F8A3E0F58388822274AC
:10FB9000F6122593E9FEEAFF8C088D09E9FA7B004D
:10FBA00012349BEAF9EFC399500479018020780858
:10FBB000122B7AEAF5087509007808122B7A7C0076
:10FBC0007D00EEFA7B001234A77404122B8D80297D
:10FBD00074F61225938C088D097808122B7AEAF5B1
:10FBE000087509007808122B7A7C007D00E9FA7B01
:10FBF000001234A17404122B8D7F0202281974F5AF
:10FC0000122593E9601714601C14602114602614F7
:10FC1000602B14603014603F14604E806675087C61
:10FC2000750918802675084075090D804275086BA6
:10FC300075091A802875086E75091A802075087074
:10FC400075091A802A75086D75091A750A007808F1
:10FC5000122B767C01802275087875091A750A00C6
:10FC60007808122B767C02801075088C75091A753D
:10FC70000A007808122B767C087D00123357740333
:10FC8000122B8D7F0302281974F7122593E9FE7455
:10FC9000016E70097D007C0079001239D5800874EE
:10FCA000F71225931231EF7F0102281974F71225FC
:10FCB000931231F580F174F212259374FF122C0B1C
:10FCC000890A8A088B09EB5480700302FDCF800FEC
:10FCD000A3E0F91231E9EEFAEFFB123381A90A121F
:10FCE00033938A0C8B0DAE0CAF0DEE4F700302FDFB
:10FCF000C78E828F83E024E6603D244960741470CF
:10FD00000302FDA514601624F3700302FDAE147007
:10FD10000302FDB81460B924E5600B80B9EEFAEF78
:10FD2000FB12358580B0A3E0FA8E828F83A3A3A354
:10FD3000E0F9123573809FEE2422F582E43FF583CB
:10FD40001229A5EE2420F582E43FF5831229A58E21
:10FD5000828F83A3A3A3A3E0FCA3E0FD8E828F8305
:10FD6000A3A3A3A312FF301232077404122B8D0237
:10FD7000FCD6A3E0640660148E828F83A3E0640740
:10FD8000600A8E828F83A3E064097005790002FC0B
:10FD9000D38E828F83A3E060076401600302FCD6E8
:10FDA000792202FCD312FF301231FB02FCD6A3E011
:10FDB000FA8E828F8302FD2EA3E0F98E828F83A3B9
:10FDC000A312FE3E02FCD6AA08E50964808060EB1F
:10FDD0005440600B12FF87AA08E50964408050EB8D
:10FDE00054206018792190181212FE3E9018127457
:10FDF000FFF0A3F0AA08E50964208033EB54107AE1
:10FE000000602F7908124A8BAC18AD197A0179037A
:10FE100012FE47A2E2500512353D800D7CF47D01B3
:10FE20007B327A007902124A85AA08E5096410FB40
:10FE300080027B007401122B8D7F06022819E0FAE4
:10FE4000A3E0FB1235792212355B85188285198370
:10FE5000E02274F612259374F7122C0BEA240CF5A9
:10FE600082E43BF583E0F508A3E0F5097808122762
:10FE7000CD0000020000807FFE06809CFE2BFF125A
:10FE8000399F8A828B83E5822403FCE43583FDA3BA
:10FE9000AA82AB83790112320102FF2B1239A58AA3
:10FEA000088B09AE08AF09901812E0F47003A3E0C4
:10FEB000F460787408122E61740212FFC6E0F8A391
:10FEC000E0F9851882851983E8F0A3E912FFC6A33B
:10FED000A3A3E0F5087808122B7E7401122BEB9097
:10FEE000181212FF381241437401122B8DE9703B36
:10FEF0007A007B20901811E0F91234EF90815212B1
:10FF0000299D12FAB2122B8D7D007C0079008E8221
:10FF10008F8312FF311239DB790090181212FF32F1
:10FF20001231F590181274FFF0A3F0740902FBF679
:10FF3000A3A3E0FAA3E0FB22E0FAA3E0FB12FF4157
:10FF40002212FB83E0F92274F7122593E99018112D
:10FF5000F090181274FFF0A3F090180C7411F0A335
:10FF60007418F090180BE4F0FA12FF897A007B8085
:10FF7000901811E0F9123A7D7A067B80901811E012
:10FF8000F9123A7D02FCA77A0012FF41124B1522AA
:10FF900074F412259389088A09ECFEEDFF7A047B3C
:10FFA0000012337BEA4B601B8A828B83E508F0A347
:10FFB000E50912FFC6A3EEF0A3EFF0901811E0F9E7
:10FFC00012338702FAADF08A828B83A322C082C0EB
:10FFD00083851882851983E0F8A3E0F9E849601267
:10FFE0008A828B83ECF0A3E824FF18E934FFF948F8
:10FFF00070F2D083D082022B22022B22FFFFFFFF60
:020000040001F9
:10000000C082C083790012CFA2C082C0839019FD44
:1000100012C856D083D082C3E09CA3E09D500DEA65
:10002000240B12804F12802F60027901029E4BEA4E
:1000300075F00BA4FAA8F075F00BEBA428FB90194F
:10004000FFE02AF8A3E03B8882F583E0540F22F515
:1000500082E43B12B98B2274F7122593890812B0FF
:10006000A41283B7ACF075F00BE9A42CF99019FF3A
:10007000E028F8A3E039F9E8FEE9FF7401650860BB
:10008000067402650870228A828B8312856D740261
:1000900065087021EA2403FA50010B123CF9E9705B
:1000A000148E828F83E4F0800CEA2403FCE43B127C
:1000B0008564123CF38E828F83E0D2E7F01237C55D
:1000C00002AC5A74F412259312863E79008E828F08
:1000D00083E06078890A890B8063E50A75F00BA4D8
:1000E000FAA8F075F00BE50B12803B7048E50A7535
:1000F000F00BA4F8AAF075F00BE50B1285818E8247
:100100008F83E085088285098312A5321284E2EE8E
:100110002403FCE43F1281FA123CF312AEA8E50A74
:10012000F0A3E50B129B68D2E7F01237C579019076
:1001300019FD12943B050AE50A7002050B9019FDA2
:1001400012C08EC3E50A9AE50B9B408E029B727427
:10015000F5122593EAFEEBFF750A01740B122E616E
:1001600012CCB3EC4D6015EC12BD583D12864C79A3
:1001700001123CDBE508450960758023E508450967
:10018000604412BD56350912864C1281FB123CF9AF
:10019000E96401701BEEFAEFFB123CE1E9F50A8518
:1001A00008828509831284DA7902AA08AB098011D2
:1001B000128565123CF9E9640170347903EEFAEFB7
:1001C000FB123CDB80298E828F83A3E064FE7003E8
:1001D000A3E0F4700B128565123CF9E96401700C20
:1001E000EEFAEFFB123CE1E9F50A8003750A000222
:1001F0008CCBE50A2403FCE4350BFDE5082403FA67
:10020000E43509FB2274F71225939019FD12AFD83B
:10021000EA4B602FEA75F00BA4FAA8F075F00BEB2F
:10022000A428FBEAFEEBFF12341D9019FF12AFD891
:100230009019FF12ADED6012EEFCEFFD7900123364
:100240006380079019FFE4F0A3F002AC5AC082C0AB
:1002500083EC4D600512353180097C087D00790002
:10026000123363029E4BC082C0837900EA4B601652
:100270007800E8FCEA2C12B0B06004790178080834
:10028000E8C3940840EC029E4BC082C0837901EC25
:100290006A7002ED6B6011EA4B600BEC4D60071267
:1002A000352BE9F980027900029E4B74F7122593F1
:1002B00074F3122C0BECFEEDFF851882851983E494
:1002C000F004122E61EAF0A3EB12C14E123D1D7430
:1002D00003122E61AC82AD83EEFAEFFB123CF3EE1B
:1002E000FAEFFB123CF902AC5574F712259374F344
:1002F000122C0BECFEEDFF851882851983E4F0EAE1
:10030000FCEBFD7403122E61AA82AB83123CF3AAAC
:1003100018AB19123D237401122E6112A5438E826F
:100320008F8312AF9474FE68700374FF6960047960
:10033000018002790002AC5574F7122593EAFEEBB6
:10034000FF123CD5E9F5087401650870111283A20B
:10035000F4FA88828983E05A4480F01237C5A908EC
:1003600002AC5A74F7122593EAFEEBFF7508008E73
:10037000828F83E0602A123CD5E9F5087401650894
:10038000701E1283A2FA88828983E05A70128E82CC
:100390008F83E04480FA88828983E04AF01237C56F
:1003A00080BC12AD1CF81283B7128759F8A3E0394C
:1003B000F98E828F83E022A3E0F9E875F00BA4F8B0
:1003C0002274F41225938A088B097C007D00EA12BE
:1003D00081FD123CF3E5081284FC790085088285D2
:1003E0000983A3E064FE7003A3E0F460787E007FDD
:1003F000008065EEFAEFFB12802F6057EEFAEFFBFC
:10040000EA75F00BA4FAA8F075F00BEBA428FB90AA
:1004100019FFE02AF50AA3E03BF50B850882850960
:100420008312C08D850A82850B83A3E06A7003A3C3
:10043000E06B701FE50A2403FAE4350BFB123CF96C
:10044000E9640170061281F2123CF31284F1790121
:1004500012C9BD0EEE70010F9019FD12C08EC3EED1
:100460009AEF9B408E029B7274F31225938A088B3D
:10047000098A828B831284DAEA1284FC750C00EA02
:100480001281FD123CF9E9640170477E007F008013
:100490003C12874BFAA3E0398A82F583E0540F605F
:1004A0002712874BF50AA3E039F50B1281F21235BA
:1004B0002BE964017012850A82850B831284E21293
:1004C00084F1750C0112C9BD0EEE70010F12876820
:1004D00040BFA90C7F05022819A3A374FEF0A30452
:1004E000F022A312AC46850882850983A312A24B91
:1004F00022E508128506EEF0A3EFF02212850674BD
:10050000FEF0A304F022240BF582E43509F58322E2
:1005100074F5122593EAFEEBFF8E828F831284DA44
:100520007C007D00128565123CF3EEFAEFFB123C75
:10053000D5E9F50A7401650A702712AC3F1285757A
:10054000850882F58312856D1281FB123CF9E964FE
:1005500001700EE5082403FCE43509128564123CA1
:10056000F3028CCBFDEE2403FAE43FFB22A312C07E
:100570009C12A24B22E875F00BA4F8AAF075F00BC0
:10058000E912875FF508A3E039F5092274F2122514
:100590009374E6122C0B12863E750A0175080075DD
:1005A0000900750C00750D00851882851983E4F02B
:1005B000EE2403FCE43FFD7403122E61AA82AB8398
:1005C000123CF3AA18AB19123D23E96401701F74A1
:1005D0000B122E6112864E7401122E6112C096709B
:1005E00003A3E069604AA818A91988088909740D4D
:1005F000122E6112A531A312A543740E122E6112A0
:10060000AF94740D122BE3123D1DE964017009745F
:100610000D122BDB880C890D780C122B7AAC08ADEF
:1006200009EEFAEFFB123CE77402122B8DE9F50A92
:10063000EEFAEFFB123D17A90A741A02AEBAEAFEEF
:10064000EBFF12AEAC74FEF0A304F022F58312C0EF
:100650007CF912AEAC12A24B22C082C08378007922
:1006600000800508E87001099019FD129850E99B77
:100670005029E8FAE9FBEA75F00BA4FAACF075F042
:100680000BEBA42CFB9019FFE02AFCA3E03B8C822F
:10069000F583E0540F70CC790080027901029E4B03
:1006A00074F61225937E007F008039EEF8EFF91280
:1006B00085757808122B7A75080B75090078081271
:1006C0002B7AEEFCEFFDEC75F00BA4FC75F00BED56
:1006D000A42AFD7A237B001234A77404122B8D0EFA
:1006E000EE70010F12876840C2028BE374F6122588
:1006F000937E007F00804C12874BF8A3E039F98885
:10070000828983E0A2E75036C2E7F08582088583BC
:10071000097808122B7A75080B7509007808122BD6
:100720007AEEFCEFFDEC75F00BA4FC75F00BEDA47C
:100730002AFD7A237B001234A17404122B8D0EEE55
:1007400070010F12876840AF028BE3EEF8EFF9E813
:1007500075F00BA4F812875922AAF075F00BE9A4E2
:100760002AF99019FFE028229019FD12AC46C3EE39
:1007700098EF992274F6122593E4F508F5097808A4
:10078000122B7A9019FD12943675F00BA4FCA8F088
:1007900075F00BEDA428FD7A237B001234957402CA
:1007A000122B8DE9FE6003123D4D02C6B274F612A3
:1007B000259374FF122C0B7E007F00803C851882ED
:1007C000851983E412919E122B7A75080175090030
:1007D0007808122B7AEEFCEFFDEC75F00BA4FCA868
:1007E000F075F00BEDA428FD7A237B001234A17480
:1007F00004122B8D0EEE70010F12876840BF74013A
:10080000028BE0C082C083905156E49375F01CA423
:10081000FCADF079FF7AF37B05123363029E4B74D3
:10082000F7122593E9FCEAFD7A007B008010EB12B9
:100830008E799C4008E0F8EDC39840010A0B905176
:1008400056E493F8EBC39840E57B0002AC5A74EC95
:1008500012259374F3122C0B8A0C8B0D8C088D09C6
:10086000890AEC45096016AA08AB09123D838A0E75
:100870008B0FAE0EAF0FEE4F600302894C7A0080F3
:10088000010A90515612BFD3500F128A4170F27470
:10089000F328FE740539FF80047E007F00EE4F7060
:1008A000030289F590513B128A1260257403650A90
:1008B00060067404650A70197A047903123D598A36
:1008C0000E8B0F905156E493F890513B128A2B50A7
:1008D0002D905135128A12602C7401650A600674DD
:1008E00002650A70207A027901123D598A0E8B0F37
:1008F000905156E493F8905135128A2B40077A00B4
:100900007B00028A0D8518828519837401F0122EEE
:1009100061E50CF0A3E50DF0AC08AD097403122EEF
:1009200061AA82AB83123CF3AA18AB19123D2F7453
:100930000B122E6112A2448E828F83A3A3A3A3A3C2
:10094000A3E412C852AA0CAB0D1245C37800E50A05
:100950006007C39405500278048E828F83E50CF003
:10096000A3E50D128D3CA3A3E50AF0E88E828F83E8
:10097000A3A3A3A3A312C3635001097A027B0012AD
:10098000233712982BA3129CCA129857E50A605B72
:10099000C394035056901CCBE07018905014780C00
:1009A000122D3A129802122DF2905014780C122D3A
:1009B0003A8027F50875090074027808122D141280
:1009C0008A1C122D3A90813E7810122DD4780C7921
:1009D0001012242E129802122DF2EE2413129805F2
:1009E000122DF2EE241B12C35A800912980E1284A3
:1009F000DDA3F0A3F07A047900123D59128D2D4049
:100A000005901CE4E4F0124485EEFAEFFB740D024D
:100A1000A051E493F8740193F9E84922741425086D
:100A2000F58274503509F583780C22E493FA740149
:100A300093FBE8C39AF8E49BF9C3E50E98E50F9998
:100A400022EA128A47F42275F01CA4F8A9F074F780
:100A500028F582740539F583E02274EE122593742B
:100A6000F3122C0BEAFEEBFF8C108D11750800AA17
:100A700010AB11123D83EA4B7003028B758A828B97
:100A800083E06E7003A3E06F7003028B758A828B24
:100A900083A3A3A3A3E0C394054003028B758A82BA
:100AA0008B8312C9ABE060728A828B83A3A3A3A35A
:100AB000E0C394035064901CCBE0702190501478F4
:100AC00008122D3A128B7C122DF2905014780812D5
:100AD0002D3AEA2413128B7F122DF28030F508751F
:100AE000090074027808122D14128A1C122D3A90F3
:100AF000813E7808122DD4780C790812242E129A8F
:100B00002C122DF2EA2413129A2F122DF2EA241B32
:100B1000F582E43BF583E4F0801B7508FE7509FF60
:100B2000750AFF750BFF128B7C122DF2EA2413124B
:100B30008B7F122DF2750800750900750A00750B80
:100B400000EA240C128B7F122DF2851882851983FE
:100B50007401F0122E61EEF0A3EFF0AC10AD117441
:100B600003122E61AA82AB83123CF3AA18AB1912AE
:100B70003D2F750801A908740D02C9A3EA2417F5D1
:100B800082E43BF58378082274F6122593123D7DAA
:100B90008A088B09A808A909E84960148882898312
:100BA000A3A3A3A3E06009C39405500479018002C4
:100BB0007900802F74F6122593123D7D8A088B09E7
:100BC000A808A909E849601488828983A3A3A3A37C
:100BD000E06009C394035004790180027900800326
:100BE000122B8D7F0202281974F6122593123D7D77
:100BF0008A828B83E5824583600BA3A3A3A3E07065
:100C00000479018002790080DAC082C083EAFCEBBB
:100C1000FD7A007B00029E48C082C0837C007D007C
:100C2000029E4874F512259374F3122C0BEAFEEB26
:100C3000FF8C088D09C3EC94F8ED94FF4004EE4F4F
:100C40006065750A00801974FF6508700474FF659B
:100C500009600B12CF9C7004A3E06509603B050A94
:100C6000905156E493F8E50AC398503BE50A128A7E
:100C70004260EBEE4F60D0128CB2122E6112C14A6C
:100C8000123D29E960D87403122E61AC82AD83EE67
:100C9000FAEFFB12352BE960C5E50A75F01CA4F8E4
:100CA000A9F0128E7080047A007B00740D122B8DD7
:100CB000801B8518828519837401F074F528F582EC
:100CC000740539F58312AC46740B22A90A7F03021E
:100CD000281974F412259374F3122C0B7508001262
:100CE0003D838A0A8B0BAE0AAF0BEE4F6025851849
:100CF00082851983128D3A128CC5122E6112C14A57
:100D0000123D117C1C7D0079FFEEFAEFFB1233637C
:100D10007508017A047900123D59128D2D50099001
:100D20001CE47401F0124485A908029B6D90515691
:100D3000E493F8C3EA98EB940022740112A536A359
:100D4000A32274F7122593E9FE74FE6A700374FF00
:100D50006B7C00700380240C128DA5501EEC128A4F
:100D60004260F4128F3F7003A3E06B70EA800BECDB
:100D7000128DBA6019E0640360140C128DA5501E28
:100D8000EE60ECEC128DAF60F1C3940550ECEC75A5
:100D9000F01CA4FCADF012D51212C08E80047AFEB5
:100DA0007BFF02AC5A905156E493F8ECC39822753D
:100DB000F01CA4F8A9F0128A4E2275F01CA4F8A920
:100DC000F0128A4E640122123D95029E4BC082C0F1
:100DD00083790180F274F01225938A0A8B0B7A04CE
:100DE0007901123D598A0C8B0DEA450D6040EA2AC3
:100DF000FAEB33FB12341D8A088B09AE08AF09EEFB
:100E00004F60267AFE7BFF123D9B74FE6A7003746E
:100E1000FF6B601E85088285098312AFD8E5082420
:100E200002F50850E2050980DE750C0080047E00A2
:100E30007F00850A82850B83E50CF0EEFAEFFB025A
:100E40009106C082C0837C008009EA24FF1AEB343B
:100E5000FFFB0C128DA55011EC128E79940550F207
:100E6000EA4B70E6128E7080047A007B00029E4B83
:100E700074F328FA740539FB22128A47C32274F7E7
:100E800012259374F3122C0B7E00807DEF75F01702
:100E9000A4F8A9F0128F3012C08EEE75F01CA4F8E1
:100EA000A9F0128F3F7003A3E06B603DEF75F01760
:100EB000A4F8AAF0EAF9128F3012A5437401122E99
:100EC00061E0687003A3E069601FEF75F017A4F894
:100ED000EAF9745928FC740939FD7403122E61AAC9
:100EE00082AB8312352BE96013EF75F017A4F8A9D4
:100EF000F0745728FA740939FB1245CF0F90514905
:100F0000E493F8EFC39840840E12D4FF501FEE1202
:100F1000DA7DF47003A3E0F460EE128CB2122E615D
:100F200012C14A123D29E960DF7F0080D002AC5532
:100F3000128F3422745728F582740939F5832212EE
:100F4000DA886A2274F412259374F3122C0B7E0053
:100F5000803890815E7808122DD4EE75F01CA4F8CC
:100F6000A9F0740628F582740639F5837808122CE6
:100F70006260169081127808122DD4EE75F01CA4D0
:100F8000F812900C7808122CC80E12D4FF507AEE8A
:100F9000128DAF60F4C3940350EF12900C122E0E1A
:100FA000E8494A4B70AC9019D6E06401702D901B53
:100FB0000612ADED6025EE75F01CA4F8A9F074F3EF
:100FC00028F8740539F912906212299D8882898364
:100FD0001290F71227797404122B8D8518828519C7
:100FE000837401F0EE75F01CA4F8A9F0128CBB120A
:100FF0002E6112C14A123D29E9608E7403122E61DE
:10100000AA82AB83123D8F8080029B6D740A28F503
:1010100082740639F5832274F6122593123D7D8A77
:10102000088B09A808A909E849603288828983A346
:10103000A3A3A3E06023C39403501E129062122E58
:101040001AE82417F582E439F583122E3EE8241BB2
:10105000F582E439F5837401F079018002790002A8
:101060008BE3E82413F582E439F5832274F012252A
:1010700093EAFEEBFF901B0012ADED6072901B0631
:1010800012ADED606A901B0A12ADED606212D38B57
:10109000122779E97059901CCBE0700A90501478AF
:1010A00008122D3A8028F508750900740278081294
:1010B0002D1412D56D745012D36C7808122D3A90FD
:1010C000813E780C122DD47808790C12242E7808E1
:1010D000122B721290F11227797404122B8DE9648D
:1010E00001700C8E828F83A3A312D379122779808B
:1010F000158E828F83A3A312B98D901B0612D38302
:1011000022740D122B8D7F0802281974F612259374
:10111000E4F508F5097808122B7A905156E493F516
:101120000874037808122D1412942812349574024E
:10113000122B8DE9FE740A6E6025E4F508F5097836
:1011400008122B7A905156E49375F005A4FCADF08B
:101150007A3F7B001234957402122B8DEE600312DD
:101160003DCB02C6B274F612259374FE122C0B8589
:101170001882851983E4F0A312919E122B7A7508C8
:10118000027509007808122B7A7C007D007A227B98
:10119000001234A17404122B8D7402028BE0F0A8AB
:1011A00018A9198808890978082274EE1225937401
:1011B000DE122C0B8A0E8B0F8C088D09750C007AB1
:1011C000227B0012349B8A0A8B0B7A3F7B001234FD
:1011D0009B8A108B11AE10AF11E50A450B6017E525
:1011E00008650A7004E509650B600BAC0AAD0B7A63
:1011F000227B001234AD7436122E6112943BEE4FF6
:101200006015E50A6E7003E50B6F600BEEFCEFFDF9
:101210007A3F7B001234ADE4F510F5117810122BF3
:101220007AAC08AD097A227B001234957402122B35
:101230008DE9640A700302941EE4F508F509780844
:10124000122B7AAC0AAD0B7A3F7B001234957402F4
:10125000122B8DE9640A700302941E7404122BDBB6
:10126000880889097808122B7A75080275090078B0
:1012700008122B7A7C007D007A017B031234A7745C
:1012800004122B8DE9600302941E85188285198350
:10129000E4F0A3F07E000293957406122BDB88081D
:1012A00089097808122B7A750808750900780812E0
:1012B0002B7A8E0874037808122D14E5082402FC9A
:1012C000E43509FD7A017B031234A77404122B8DD7
:1012D000E9600302941E7408122E61E0F47003A307
:1012E000E0F470030293947406122BDB88088909DA
:1012F0007808122B7A7508087509007808122B7A7D
:101300007404122E6112CCB374037808122D1412D7
:1013100094281234A17404122B8DE9600302941EE8
:101320007402122BDB880889097808122B7A750859
:10133000057509007808122B7AEE75F005A4FCAD4E
:10134000F07A027B031234A77404122B8DE97041EA
:101350007402122BDB880889097808122B7A750829
:10136000057509007808122B7A7404122E61129404
:101370003675F005A4FCA8F075F005EDA428FD7AFB
:101380003F7B001234A17404122B8DE96003029498
:101390001E1299440E851882851983C082C08390DD
:1013A0005156E493F8D083D082C3E098A3E0940030
:1013B0005021851882851983C082C0837404122E3F
:1013C0006112A543D083D082C3E098A3E099500373
:1013D000029299A818A919880889097808122B7A05
:1013E0007508027509007808122B7A7C007D007A56
:1013F000227B001234A17404122B8DE97020AC0EF4
:10140000AD0F7A017B031234ADE970127434122EE1
:101410006112C8567A027B031234ADE96003750C81
:1014200001A90C742202C9A3E5082402FCE43509D1
:10143000FD7A227B002212C85AEC22E0F50AA3E0D2
:10144000F50B2274EC12259374FE122C0B750A0016
:10145000851882851983E4F0A3F090515693F50E18
:10146000F50875090074037808122D14E5082402A4
:10147000F50850020509E50E75F005A4F50EE5F036
:10148000F50F7A227B0012349B8A0C8B0DAE0CAFC9
:101490000D7A3F7B0012349B8A108B11A818A91972
:1014A000880C890D780C122B7A750C02750D00785A
:1014B0000C122B7A7C007D007A227B001234A774F8
:1014C00004122B8D7A017B0312349B8A0C8B0D7ACC
:1014D000027B0312349B8A128B13A812A913E50C0A
:1014E000450D700AE5086E7003E5096F7025E8493F
:1014F000700CE50E65107004E50F65117015E50CB4
:10150000450D607BEE4F604E85188285198312AFC2
:10151000DE60437C017D037A227B00124659E9F8A4
:10152000880A705B7C027D037A3F7B00124659E992
:10153000F8880A704AEEFCEFFD7A227B001234AD87
:10154000E9700EAC10AD117A3F7B001234ADE9604A
:1015500011750A018029AE0CAF0DE84960048810AE
:101560008911780E122B7A7810122B7AAC08AD09FB
:10157000EEFAEFFB123DD17404122B8DE9F50AA9A6
:101580000A740202A05174EC12259374D0122C0B31
:10159000851882851983E4F0A3F0123DD7E9600332
:1015A0000297EAA818A919880889097808122B7ADD
:1015B0007508027509007808122B7A7C007D007A84
:1015C000227B001234A77404122B8DE9600302976A
:1015D000EA905156E493F885188285198312985041
:1015E000E49B50030297EA750A00750B007508002A
:1015F000803D7403122E61122E0E129821122E4A73
:101600007403122E61122E0E12A868122E4AEE24B6
:101610001BF582E43FF583E4F07A047900123D592A
:10162000128D2D4005901CE4E4F01244850508124B
:1016300097F740030297EA12A53DC3E50A98E50B28
:101640009940030297EA7414122BDB880C890D78F9
:101650000C122B7A750C08750D00780C122B7A85FC
:10166000080C7403780C122D14E50C2402FCE435EC
:101670000DFD7A227B001234A77404122B8DE970C1
:10168000AC7416122E61E0F47003A3E0F4609E05C2
:101690000AE50A7002050B7407122E617401F074DA
:1016A00016122E6112A5437412122E6112AF947499
:1016B00007122BE3123D29E9700302962D12C8533D
:1016C0007414122E6112C08E1245C3E50875F01C09
:1016D000A4F8A9F074F328FE740539FF7414122BD2
:1016E000DB880C890D750E00780C122B767C087D3A
:1016F00000EEFAEFFB1233577403122B8D12C368FE
:101700005001097A027B0012233712982B12985746
:101710007402122BDB880C890D780C122B7A750C55
:1017200005750D00780C122B7AE50875F005A4FC00
:10173000ADF07A3F7B001234A77404122B8DE96060
:1017400003029619908112780C122DD47403122E74
:1017500061780C122C6260030295F2E50875F01CAA
:10176000A4F8AAF0EAF9128DB66071C39403506C24
:10177000901CCBE07018905014780C122D3A1298EF
:1017800002122DF2905014780C122D3A8033F50C81
:10179000750D007402780C122D147414250CF5824A
:1017A000745012B95B780C122D3A90813E78101269
:1017B0002DD4780C791012242EEAF9129802122DE9
:1017C000F2EE2413129805122DF2E50875F01CA410
:1017D000F8740E28F58274063902961512980E04D4
:1017E000141284DDA3F0A30296188518828519834C
:1017F000E0F9743002A051905156E493F8E508C323
:101800009822EE2417F582E43FF583780C22129893
:101810002174FEF0A304F0A3F0A3F012A86C74FEF0
:1018200022EE2417F582E43FF58322E88E828F832F
:10183000A3A3A3A3A3A3A3A312AC1A740112AC1A6B
:10184000A374AAF0EE2410F582E43FF583E4F022BD
:1018500012B98DC3E89A22A3F012AEACE4F0EE24E4
:101860000CF582E43FF583E4F0A3F0A3F0A3F022AB
:1018700074F212259374FE122C0B8518828519833D
:10188000E4F0A3F075080002990FE50875F01CA4B8
:10189000F8A9F074F328F50C740539F50DAE087845
:1018A0000C122B7A750A08750B00780A122B7A8EA7
:1018B0000A7403780A122D14E50A2402FCE4350B9D
:1018C000FD7A227B001234A17404122B8DE50C24C6
:1018D00012F50AE4350DF50B780A122B7A750A0514
:1018E000750B00780A122B7AEE75F005A4FCADF0AA
:1018F0007A3F7B001234A17404122B8D850C8285F3
:101900000D83A3A3A3A3E0F4600312994405081276
:1019100097F7500302988AA818A9198808890978A6
:1019200008122B7A7508027509007808122B7A7C48
:10193000007D007A227B001234A17404122B8D7476
:101940000202AEBA851882851983E02401F0A3E073
:101950003400F02274F012259374F3122C0BEAFE7B
:10196000EBFF7A027901123D59EA8E828F83F07083
:1019700003029A1F75F00CA4FAABF012341D8A080A
:101980008B09EA45097003029A25AE08AF09750A6A
:1019900000801C90811212299DEEFAEFFB1233DBBE
:1019A0007404122B8D8A0C8B0DAE0CAF0D050A90B2
:1019B0005156E493F8E50AC398506AE50A128DBAC5
:1019C0006005E0640270E6128CB2122E6112C14A08
:1019D000123D29E960187403122E61AC82AD83EECA
:1019E000FAEFFB1235318A0C8B0DAE0CAF0DE50A08
:1019F00075F01CA4F8A9F0740E28F582740612D1B3
:101A0000EA6401708E128E70EA2413129A2F122D3E
:101A1000D4129A2C122BF3780C122B72029999750E
:101A20000800750900AA08AB09029101EA2417F51C
:101A300082E43BF583780C22C082C083901A08743C
:101A40003BF0A37443F0901A0A7435F0A37443F08A
:101A5000901A0E748BF0A3743EF0029E4BC082C0AD
:101A600083901A0C742FF0A37443F0029E4B74F70A
:101A7000122593EAFEEBFF901A7AE06408601FE0FB
:101A80006404601A8E828F83E054036401704412F0
:101A9000AD18F8A3E0F5838882E0640670358E8285
:101AA0008F83A3A3E064FE7003A3E0F460258E821D
:101AB0008F83A3A312C8637003A3E0697008EE24A8
:101AC0001512C84A60051244018003124407E9F563
:101AD0000880037508C2EEFAEFFB12342302835E1E
:101AE00074F41225938A088B098A828B83E0FAA307
:101AF000E0F8EA28FAE43400FB12341D8A0A8B0B62
:101B0000AE0AAF0BEE4F605A850882850983E0FC70
:101B10007D0079001233638E828F831284D9124440
:101B20003D8E828F83A3A3A3A3EAF0A3EB129B684D
:101B3000F8EE28F8E43F128651850882850983A3D0
:101B4000E0C0E012C34DD0E0F012444FEE240EF599
:101B500082E43FF583E912A4BEE0C0E012A216D0F1
:101B6000E0F0EEFAEFFB800A12A4B6E022740D1248
:101B70002B8D7F0402281974F412259374E8122C1B
:101B80000B8A088B098C0A8D0BE9FE901A7AE064A7
:101B9000046005E06408700479C2804BA3780812E1
:101BA0002DF2EE901A81129CCF1233638518828534
:101BB00019837808122DF27405122E61EEF0740468
:101BC000122E617401F07407122E61E4F0901A7AFB
:101BD0007402F09019E8E0640270059019D6E4F000
:101BE000AA18AB19123C3F7418808474F412259320
